:020000040800F2
:10000000000001107530040885FB03084910010841
:1000100079310408793104087931040800000000BE
:10002000000000000000000000000000D1010408F2
:10003000CD01040800000000C901040849DC0008E3
:1000400079310408793104087931040879310408D8
:10005000793104087931040851F2010805F30108E7
:10006000C9F201088DF2010815F2010869A400081F
:1000700059A4000849A4000839A4000829A40008CC
:1000800015A4000801A40008793104087931040896
:10009000793104087931040879310408A9E40008A9
:1000A0007931040835D300087931040845D30008B4
:1000B00025D3000815D3000879310408F5BD0008E0
:1000C000FDBD0008E5BD0008EDBD0008793104085C
:1000D00079310408BDDD0008793104081DDD000810
:1000E0006DE4000879310408C50404087931040876
:1000F000E5D2000879310408F5D20008EDA3000824
:10010000793104087931040805D3000879310408ED
:1001100079310408793104087D9002086190020861
:10012000D9A30008C5A30008B1A300089DA3000837
:1001300089A3000879310408793104087931040869
:1001400079310408793104087931040889FB0308FE
:1001500075A3000861A300084DA300087DDC00081A
:10016000D5BD0008DDBD00087931040879310408E7
:1001700079310408793104087931040879310408A7
:0801800079310408793104080B
:080188000C2C04000100000032
:1001900002020300141F0020101F002000000000B6
:1001A0000000000016000800342400204C24002029
:1001B00000000000400600081D000100102600207D
:1001C00098260020000000004806000827000400D0
:1001D000302600209C260020000000004A0600086F
:1001E00001010400E82600204C3600200000000039
:1001F000000000000802090074350020503600207D
:10020000000000009DEA010806020C00EC35002009
:100210005C360020000000006DF0010807020200BB
:100220002036002068360020000000004E0600083E
:10023000FF010100443600206C3600200000000061
:100240005006000802000C00F8350020703600202F
:100250000000000000000000F701060068350020E3
:100260007C36002000000000520600080E0202004A
:100270008C36002090360020000000005806000850
:1002800003123300DB390020A839002000000000F1
:100290005C06000825005A00F43800204E39002082
:1002A0000000000000000000F6110C00E8380020FB
:1002B000DC380020000000009006000815007000E7
:1002C000FC3700206C380020000000000000000017
:1002D0002A0060003C3700209C370020000000000E
:1002E000B5A303082C001000244000201440002077
:1002F00000000000F95302082B00240058400020A1
:100300003440002000000000C953020829005000BA
:10031000483F00207C40002000000000000000005A
:100320000A020A00C0450020D0450020000000005D
:100330009C0600081E000400DC45002060490020E7
:1003400000000000A606000822000C007C480020E7
:100350006449002000000000AA0600080B201000DD
:10036000844C0020204D002000000000B60600084C
:100370001F000E00B04A0020304D00200000000099
:10038000C606000805020100984A0020404D0020E2
:1003900000000000D406000805100600864E00206C
:1003A000084F002000000000D80600080E20EA00D8
:1003B000664D0020104F00200000000029A4030813
:1003C000130004009C4E0020FC4F002000000000A1
:1003D000E006000802010300514D002000500020FB
:1003E0000000000061CB010803000100B8510020AB
:1003F000C0510020000000000000000010000300B9
:100400002C5400203854002000000000E4060008AE
:10041000280010001C5400203C5400200000000064
:1004200005260308230010000C5400204C54002023
:10043000000000001D2603081900050004540020D8
:100440005C54002000000000E8060008F8110100DC
:10045000005400206454002000000000EE06000854
:1004600000010400FC53002068540020000000003C
:10047000F00600082F001100E85300206C54002003
:1004800000000000F406000803010A00D854002010
:10049000E4540020000000000607000814000200D9
:1004A00080580020C05800200000000010070008FD
:1004B000F9010400785D0020087B002000000000A6
:1004C000ADC00008FD012400505D00200C7B002021
:1004D000000000003DC0000806001600D0590020B2
:1004E000307B00200000000049A40308FB0101004C
:1004F0000C590020487B002000000000C9BE000805
:10050000FA010200947D0020CC7D00200000000054
:10051000F1BE0008FE010900707D0020D07D0020A2
:1005200000000000D1BE0008FC010900D88D0020A9
:10053000C48E0020000000008DBE00080A101200CA
:10054000AC8D0020D08E00200000000012070008B3
:1005500034001000FC840020E48E00200000000025
:10056000DDA3030818102C0098840020F48E0020CE
:10057000000000009D6102080D003400C4840020CA
:10058000208F002000000000A5CB01081B00F40014
:100590005C8F002014A0002000000000959202084B
:1005A00026000E0018A1002008A100200000000075
:1005B000A18A0308012008002CA700204CA70020D6
:1005C00000000000240700081A00080010A70020FF
:1005D00054A70020000000002C07000809020100B9
:1005E000E8A7002040A80020000000003407000811
:1005F00012200C008CA7002044A80020000000005E
:10060000360700080C00240098A7002050A80020FE
:100610000000000039CB0108000205006CA7002093
:1006200074A800200000000000000000040080000A
:1006300038B9002038BA0020000000000000000097
:10064000C409000019012828000020030000013C13
:100650000000180100000000000000000000000081
:10066000000000000000000000000000000000008A
:10067000000000000000000000000000000000007A
:100680000000000000000000000000000000010069
:1006900000000000000000000000000000004A010F
:1006A000B400D601000000000100C800141E0100C3
:1006B00064002C0128002B21231E6401020000008D
:1006C00001000A01290000000000000001000000F4
:1006D00000050000000000002000020100000000F2
:1006E00008000000000105000000280100000400CF
:1006F0009001000000000000000000000000000069
:10070000000000000000040101006C160000000061
:10071000030000300100005A0000000090012C018D
:10072000C8006400E8036400040A00017E05EA05CD
:10073000B405320039000000000100054659463476
:020740000000B7
:10074200500100000700000002000000000000004D
:10075200000000000102030406070809685E0C009D
:10076200FF00000001010000547B04085CA504089E
:100772000000000000000000647B04086C7B040899
:100782000000000001200000707B0408787B040850
:1007920000000000014000007C7B0408A89D0408C2
:1007A2000000000001200000887B0408947B0408FC
:1007B2000000000004000000987B0408A47B0408E9
:1007C2000000000004000000A87B0408508904080F
:1007D2000000000001000000020100000000803F54
:1007E2000000803F00000000000000000000000048
:1007F2000000803F084C04080508040000000000C7
:10080200C4680408DC6D0408B06804080000000035
:10081200344C040805080A0000000000C4680408FB
:10082200DC6D0408D067040800000000FFFFFFFF32
:100832000101D601B14D02080000000000000000D5
:1008420000FFFF0000000000AA550501000001AAF8
:10085200550B010000AA5507010000AA5509020024
:100862000000000001000000C012AA5503009F0012
:10087200010101007DC7020800000000A80200205B
:100882007CAC040800000000000000000000000032
:10089200000000005CA50408000000000000000049
:1008A2002C0300200400000028AC04080C00000007
:1008B20009CE0208481500200000000060A70408C5
:1008C2000C00000031CE02083C15002000000000A0
:1008D20068A704080800000000000000301500208E
:1008E2000400000070A704080C00000025C80208DC
:1008F200241500200000000080A704080300000067
:100902009515040818150020000000008CAC04089E
:1009120003000000951504080C15002000000000DB
:10092200BCA5040801000000000000000000000057
:1009320000000000000000000D00000000000000A8
:1009420000000000000000007CAC04080000000071
:100952000000000000000000000000005CA5040888
:1009620000000000000000002C0300200400000032
:10097200D4AB0408030000001DCC020800150020BF
:100982000800000070A704080C00000025C8020837
:10099200241500200000000080A7040803000000C6
:1009A2009515040818150020000000008CAC0408FE
:1009B20003000000951504080C150020000000003B
:1009C200BCA50408010000000000000000000000B7
:1009D20000000000000000000D0000000000000008
:1009E200000000000000000094AC040800000000B9
:1009F2000000000000000000000000005CA50408E8
:100A020000000000000000002C0300200400000091
:100A1200DCAB0408030000009515040854150020FF
:100A220000000000BCA50408010000000000000056
:100A32000000000000000000000000000D000000A7
:100A420000000000000000000000000020700020F4
:100A5200702D7200FA000000010000000100000089
:100A62000000000000000000D01000202D202D2DDD
:100A7200202D2D2D2D202D2D2D00000000000000F9
:100A8200000000000000000000000000B4A50408FF
:100A92000000000000000000000000000000000054
:100AA20095A504080400000097CB0208000000008E
:100AB20000000000BCA504080100000000000000C6
:100AC2000000000000000000000000000D00000017
:100AD200000000000000000000000000EAB9002051
:100AE2000100C40900000000E8B900200100C409A7
:100AF20000000000E6B900200100C4090000000067
:100B0200E4B900200100C40900000000E0B900209F
:100B12000100C40900000000E2B900200100C4097C
:100B220000000000DEB900200100C409000000003E
:100B3200DCB900200100C409000000000000000030
:100B4200000000004C030020B25400209CFF2C0146
:100B520000000000300100200A000000D0670408F5
:100B6200444D0020E0150C17000000003201002067
:100B720008000000DC6D04083101002005000000BF
:100B8200C4680408464D002002000000E86704081B
:100B92008C4E00200100FF7F01000000854E0020E6
:100BA20002000000F46704085A4D00200300000010
:100BB20004680408594D002003000000046804087A
:100BC200584E00200000F40101000000564E0020A3
:100BD2000000F40101000000544E00200000F40166
:100BE20001000000524E00200000F401010000004C
:100BF200504E002000FF0100704E0020E803D00795
:100C02000A0000006E4E0020006401000A0000008D
:100C12006A4E002000640100694E00200064010059
:100C22006F4E0020006401000A000000684E0020A0
:100C3200006401000A0000006D4E00200064010003
:100C42000A0000006C4E0020006401000A0000004F
:100C52006B4E0020006401000A000000674E002075
:100C620000FF01000A000000664E002000FF0100A4
:100C72000A000000624D00200000F40101000000A3
:100C8200604D00200000F401010000005E4D0020D4
:100C92000000F401010000005C4D00200000F4019E
:100CA20001000000624E00201400E8030100000071
:100CB200604E0020E8033075010000005F4E002006
:100CC20000C801005E4E002000C801005D4E0020F9
:100CD20000C801005C4E0020006401000A00000010
:100CE2005B4E002000FF01000A0000007B4E002046
:100CF20000C801007A4E002000C80100794E002091
:100D020000C80100784E002000C80100774E002084
:100D120000C80100764E002000C80100754E002078
:100D220000C80100744E002000C80100734E00206C
:100D320000C80100E8A5040800000000000000004F
:100D42000000000000000000F8A5040809000000EF
:100D520000000000F00300200400000000A60408C8
:100D62000900000000000000E4030020040000006D
:100D7200E8A904080900000000000000D8030020D0
:100D82000400000008A6040809000000000000009A
:100D9200CC030020040000000CA604080900000097
:100DA20000000000C00300200400000014A6040894
:100DB2000900000000000000B4030020040000004D
:100DC2001CA604080900000000000000A80300207F
:100DD2000400000024A6040809000000000000002E
:100DE2009C03002004000000BCA5040801000000D0
:100DF20000000000000000000000000000000000F1
:100E02000D000000000000000000000000000000D3
:100E120038A70408000000000000000000000000E5
:100E22000000000048A704080500000000000000C0
:100E3200584D002000000000BCA50408010000007D
:100E420000000000000000000000000000000000A0
:100E52000D00000000000000000000000000000083
:100E620050A704080000000000000000000000007D
:100E7200000000005CA50408000000000000000063
:100E820060150020040000005CA704080C000000AC
:100E9200F9CB0208440400200000000028AC04083A
:100EA2000C00000035C702083804002000000000D2
:100EB20060A704080C00000019C702082C040020D7
:100EC2000000000068A704080800000000000000FD
:100ED200200400200400000070A704080C00000099
:100EE20065C60208140400200000000078A7040868
:100EF20009000000000000000804002004000000B7
:100F020080A704080300000095150408FC030020D4
:100F120000000000BCA50408010000000000000061
:100F22000000000000000000000000000D000000B2
:100F320000000000000000000000000084A7040878
:100F4200000000000000000000000000000000009F
:100F520094A704080C000000000000005C040020BC
:100F6200000000009CA704080A0000000000000026
:100F7200A04E002000000000A8A704080A000000FC
:100F820000000000A84E002000000000B0A70408E6
:100F92000A00000000000000B04E00200000000027
:100FA200B8A7040808000000000000005004002058
:100FB20000000000C0A7040804000000E9D00208F5
:100FC2000000000000000000BCA5040801000000B1
:100FD200000000000000000000000000000000000F
:100FE2000D000000000000000000000000000000F2
:100FF200CCA7040800000000000000000000000070
:1010020000000000E0A704080C000000000000003F
:101012007404002000000000F0A70408040000008F
:10102200A5CE02080000000000000000F8A7040896
:101032000C00000000000000680400200000000016
:101042000CA804080400000085CE0208000000007D
:1010520000000000BCA50408010000000000000020
:101062000000000000000000000000000D00000071
:1010720000000000000000000000000014A80408A6
:10108200000000000000000000000000000000005E
:1010920028A804080700000000000000B004002097
:1010A2000000000034A8040808000000000000004E
:1010B200A40400200000000040A80408080000006A
:1010C2000000000098040020000000004CA8040862
:1010D20008000000000000008C0400200000000056
:1010E20058A8040808000000000000008004002046
:1010F20000000000BCA50408010000000000000080
:101102000000000000000000000000000D000000D0
:1011120000000000000000000000000064A80408B5
:1011220000000000000000000F030020000000008B
:1011320070A804080B000000000000002805002031
:101142000000000078A804080B0000000000000066
:101152001C0500200000000084A804080B00000009
:1011620000000000100500200000000090A8040804
:101172000B00000000000000040500200000000039
:101182009CA804080B00000000000000F8040020E6
:1011920000000000A8A804080B00000000000000E6
:1011A200EC04002000000000B0A804080B000000BE
:1011B20000000000E004002000000000BCA80408B9
:1011C2000700000000000000D8040020000000001A
:1011D200C4A804080700000000000000D00400209A
:1011E20000000000D0A804080B000000000000006E
:1011F200C404002000000000DCA80408080000006D
:1012020000000000B804002000000000BCA5040893
:1012120001000000000000000000000000000000CB
:10122200000000000D0000000000000000000000AF
:1012320000000000E8A80408000000000000000010
:101242000000000000000000FCA8040808000000E4
:1012520000000000580500200000000008A9040852
:1012620008000000000000004C0500200000000003
:1012720014A9040808000000000000004005002036
:101282000000000020A9040808000000000000007F
:101292003405002000000000BCA504080100000085
:1012A200000000000000000000000000000000003C
:1012B2000D0000000000000000000000000000001F
:1012C20028A9040800000000000000000C03002010
:1012D2000000000038A904080B0000000000000014
:1012E200A00500200000000044A904080B00000033
:1012F20000000000940500200000000050A904082E
:1013020007000000000000008C0500200000000023
:101312005CA904080700000000000000840500200A
:101322000000000068A90408070000000000000097
:101332007C0500200000000074A9040808000000D9
:101342000000000070050020000000007CA90408D5
:1013520008000000000000006405002000000000FA
:10136200BCA504080100000000000000000000000D
:1013720000000000000000000D000000000000005E
:10138200000000000000000084A904080000000022
:10139200000000000C0300200000000090A90408D7
:1013A2000700000000000000EC0500200000000023
:1013B20098A904080700000000000000E4050020CE
:1013C20000000000A0A904080700000000000000BF
:1013D200DC05002000000000A8A9040807000000A6
:1013E20000000000D405002000000000B0A904089D
:1013F2000700000000000000CC05002000000000F3
:10140200B8A904080700000000000000C40500207D
:1014120000000000C0A9040807000000000000004E
:10142200BC05002000000000C8A904080700000055
:1014320000000000B405002000000000D0A904084C
:101442000700000000000000AC05002000000000C2
:10145200BCA504080100000000000000000000001C
:1014620000000000000000000D000000000000006D
:10147200000000000000000000000000B9C80208DF
:10148200F4050020564D00201B00000014680408DB
:10149200554D00200A320100544D002001FA01008E
:1014A200504D002000C801004E4D0020E803D00737
:1014B200010000004655525946340000CFC80208C8
:1014C20059CE0208D0060020A1C602080000000082
:1014D20020070020C9D0020829CB0208FC070020FF
:1014E200F1C8020800000000B008002081C902080B
:1014F20051C902083C0900200DCA020855CA020857
:10150200DC090020644E00200103010025C9020805
:1015120001C90208F40A0020B1C90208C5CE0208B6
:10152200800B002085CA020821CF0208480C002047
:101532005A4E002001030100D8A90408000000004F
:10154200000000000000000000000000E4A9040800
:101552000800000000000000680D002000000000EC
:10156200ECA904080700000000000000600D002044
:1015720000000000FCA904080700000000000000B1
:10158200580D00200000000008AA0408070000000F
:1015920000000000500D00200000000014AA040802
:1015A2000C00000000000000440D002000000000BC
:1015B20020AA04080300000095150408380D002035
:1015C20000000000BCA504080100000000000000AB
:1015D2000000000000000000000000000D000000FC
:1015E20000000000000000000000000028AA04081B
:1015F20000000000000000000000000000000000E9
:1016020038AA04080A00000000000000B47B0408A5
:101612000000000040AA04080A00000000000000C8
:10162200347B04080000000048AA04080A000000F5
:10163200000000007C4E00200000000050AA0408B8
:101642000A00000000000000740D002000000000ED
:10165200BCA504080100000000000000000000001A
:1016620000000000000000000D000000000000006B
:10167200000000000000000058AA0408000000005A
:101682000000000000000000000000006CAA040836
:101692000300000095150408940D002000000000CE
:1016A20078AA0408030000009515040834010020FC
:1016B2000000000080AA0408030000009515040839
:1016C200880D00200000000088AA04080300000022
:1016D200951504087C0D002000000000BCA504083C
:1016E20001000000000000000000000000000000F7
:1016F200000000000D0000000000000000000000DB
:101702000000000094AA040800000000000000008D
:101712000000000000000000A0AA0408070000006A
:101722006DCF0208F00D002000000000C4AF0408D5
:101732000300000095150408E40D002000000000DD
:10174200ACAA04080300000095150408D80D002077
:1017520000000000B4AA0408030000009515040864
:10176200CC0D002000000000BCAA04080700000005
:1017720051CF0208C40D00200000000044AC040850
:101782000300000095150408B80D002000000000B9
:10179200C8AA04080300000095150408AC0D002037
:1017A20000000000D4AA04080300000095150408F4
:1017B200A00D002000000000BCA5040801000000EC
:1017C2000000000000000000000000000000000017
:1017D2000D000000000000000000000000000000FA
:1017E20081C8020849C80208F80D0020F5CA02089B
:1017F20000000000AC0E002000000000000000000D
:10180200380F0020CDCA020889CF0208C40F002079
:10181200E0AA040800000000000000000000000030
:1018220000000000ECAA040803000000951504085B
:10183200C410002000000000F4AA04080300000005
:1018420095150408B81000200000000000AB040841
:101852000300000095150408AC10002000000000F1
:101862000CAB04080300000095150408A01000202A
:101872000000000014AB04080200000015D90208A1
:1018820000000000000000001CAB04080200000081
:1018920015D90208010000000000000028AB04086E
:1018A2000200000015D9020802000000000000003A
:1018B200000000000D000000000000000000000019
:1018C200000000004A4D002088136F17010000003D
:1018D2004C4D002088136F170000000034AB040841
:1018E20000000000000000000000000000000000F6
:1018F20044AB040808000000000000009011002022
:101902000400000050AB04080800000000000000C2
:10191200841100200000000080A7040804000000D9
:101922005DCC02080000000000000000BCA5040815
:1019320001000000000000000000000000000000A4
:10194200000000000D000000000000000000000088
:1019520000000000484D002088136F1701000000AE
:10196200904A002088136F1700000000DDC70208AC
:10197200000000009C110020984E00200100000091
:1019820084680408924A002001000000906804085C
:10199200884A0020020000009868040832BA002039
:1019A200000000000000000030BA0020000000002B
:1019B200000000002EBA002000000000000000001D
:1019C2002CBA002000000000000000002ABA00200B
:1019D200000000000000000028BA00200000000003
:1019E20000000000280100200000000000000000AC
:1019F200474D002002000000A46804088CAB0408D4
:101A020000000000000000000000000000000000D4
:101A120044AB04080800000000000000201200206F
:101A22000400000050AB04080800000000000000A1
:101A3200141200200000000080A704080400000027
:101A4200B1C702080000000000000000BCA50408A5
:101A52000100000000000000000000000000000083
:101A6200000000000D000000000000000000000067
:101A7200000000009CAB0408000000000000000011
:101A82000000000000000000ACAB04080C000000E5
:101A9200ADCD02085012002004000000B8AB0408CB
:101AA2000C00000001C802084412002004000000DB
:101AB200C4AB04080C00000071CD020838120020EB
:101AC20000000000D0AB0408030000003DCC020877
:101AD2002C12002008000000DCAB04080300000008
:101AE200951504085415002000000000BCA5040848
:101AF20001000000000000000000000000000000E3
:101B0200000000000D0000000000000000000000C6
:101B120000000000B4A5040800000000000000005E
:101B2200000000000000000095A504080400000069
:101B320079CC02080000000000000000BCA50408E7
:101B42000100000000000000000000000000000092
:101B5200000000000D000000000000000000000076
:101B62000000000030AC040800000000000000008B
:101B72000000000000000000688204080C00000061
:101B820000000000B01200200400000040AC040875
:101B92000800000000000000A41200200400000061
:101BA2004CAC04080800000000000000981200205D
:101BB2000400000054AC040808000000000000000B
:101BC2008C120020040000005CAC04080800000035
:101BD20000000000801200200400000064AC040831
:101BE2000800000000000000741200200400000041
:101BF2006CAC04080800000000000000681200201D
:101C02000400000074AC040808000000000000009A
:101C12005C12002004000000BCA5040801000000C2
:101C220000000000000000000000000000000000B2
:101C32000D00000000000000000000000000000095
:101C4200C9C7020800000000BC120020000000000A
:101C5200000000003413002000000000000000001B
:101C6200D41300208E4A002004000000B06804084B
:101C72008C4A0020E0150C17000000008B4A00205F
:101C820008000000DC6D04088A4A002005000000FC
:101C9200C4680408000000000000000024140020B2
:101CA2002D202D2D202D2D2D2D202D2D2D2D0000E3
:101CB2000000000000000000000000000000000022
:101CC20000000000010203040102030406070809E0
:101CD200000101010100000001000000006002405B
:101CE2001060024000000000000B00000000200015
:101CF2000000000000000000006002402860024076
:101D020000000000060C000000002000000000009F
:101D1200000000000060024040600240000000003D
:101D2200100D000000002000000000000000000074
:101D3200006002405860024000000000160E0000E1
:101D420000002000000000000000000000600240CF
:101D52007060024000000000200F00000000200020
:101D620000000000000000000060024088600240A5
:101D7200000000002610000000002000000000000B
:101D82000000000000600240A0600240000000006D
:101D920030110000000020000000000000000000E0
:101DA20000600240B860024000000000362F0000D0
:101DB200000020000000000000000000006402405B
:101DC20010640240000000000038000000004000E3
:101DD200000000000000000000640240286402408D
:101DE2000000000006390000000040000000000072
:101DF2000000000000640240406402400000000055
:101E0200103A000000004000000000000000000046
:101E1200006402405864024000000000163B0000CB
:101E220000004000000000000000000000640240CA
:101E32007064024000000000203C000000004000EE
:101E420000000000000000000064024088640240BC
:101E520000000000264400000000400000000000D6
:101E62000000000000640240A06402400000000084
:101E720030450000000040000000000000000000AB
:101E820000640240B86402400000000036460000D0
:101E92000000400000000000000000000000803F41
:101EA200000000010000000000000000000000002F
:101EB2003DE50308F5E40308E5F30308000000002C
:101EC200E5E0030849E40308C9E40308B1E30308B1
:101ED2000000000000000000D9E0030855F60308E6
:101EE20051F603084DF6030841F603083DF60308D0
:101EF20049F6030845F60308C9F60308BDF60308C8
:101F020095F60308A9F6030881F603086DF603089F
:101F120059F6030800000101FFFF0000C47F040816
:101F2200000000000000000075CB0108A08601003F
:101F3200040000000000000000000000000000009B
:101F4200000000000000000000000000000000008F
:101F5200C4AF0408F0A3040800000000595F0108A0
:101F62007D000000060000000000000000000000EC
:101F7200000000000000000000000000000000005F
:101F82000000000080B20408000000000000000011
:101F9200E9090108E8030000030000000000000056
:101FA200000000000000000000000000000000002F
:101FB200000000000000000088B2040800000000D9
:101FC200000000007DA503081027000003000000A8
:101FD20000000000000000000000000000000000FF
:101FE20000000000000000000000000094B204089D
:101FF200000000006152020891EA0008204E000031
:1020020005000000000000000000000000000000C9
:1020120000000000000000000000000000000000BE
:102022005C81040800000000000000007D1001082F
:102032001027000001000000000000000000000066
:10204200000000000000000000000000000000008E
:102052000000000098B20408000000000000000028
:10206200E5E40008E80300000500000000000000AD
:10207200000000000000000000000000000000005E
:102082000000000000000000A4B2040800000000EC
:102092000000000039CE0108204E000003000000BD
:1020A200000000000000000000000000000000002E
:1020B200000000000000000000000000B4B20408AC
:1020C200000000000000000041CC0108204E00008A
:1020D20003000000000000000000000000000000FB
:1020E20000000000000000000000000000000000EE
:1020F200C4B204080000000000000000D90D01086D
:10210200400D03000300000000000000000000007A
:1021120000000000000000000000000000000000BD
:102122000000000090800408000000000000000091
:10213200DDDD0108102700000100000000000000A2
:10214200000000000000000000000000000000008D
:10215200000000000000000064810408000000008C
:102162000000000065A6020810270000030000001E
:10217200000000000000000000000000000000005D
:10218200000000000000000000000000FCA30408A2
:102192000000000000000000B1E9000850C3000088
:1021A200010000000000000000000000000000002C
:1021B200000000000000000000000000000000001D
:1021C200D0A60408000000000000000019E5000885
:1021D200A8610000010000000000000000000000F3
:1021E20000000000000000000000000000000000ED
:1021F20000000000D4B2040800000000000000004B
:10220200E5D60308A08601000100000000000000DE
:1022120000000000000000000000000000000000BC
:1022220000000000000000007081040800000000AF
:1022320000000000D5150108A00F000001000000F9
:10224200000000000000000000000000000000008C
:10225200000000000000000000000000E0B20408DE
:102262000000000000000000D190030810270000C9
:10227200010000000000000000000000000000005B
:10228200000000000000000000000000000000004C
:10229200D4810408000000000000000095AF02088D
:1022A20010270000010000000000000000000000F4
:1022B200000000000000000000000000000000001C
:1022C20000000000DCA30408000000000000000081
:1022D20035D102081A410000010000000000000090
:1022E20000000000000000000000000000000000EC
:1022F2000000000000000000ECB204080000000032
:1023020000000000C9B40108400D030000000000F5
:1023120000000000000000000000000000000000BB
:10232200000000000000000000000000F4B20408F9
:10233200000000000000000065B40108400D030029
:10234200000000000000000000000000000000008B
:10235200000000000000000000000000000000007B
:10236200FCB20408000000000000000069AB020893
:10237200A086010003000000000000000000000031
:10238200000000000000000000000000000000004B
:10239200000000000000803F00000000000000007C
:1023A200000000000000803F00000000000000006C
:1023B200000000000000000000000000000000001B
:1023C2000000000000000000000000000000803F4C
:1023D20000000000000000000000000009024300AD
:1023E200020100C0320904000001020201000524BA
:1023F2000010010524010001042402020524060044
:1024020001070582030800FF09040100020A000017
:10241200000705010240000007058102400000009C
:10242200FF0000000403090412010002020200403E
:10243200830440570002010203010000E11D03086A
:1024420025E603089518030829E10308D1E50308E6
:1024520039E1030855E1030819E1030809E103081A
:102462000000000000000000FFFFFFFF010000006D
:10247200341D0020000000000000000000000000E9
:10248200000000000000000000000000000000004A
:10249200000000000000000000000000000000003A
:1024A200000000000000000000000000000000002A
:1024B200000000000000000000000000000000001A
:1024C200000000000000000000000000000000000A
:1024D20000000000430000000000000000000000B7
:1024E20000000000000000000000000000000000EA
:1024F2000000000043000000000000000000000097
:1025020000000000000000000000000000000000C9
:102512000000000043000000000000000000000076
:1025220000000000000000000000000000000000A9
:102532000000000043000000000000000000000056
:102542000000000000000000000000000000000089
:102552000000000043000000000000000000000036
:102562000000000000000000000000000000000069
:102572000000000043000000000000000000000016
:102582000000000000000000000000000000000049
:1025920000000000430000000000000000000000F6
:1025A2000000000000000000000000000000000029
:1025B2000000000017340408F33304080000000090
:1025C2002FB60408A8A50408CE8C0408CE8C0408F3
:1025D200CE8C0408CE8C0408CE8C0408CE8C040861
:1025E200CE8C0408CE8C0408CE8C0408FFFFFFFFBB
:1025F200FFFFFFFFFFFFFFFFFFFF0000010041534E
:1026020043494900000000000000000000000000F3
:102612000000000000000000000000000000415324
:1026220043494900000000000000000000000000D3
:102632000000000000000000000000000000000098
:042642000100000093
:10800000012380F8453070474FF400638382704746
:108010004FF40063838270470122482117F0D2BADF
:108020000122582117F0CEBA4FF4006383827047C3
:108030004FF4805383827047BFF34F8F0549064B3F
:10804000CA6802F4E0621343CB60BFF34F8F00BFF6
:10805000FDE700BF00ED00E00400FA0570B4037B0B
:1080600004681F2B08D9203B2021626801FA03F322
:108070001A421CD170BC70472021226801FA03F318
:108080001A42F7D0426914495C2000FB0212516881
:108090005689CD680868296821F001012960828924
:1080A00092B222EA06028281A36070BC70474269E4
:1080B00009495C2000FB021251685689CD680868A6
:1080C000296821F001012960828992B222EA060220
:1080D0008281E36070BC7047F85900202B4B1978FF
:1080E000002951D02A4B30B41C6898880022626263
:1080F000A5899A80284380B20129A08143D09C6839
:1081000098896262A589284380B20229A0819A8158
:1081100039D01C69988A6262A589284380B20329F4
:10812000A0819A822FD09C69988B6262A58928438E
:1081300080B20429A0819A8325D01C6A988C62623F
:10814000A589284380B20529A0819A841BD09C6A06
:10815000988D6262A589284380B20629A0819A85FC
:1081600011D01C6B988E6262A589284380B20729C2
:10817000A0819A8607D0986B998F426284892143A7
:1081800089B281819A8730BC704700BFD85C0020DB
:10819000DC5C002010B4037B01681F2B09D9203B55
:1081A00020224C6802FA03F31C4214D15DF8044B00
:1081B000704720220C6802FA03F31C42F6D00C4AE6
:1081C00040680024147002685DF8044B22F001023C
:1081D00002608B607047064A406800241470026891
:1081E0005DF8044B22F001020260CB60704700BFD3
:1081F00075910020F0B5C40022189200AE498B584A
:108200005B689D8AADB2EEB2F7070A445CD4B7074B
:1082100032D5BFF35F8F167EF6B2012E00F0C78015
:10822000A64D1A8BBFF35F8F221801EB8202167ED8
:10823000022E00F0D580221801EB8202167E032E5A
:1082400000F088809A8895F9006092B242F48062CA
:108250009A80221801EB8202127E013296425BD193
:10826000AA7800266E70002A40F09580204401EB29
:10827000800000234375F0BD77074ED416F040060A
:1082800000F0C9808D4D1E8A95F900E0176AF6B29C
:1082900007F80E605FFA8EFE0EF1010C4FFA8CFCAF
:1082A000177E85F800C00CF103029742664600F085
:1082B0001C81221801EB8202127E9445C9D10EF175
:1082C000020676B22E70C4E71E887C4D26F4006646
:1082D0003604360C1E801E88B6B246F480661E80B8
:1082E000967E00272F70002E48D06E78002E42D048
:1082F000221801EB82020126127E6E70022A00F023
:10830000B980221801EB8202927D42F001021A82AA
:10831000204401EB8000037EF0BD684D967E01276E
:10832000AF70002E73D06E78002E7BD1221801EB37
:108330008202527E002A00F0A3801A882E7892B220
:10834000013642F4007276B21A802E701A88D20575
:10835000FCD47EE7927E002A3FF474AF6A78002A4C
:108360003FF470AF9A8895F9006022F4806212049D
:10837000120C9A806DE7D27DFF2AB9D0221801EB4A
:108380008202967D06F0FE061E82D37DFF2BBFD0B3
:10839000FF232B70BCE79A8822F440721204204419
:1083A000120C01EB80009A8000234375F0BD927E91
:1083B000424D002A3FF435AF6A78002A3FF431AFCE
:1083C0001A8822F480621204120C1A80BFF35F8FA5
:1083D0001A8B1A88AE7092B242F400721A8031E79A
:1083E000927E002A3FF427AF6A78002A3FF423AF39
:1083F0001A8895F9006022F480621204120C1A8027
:108400009A8822F480621204120C9A8021E76A781A
:10841000002A8BD091E715F0800F284D3AD195F9BD
:10842000006016E7167ED2F820E01F88022E95F92C
:10843000006045D927F480673F043F0C1F801F8AE6
:10844000FFB20EF806701F88D2F820E0BFB247F4E2
:1084500000771F80F2B21F8A561C76B2FFB20EF868
:1084600006709F88961CBAB276B242F480622E7073
:108470009A806BE71A8892B242F400621A8040E751
:108480001A8895F9006092B242F4807201271A802E
:108490006F705BE795F90070B7F1FF3F2CD0D6699C
:1084A000F65D1E8292F818E001377AB296451646BC
:1084B0002A707FF4CEAEA3E780350020081F00208D
:1084C000BFB247F400771F801F8AFFB20EF8067014
:1084D000F6B21F8AD2F820E0721C52B20336FFB205
:1084E00076B20EF802702E7030E79A8822F480621D
:1084F0001204120C9A80DCE6D77D1F822E70957EC6
:108500001DB9127E002A7FF403AF9A8822F480629C
:108510001204120C9A80FBE6F0B5876983B0064618
:1085200017B13B68BA885A837069DFF8A4E0838981
:10853000C3244FF47A734FF0060C6D464FF6FF716B
:108540000EF1010E03E0013B9BB28B4220D0028969
:108550009207F8D5A3B283814FF47A7302E0A3B2F5
:108560008B4215D00289D20703F1FF34F7D58289F7
:1085700092B20DB12A700135BCF1000F0BD00CF195
:10858000FF3CFF24BEF1000FE1D09EF80040D7E78A
:1085900016F02CFFB76917B13B68BA881A839DF8AB
:1085A00005009DF801509DF802109DF803409DF8CC
:1085B00004209DF8063041EA052143EA002342EAFF
:1085C0000422012031877287B38703B0F0BD00BF5A
:1085D00028450408F8B5057B466903681F2D29D98D
:1085E000A5F120045F682021A1400F422A4613D044
:1085F0001022A240D960DA605A68E240D10703D560
:10860000012202FA04F4DC600446304605F026FC40
:10861000227B23681F2A20D9A2F1200008215A6852
:108620008140114200D0D9600422596882400A4238
:1086300021D1F8BD20211C68A9400C422A460CD04B
:108640001022AA4099609A601A68EA40D207DBD5E6
:10865000012202FA05F59D60D6E7082118689140CD
:10866000014200D099600421186801FA02F2024226
:1086700003D09A60F8BDDA60F8BDF8BD07B50323F2
:1086800001AA002116F01AFF9DF805309DF804009C
:108690001B0243EA00439DF80600184303B05DF84F
:1086A00004FB08B5FFF7EAFF014B186008BD00BFE7
:1086B00084360020144B984224D003F580639842FE
:1086C00020D0028822F040021204120C028002889C
:1086D00022F038031B041B0C59B141F480710029AE
:1086E00091FAA1F2B2FA82F108BF4FF0FF310139DD
:1086F000C9000B439BB2038003889BB243F0400345
:10870000038070474908DCE70038004008B540F2B4
:10871000E93300E0A3B10289013B12F0020F9BB2E2
:10872000F8D089B2818140F2E93300E043B1028997
:10873000013B12F0010F9BB2F8D08089C0B208BD96
:1087400016F054FEC0B208BD2DE9F04F85B001907F
:1087500090F85500002840F08886019B58699D4B91
:10876000984200F0C2869C4A90420CBF30223822C8
:10877000038823F040031B041B0C038003889BB277
:1087800023F038031A43028003889BB243F040036E
:108790000380019B9B6913B11A689B88538340F245
:1087A000E93302E0002B00F0DF860289013B12F082
:1087B000020F9BB2F6D06B23838140F2E93302E0D3
:1087C000002B00F0D1860289013B12F0010F9BB211
:1087D000F6D0838940F2E93302E0002B00F0C08636
:1087E0000289013B12F0020F9BB2F6D080238381F5
:1087F00040F2E93302E0002B00F0B2860289013B2F
:1088000012F0010F9BB2F6D08389019B9B6913B1D3
:108810001A689B881383714C714DDFF8CC917148B5
:10882000DFF8C8E14FF0640A4FF0100C4FF47A768D
:10883000D9F80430C3F30803002B40F05085EFF360
:108840001183002B40F04B852168826800BF2368AC
:108850009942F9D12F6806FB07F39B1AB3FBF7F394
:1088600006FB013101270091D9F80430C3F3080356
:10887000002B40F0F984EFF31183002B40F0F484D7
:108880002368816800BF22689342F9D1D5F800B00F
:1088900006FB0BF2521AB2FBFBF206FB0323009A13
:1088A0009B1AB3F57A7FDFD3BAF1010AC0D1019BDD
:1088B0009B6913B11A689B885383019E6821706974
:1088C000FFF724FF03217069FFF720FFB36913B19D
:1088D0001A689B881383DFF810914248DFF80CE197
:1088E0004FF0640A4FF0100C4FF47A76D9F8043048
:1088F000C3F30803002B40F0D584EFF31183002B62
:1089000040F0D0842168826800BF23689942F9D181
:108910002F6806FB07F39B1AB3FBF7F306FB013145
:1089200001270091D9F80430C3F30803002B40F06D
:108930007284EFF31183002B40F06D84236881680B
:1089400000BF22689342F9D1D5F800B006FB0BF2C4
:10895000521AB2FBFBF206FB0323009A9B1AB3F5F3
:108960007A7FDFD3BAF1010AC0D1019B9B6913B1B1
:108970001A689B885383019B586940F2E93302E0EF
:10898000002B00F0E7850289013B12F0020F9BB239
:10899000F6D06B23838140F2E93302E0002B00F034
:1089A000D9850289013B12F0010F9BB2F6D0838971
:1089B00040F2E93302E0002B00F0C8850289013B58
:1089C00012F0020F9BB2F6D00123838140F2E9330B
:1089D00011E000BF00380040003C00400C7D00204A
:1089E000107D002010E000E000ED00E0087D002098
:1089F000002B00F0AB850289013B12F0010F9BB206
:108A0000F6D08389019B9B6913B11A689B881383F5
:108A1000DFF8AC92A948DFF8ACE24FF00F0A4FF054
:108A2000100C4FF47A76D9F80430C3F30803002B06
:108A300040F08E84EFF31183002B40F0898421688D
:108A4000826800BF23689942F9D12F6806FB07F3BB
:108A50009B1AB3FBF7F306FB013101270091D9F80C
:108A60000430C3F30803002B40F0B883EFF3118305
:108A7000002B40F0B3832368816800BF22689342D3
:108A8000F9D1D5F800B006FB0BF2521AB2FBFBF29B
:108A900006FB0323009A9B1AB3F57A7FDFD3BAF162
:108AA000010AC0D1019991F84F208B69042A34BF83
:108AB00018261A2613B11A689B885383019B58699C
:108AC00040F2E93302E0002B00F03A850289013BD5
:108AD00012F0020F9BB2F6D01B23838140F2E933E0
:108AE00002E0002B00F02C850289013B12F0010FFF
:108AF0009BB2F6D0838940F2E93302E0002B00F00C
:108B00001B850289013B12F0020F9BB2F6D08681D1
:108B100040F2E93302E0002B00F00E850289013BB0
:108B200012F0010F9BB2F6D08389019B9B6913B1B0
:108B30001A689B881383DFF888916048DFF884E126
:108B40004FF00F0A4FF0100C4FF47A76D9F804303A
:108B5000C3F30803002B40F0DF83EFF31183002BF6
:108B600040F0DA832168826800BF23689942F9D116
:108B70002F6806FB07F39B1AB3FBF7F306FB0131E3
:108B800001270091D9F80430C3F30803002B40F00B
:108B90000883EFF31183002B40F00383236881687F
:108BA00000BF22689342F9D1D5F800B006FB0BF262
:108BB000521AB2FBFBF206FB0323009A9B1AB3F591
:108BC0007A7FDFD3BAF1010AC0D1019B9B6913B14F
:108BD0001A689B885383019E1C217069FFF796FDDC
:108BE00018217069FFF792FDB36913B11A689B8869
:108BF0001383DFF8CC903148DFF8C8E04FF00F0A5C
:108C00004FF0100C4FF47A76D9F80430C3F3080310
:108C1000002B40F0D683EFF31183002B40F0D1837B
:108C20002168826800BF23689942F9D12F6806FB4A
:108C300007F39B1AB3FBF7F306FB01310127009101
:108C4000D9F80430C3F30803002B40F08D82EFF312
:108C50001183002B40F088822368816800BF22685E
:108C60009342F9D1D5F800B006FB0BF2521AB2FBD1
:108C7000FBF206FB0323009A9B1AB3F57A7FDFD33E
:108C8000BAF1010AC0D1019A936992F84E6013B10A
:108C90001A689B885383019B586940F2E93302E0CC
:108CA000002B00F043840289013B12F0020F9BB2BB
:108CB000F6D01A23838140F2E93308E010E000E0A7
:108CC00000ED00E0087D0020002B00F02F840289D9
:108CD000013B12F0010F9BB2F6D0838940F2E933D9
:108CE00002E0002B00F01E840289013B12F0020F0B
:108CF0009BB2F6D0B6B2868140F2E93302E0002B97
:108D000000F010840289013B12F0010F9BB2F6D0F3
:108D10008389019B9B6913B11A689B881383DFF8D1
:108D200020928648DFF81CE24FF00F0A4FF0100C3B
:108D30004FF47A76D9F80430C3F30803002B40F0DF
:108D40002483EFF31183002B40F01F832168826896
:108D500000BF23689942F9D12F6806FB07F39B1ADD
:108D6000B3FBF7F306FB013101270091D9F804307A
:108D7000C3F30803002B40F0DA81EFF31183002BDB
:108D800040F0D5812368816800BF22689342F9D101
:108D9000D5F800B006FB0BF2521AB2FBFBF206FB51
:108DA0000323009A9B1AB3F57A7FDFD3BAF1010A45
:108DB000C0D1019A936992F8506013B11A689B88E8
:108DC0005383019B586940F2E93302E0002B00F025
:108DD000A4830289013B12F0020F9BB2F6D0192343
:108DE000838140F2E93302E0002B00F09683028990
:108DF000013B12F0010F9BB2F6D0838940F2E933B8
:108E000002E0002B00F086830289013B12F0020F82
:108E10009BB2F6D0B6B2868140F2E93302E0002B75
:108E200000F078830289013B12F0010F9BB2F6D06B
:108E30008389019B9B6913B11A689B881383DFF8B0
:108E400000913E48DFF8FCE04FF0640A4FF0100C50
:108E50004FF47A76D9F80430C3F30803002B40F0BE
:108E6000E882EFF31183002B40F0E38221688268EF
:108E700000BF23689942F9D12F6806FB07F39B1ABC
:108E8000B3FBF7F306FB013101270091D9F8043059
:108E9000C3F30803002B40F02D81EFF31183002B67
:108EA00040F028812368816800BF22689342F9D18D
:108EB000D5F800B006FB0BF2521AB2FBFBF206FB30
:108EC0000323009A9B1AB3F57A7FDFD3BAF1010A24
:108ED000C0D1019B9B6913B11A689B885383019B86
:108EE000586940F2E93302E0002B00F00E8302895A
:108EF000013B12F0020F9BB2F6D03723838140F280
:108F0000E93302E0002B00F000830289013B12F0FC
:108F1000010F9BB2F6D0838940F2E93302E0002BC7
:108F200000F0F0820289013B12F0020F9BB2F6D0F2
:108F30001023838140F2E93309E000BF10E000E034
:108F400000ED00E0087D0020002B00F0DB820289AC
:108F5000013B12F0010F9BB2F6D08389019B9B6904
:108F600013B11A689B881383DFF8F492B948DFF8CD
:108F7000F4E24FF00F0A4FF0100C4FF47A76D9F864
:108F80000430C3F30803002B40F03782EFF3118362
:108F9000002B40F032822168826800BF236899422A
:108FA000F9D12F6806FB07F39B1AB3FBF7F306FB17
:108FB000013101270091D9F80430C3F30803002BD5
:108FC0007BD1EFF31183002B77D12368816800BF39
:108FD00022689342F9D1D5F800B006FB0BF2521A81
:108FE000B2FBFBF206FB0323009A9B1AB3F57A7FD0
:108FF000E1D3BAF1010AC2D1019B9B6913B11A688E
:109000009B885383019B586940F2E93302E0002BAF
:1090100000F073820289013B12F0020F9BB2F6D07E
:109020003823838140F2E93302E0002B00F06582AF
:109030000289013B12F0010F9BB2F6D0838940F206
:10904000E93302E0002B00F053820289013B12F069
:10905000020F9BB2F6D00123838140F2E93302E094
:10906000002B00F045820289013B12F0010F9BB2F8
:10907000F6D08389019B9B6913B11A689B8813837F
:10908000754B984200F08382744A90420CBF0822CC
:109090001022038823F040031B041B0C0380038869
:1090A0009BB223F038031A43028003889BB243F03B
:1090B0004003038005B0BDE8F08FEFF311888CF317
:1090C000128881680368DB0344BFCEF800708168B2
:1090D0002368DEF800205FFA88F888F31188D5F855
:1090E00000801A4406FB08F35B1AB3FBF8F306FB97
:1090F000023379E7EFF311888CF3128881680368F3
:10910000DB0344BFCEF8007081682368DEF80020DE
:109110005FFA88F888F31188D5F800801A4406FBB6
:1091200008F35B1AB3FBF8F306FB0233C9E6EFF36F
:1091300011888CF3128881680368DB0344BFCEF882
:10914000007081682368DEF800205FFA88F888F3F1
:109150001188D5F800801A4406FB08F35B1AB3FBAC
:10916000F8F306FB02331CE6EFF311888CF3128848
:1091700081680368DB0344BFCEF800708168236810
:10918000DEF800205FFA88F888F31188D5F80080AF
:109190001A4406FB08F35B1AB3FBF8F306FB023331
:1091A00069E5EFF311888CF3128881680368DB03AB
:1091B00044BFCEF8007081682368DEF800205FFAB3
:1091C00088F888F31188D5F800801A4406FB08F364
:1091D0005B1AB3FBF8F306FB0233EEE4EFF31188FE
:1091E0008CF3128881680368DB0344BFCEF80070FB
:1091F00081682368DEF800205FFA88F888F3118818
:10920000D5F800801A4406FB08F35B1AB3FBF8F3A9
:1092100006FB02333EE4EFF311888CF31288816879
:109220000368DB0344BFCEF8007081682368DEF872
:1092300000205FFA88F888F31188D5F800801A4476
:1092400006FB08F35B1AB3FBF8F306FB0233FFF7E8
:1092500084BB00BF10E000E000380040003C00404C
:1092600000ED00E0087D0020EFF311888CF31288F8
:1092700081680368DB0344BFCEF80070816823680F
:10928000DEF800205FFA88F888F31188D5F80080AE
:109290001A4406FB08F35B1AB3FBF8F306FB023330
:1092A000FFF7FDBAEFF311828CF312888768036829
:1092B000D90303D50123CEF8003087682368DEF890
:1092C0000010D2B282F311882A68194406FB02F317
:1092D000DB1BB3FBF2F306FB0131FFF721BBEFF31E
:1092E00011828CF3128887680368D90303D50123A0
:1092F000CEF8003087682368DEF80010D2B282F31F
:1093000011882A68194406FB02F3DB1BB3FBF2F356
:1093100006FB0131FFF7A6BAEFF311828CF3128836
:1093200087680368D90303D50123CEF80030876826
:109330002368DEF80010D2B282F311882A6819443B
:1093400006FB02F3DB1BB3FBF2F306FB013117E470
:10935000EFF311828CF3128887680368D90303D571
:109360000123CEF8003087682368DEF80010D2B2FF
:1093700082F311882A68194406FB02F3DB1BB3FB56
:10938000F2F306FB0131FFF768BBEFF311828CF3B8
:10939000128887680368D90303D50123CEF800300B
:1093A00087682368DEF80010D2B282F311882A6839
:1093B000194406FB02F3DB1BB3FBF2F306FB01319E
:1093C000D2E4EFF311828CF3128887680368D90323
:1093D00003D50123CEF8003087682368DEF800103B
:1093E000D2B282F311882A68194406FB02F3DB1B10
:1093F000B3FBF2F306FB013120E4EFF311828CF3AF
:10940000128887680368D90303D50123CEF800309A
:1094100087682368DEF80010D2B282F311882A68C8
:10942000194406FB02F3DB1BB3FBF2F306FB01312D
:10943000BFE5EFF311828CF3128887680368D903C4
:1094400003D50123CEF8003087682368DEF80010CA
:10945000D2B282F311882A68194406FB02F3DB1B9F
:10946000B3FBF2F306FB01310EE503F015FF0446F2
:10947000002800F0848000684B4900F13F4303F569
:109480007E039A0A20258A5CA57102F01F06520904
:1094900001230021032A03FA06F3E1717ED0042A96
:1094A00077D0022A66D0A388029302A900230393EF
:1094B00028F0ECFF01993D4B41F80C3F20462CF081
:1094C0005DFDA388B3FA83F3C3F11F03012212FAEF
:1094D00003F33FF442A936490A6813430B60019B2A
:1094E0005869344B98427FF43EA93022FFF740B9C7
:1094F00015F07CFF019B5869BDE515F077FF019BD6
:1095000058699CE515F072FF28E515F06FFF019B87
:10951000586901E515F06AFF8BE415F067FF019BC0
:1095200058696BE415F062FFFFF7F3BB15F05EFFBF
:10953000019B5869FFF7D2BB15F058FFFFF7F5BA4A
:1095400015F054FF019B5869FFF7D5BA15F04EFF8F
:10955000FFF758BA15F04AFF019B5869FFF728BA80
:1095600015F044FFFFF751B915F040FF019B586912
:10957000FFF730B9104A516C0B43536493E70199DC
:109580000A4B41F80C3F2CF0F9FCFFF7E6B8082233
:109590007FE5094A116B0B43136384E7064A116C9C
:1095A0000B4313647FE700BFDC6F040801800008F1
:1095B000003C014000380040003802400C4B98420B
:1095C00013D0A3F5806398420FD003F580439842EF
:1095D0000BD003F58063984207D003F5806398426F
:1095E00003D0044B186840087047024B1868704756
:1095F00000040140CC850020F0B5774B774A87B056
:109600001968914200AF00F0DB800023744A3B6090
:109610007B60136843F48033136003E03B68B3F569
:10962000A04F09D0136803F400337B603B6801331B
:109630003B607B68002BF1D0694B1B6813F400334F
:1096400018BF01237B607B68012B7BD0654D644B89
:10965000654AEA606549586F654A0860AA605E6BB2
:10966000644C654A654826F080065E635E6F46F08E
:1096700080765E67196B0C431C63596B5963996B59
:109680009963196C41F05B5141F47B1141F41F6106
:1096900041F00F011964596C07F118040A4348F2AC
:1096A000FF715A6444F8101D002621460123FB7304
:1096B0003E737E73BE7328F0E9FE21464FF6FF73BA
:1096C0004F48BB6028F0E2FE4FF6FF7321464D483D
:1096D000BB6028F0DBFE21464B4828F0D7FE214630
:1096E0004A4828F0D3FE2146494828F0CFFE2146BB
:1096F000484828F0CBFE2146474828F0C7FE2146BF
:10970000464828F0C3FE204628F078FC444B454CE0
:109710001B68BA6844484549A4FB03439B09A0FB66
:109720000202013B920CB3F1807F0A6007D2404AEB
:10973000F0200721536085F82300966011601C37E4
:10974000BD46F0BD264B3B4D1A6C3B4842F0805263
:109750001A642C684268816844F440442C609C6818
:109760009C609C6844F400449C609C6844F4A05451
:109770009C600068120642EA801242F480024908A6
:1097800042F00802013942EA01425A601A6842F086
:1097900080721A601A689201FCD52849104A40F27A
:1097A00005700860996821F003019960996841F09B
:1097B00002019960936803F00C03082BFAD145E786
:1097C00000221A6062B61E4B1B6883F308881D4B8B
:1097D0001B689847FEE700BFFCFF0120EFBEADDE2F
:1097E0000038024000ED00E00005FA05745D00203D
:1097F00000000008FF916700335F0700000002408F
:109800000004024000080240000C02400010024028
:109810000014024000180240001C024000200240D8
:10982000CC850020D34D621083DE1B43107D0020C9
:1098300010E000E00070004000000020003C02400A
:109840000000FF1F0400FF1F08B5054B1B6803B194
:109850009847044B044A1A6072B6FEF7EDFB00BF4E
:1098600064550020FCFF0120EFBEADDEF0B590F89E
:10987000553083B00446002B40F0AA806D46514E0F
:10988000F378002B00F0FF8060694F4B984200F0A6
:109890001F824E4A90420CBF30223822038823F0A8
:1098A00040031B041B0C038003889BB223F0380386
:1098B0001A43028003889BB243F040030380A369EC
:1098C00094F84E6013B11A689B88538340F2E933D1
:1098D00004E0013B9BB2002B00F02C82028992072E
:1098E000F7D51A23838140F2E93304E0013B9BB2B0
:1098F000002B00F01F820289D707F7D5838940F239
:10990000E93304E0013B9BB2002B00F01082028996
:109910009107F7D5B6B2868140F2E93304E0013B06
:109920009BB2002B00F003820289D207F7D583890E
:10993000A36913B11A689B881383012004F08CF883
:109940006369214A934200F0018220498B4214BF8F
:10995000082100211A8822F040021204120C1A80F9
:109960001A8892B222F0380211431980198889B2FC
:1099700041F0400119802A460623432104F11000DA
:1099800015F09CFD002800F0CF819DF802609DF845
:1099900003309DF800509DF801109DF804009DF8DB
:1099A000052043EA06231BB241EA052142EA0022D0
:1099B00063872187A2875BB2013300F08B8103B0FC
:1099C000F0BD00BF081F002000380040003C0040F0
:1099D0001E09013E032E03F00F0300F2AF81994AE6
:1099E00032F8160040FA03F2D10740F1A7810125B1
:1099F00005FA03F3013B184039F0B8F9924B934A4A
:109A00009B5D184412EBC00600F0988100232021D2
:109A1000F371B17152F830008D4A00F13F4303F504
:109A20007E039B0AD25C02F01F035209032A05FA47
:109A300003F300F09781042A00F08F81022A00F0DE
:109A40008781B388009369460023019328F01EFDA7
:109A50002146804B41F80C3F30462CF08FFAB388FA
:109A6000B3FA83F3C3F11F03012212FA03F36D4625
:109A70003FF405AF7849794E0A6813430B60F378D9
:109A8000002B7FF401AF6069754B984200F0718143
:109A9000744A90420CBF30223822038823F04003DE
:109AA0001B041B0C038003889BB223F038031A436A
:109AB000028003889BB243F040030380A36913B183
:109AC0001A689B8853836B21FEF720FE8021606912
:109AD000FEF71CFEA36913B11A689B8813839620B6
:109AE00004F014F8A36913B11A689B8853836821A2
:109AF0006069FEF70BFE03216069FEF707FEA369AC
:109B000013B11A689B881383962003F0FFFFA369A3
:109B100013B11A689B8853836B216069FEF7F6FDC9
:109B200003216069FEF7F2FDA36913B11A689B88EF
:109B300013830F2003F090FFA36913B11A689B8869
:109B400053836A216069FEF7E1FD10216069FEF729
:109B5000DDFDA36913B11A689B8813830F2003F0FE
:109B60007BFFA36913B11A689B8853836C216069DA
:109B7000FEF7CCFD00216069FEF7C8FDA36913B1B3
:109B80001A689B8813830F2003F066FFA36994F87B
:109B9000507013B11A689B88538319216069FEF7CE
:109BA000B5FD39466069FEF7B1FDA36913B11A68C6
:109BB0009B8813830F2003F04FFFA36913B11A682A
:109BC0009B8853831B216069FEF7A0FD1821606903
:109BD000FEF79CFDA36913B11A689B8813830F20BD
:109BE00003F03AFFA36913B11A689B8853831C21C1
:109BF0006069FEF78BFD10216069FEF787FDA369A0
:109C000013B11A689B8813830F2003F025FFA36903
:109C100013B11A689B88538337216069FEF776FD7C
:109C200010216069FEF772FDA36913B11A689B8861
:109C300013830F2003F010FFA369ABB11A689B8850
:109C4000538311E0C0700408BC7004084C7B0020F2
:109C5000DC6F040801800008003C0140081F002060
:109C600000380040003C004038216069FEF74EFD9E
:109C700001216069FEF74AFDA36913B11A689B8848
:109C800013830F2003F0E8FE63693B4A93426ED0D2
:109C90003A498B4214BF082100211A8822F0400261
:109CA0001204120C1A801A8892B222F03802114360
:109CB00019801A8892B242F040021A80012003F003
:109CC000CBFE0123F37060692B4B98427FF4E1AD2A
:109CD0003022E3E594F9383001337FF470AE0A2680
:109CE00032202BF08DFE4FF4FA7503F069FE044626
:109CF00003F066FE001BB0F57A7FF9D3013DF4D185
:109D000007202BF0DFFC4FF47A7503F059FE044670
:109D100003F056FE001BB0F57A7FF9D3013DF4D174
:109D2000013EDDD1FFF790FDB4F93A3043E615F07E
:109D30005DFBFDE515F05AFB6069E0E52146104B3F
:109D400041F80C3F00202CF019F997E5002101E6BD
:109D50000C4A516C0B43536473E60A4A116B0B4374
:109D600013636EE6074A116C0B43136469E6002126
:109D700093E7302291E600BF00380040003C0040ED
:109D8000018000080038024008B5034B1B6803B18E
:109D9000984772B6FEF750F964550020084B10B58D
:109DA00007281B68C8BF143818440C46007E03F00F
:109DB00073FA20B12146BDE8104004F001BB10BD8C
:109DC0007035002038B50C4B07281B68CCBFA0F1BC
:109DD0001404044623440546187E03F05DFA50B18E
:109DE00028220134C47182712BF008FC284600211E
:109DF000BDE83840D2E738BD70350020064A002360
:109E00005168814202F11C0204D00133102BF7D1BA
:109E100000207047D8B270479C150020074BC0EB5C
:109E2000C00030B403EB8000054C0569236B2B4365
:109E300023630176427630BC704700BF9C1500203A
:109E4000003802402DE9F04F614C54F8204083B0B7
:109E5000002C00F0B880256E002D00F0B68017466B
:109E60005C4A9846064604F166032869226004F2BB
:109E700066226361A2614FF400736A68A160E360C7
:109E80002361A265A14668B1FFF7B8FF721CD2B288
:109E90000C21FFF7C3FFA36DA9682A69626304332D
:109EA000E1636365E86880B3FFF7A8FF721CD2B274
:109EB0000B218246FFF7B2FF4748DFF820E1EB7F36
:109EC000DEF83010CAEBCA0A00EB8A009B0902696F
:109ED0000A43CEF83020DFF808E1417B44610022DC
:109EE0008DF80530C0F808E0012301A88DF80410B2
:109EF0008DF806208DF8073028F038F8A36DA96892
:109F0000EA68A26304332164236594F8650003F0D2
:109F1000C3F9824694F8640003F0BEF98346287FB3
:109F200000284DD118F0080F36D1BA070DD5BAF177
:109F3000000F0AD00B22731C8AF806208AF807301B
:109F400050466A7F222103F00FF8FB0715D4E36B1C
:109F50007BB9AA7F8DF8042095F820208DF8063073
:109F600001A8930901228DF805308DF8072027F00C
:109F7000FDFF484603B0BDE8F08FBBF1000FE6D00F
:109F800001360C238BF807608BF8063058466A7F41
:109F9000222102F0E9FFDAE70136F6B2BAF1000F4A
:109FA00004D00B238AF807608AF8063018F0100FE7
:109FB000504614BF022112216A7F02F0D5FFC6E786
:109FC0002BF0FEFAAEE7A146D3E7A946D1E700BFE2
:109FD00050350020304504089C1500200038024010
:109FE000D585000800B970472DE9F04194B00646C8
:109FF0002CF09CF9B64DC36802682A600446002B19
:10A0000000F03C81304603F047F9B24B586018B17C
:10A01000292200238271C371227A2A2102F0A4FF2F
:10A02000286803F047FB2BF0CBFAD5F80080B8F88E
:10A03000003023F001031B041B0CA8F8003040463D
:10A04000FFF7BCFAA44B984200F21B810026DFF810
:10A05000C0E2A24FB8F80030A14906F1010CB0FBF4
:10A06000FCF04FF0030CB0FBF1F081B2B1FBFCF15E
:10A07000AEF80010490039809A4988459BB200F03B
:10A080000A8101F58061884500F00581B8F1804FB3
:10A0900000F00181A1F58031884500F0FC8001F5D8
:10A0A0008061884500F0F78001F58061884500F007
:10A0B000F2808D49884500F0048101F58061884572
:10A0C00000F0FF8023F44071864B89B29845A8F8D0
:10A0D0000010C8F82C00A8F8286000F0EE80834B30
:10A0E000984500F0EA800121A8F81410E279602078
:10A0F0000023ADF800009007ADF80230ADF8043051
:10A100000293ADF80C30ADF80E30ADF81030ADF86C
:10A11000123040F1C48012F0010F0CBF1A46082221
:10A120000423ADF80E20ADF80430002328686179CF
:10A1300002936A4602F0E2FC60792B680C2816D87C
:10A14000DFE810F0FA001500150015000D001500ED
:10A1500015001500F100150015001500E8001A8B18
:10A1600022F400621204120C42F400621A83B3F863
:10A1700044205F4E6FEA42426FEA524292B2A3F825
:10A1800044201A8892B242F080021A80E279198C37
:10A1900092074CBF04220122824092B289B221EA86
:10A1A00002011984198C89B20A431A841A8892B25E
:10A1B00042F001021A80207D00222921FFF72EFEA5
:10A1C000227D4C4B4C494D481C2707FB02320B6B40
:10A1D00017693B430B63537B90600027576105A8C9
:10A1E0008DF8143001238DF815308DF817308DF867
:10A1F000167027F0BBFEE068306027F0EDFF306896
:10A20000036823F00103036027F0E6FF05A827F0A9
:10A21000A5FF2A68637930680A9734321A44069297
:10A2200040F22A3209924FF480620B92344B226939
:10A230000592079340224FF4805305A908920C938E
:10A240004FF480424FF440330D920F930E9727F056
:10A2500097FF6379286831682A4C0C2B9CBF2A4AE7
:10A2600032F81330828988BF3B4692B21343838110
:10A270000B68012243F010030B60227014B0BDE89C
:10A28000F08100F1B77303F558532049B3FBF1F3A4
:10A29000013B9EB2DBE623F070039BB209E712F0AC
:10A2A000010F0CBF002202224FF48073ADF80210A0
:10A2B000ADF80C20ADF8103037E70023A8F83030A7
:10A2C00011E7A8F80030C8F82C00A8F828600AE7C1
:10A2D000004F0020081F0020FF6BDC02F64E00201C
:10A2E00000350C0000000140001000400004014057
:10A2F000FC4E00209C15002000380240958100088B
:10A300006C930020F84E0020486F0408006CDC02BB
:10A31000F44E00209A8B22F400621204120C42F4D4
:10A3200000629A8323E79A8B22F008021204120C2F
:10A3300042F008029A831AE71A8B22F008021204EC
:10A34000120C42F008021A8311E700BF0348D0F84C
:10A35000AC3113B100F5D270184770479C1500203E
:10A360000348D0F8903113B100F5C4701847704716
:10A370009C1500200348D0F8743113B100F5B67075
:10A38000184770479C1500200348D0F8583113B186
:10A3900000F5A870184770479C1500200348D0F8B6
:10A3A0003C3113B100F59A70184770479C15002096
:10A3B0000348D0F8203113B100F58C70184770476E
:10A3C0009C1500200348D0F804310BB1FC3018472D
:10A3D000704700BF9C1500200348D0F8E8300BB14F
:10A3E000E0301847704700BF9C1500200348D0F8A4
:10A3F000CC300BB1C4301847704700BF9C1500200B
:10A400000348D0F8B0300BB1A8301847704700BFF0
:10A410009C1500200348D0F894300BB18C301847BD
:10A42000704700BF9C1500200248836F0BB170304D
:10A43000184770479C1500200248C36D0BB154307B
:10A44000184770479C1500200248036C0BB1383048
:10A45000184770479C1500200248436A0BB11C3016
:10A46000184770479C1500200248836803B11847BD
:10A47000704700BF9C150020F8B584894FF6FF7621
:10A480004FF47A7433B319B30F78013101E0B44259
:10A4900018D00589013CAD07A4B2F8D5BCB28481BF
:10A4A0004FF47A7402E0BCB2B4420BD00589ED07D8
:10A4B00004F1FF37F7D58589ADB20AB115700132C5
:10A4C000013BDFE714F092FF003018BF0120F8BD18
:10A4D000FF27DEE70120F8BDF8B50501684C694BA0
:10A4E000625961199A4204EB050704BF01230B73FB
:10A4F0000646387A2BF064F83B7A03F01F015B09BB
:10A500000122032B02FA01F26DD0042B66D0022B3C
:10A510005CD063190136187902F0BEFEF6B2074628
:10A5200010B11223C67183716319587902F0B4FE19
:10A5300010B11323C67183716319987902F0ACFED0
:10A5400010B11423C671837166190A21F279384655
:10A5500002F00AFD707902F09FFEF2790A2102F002
:10A5600003FDB07902F098FEF2790A2102F0FCFCBA
:10A570006359454A934247D0424A934250D0434A96
:10A58000934259D0424A934262D0424A93426BD09E
:10A59000414A93422CD02C44227BE2B90120022272
:10A5A000198801F4415141F445710A4302431A806C
:10A5B0009A8B22F400621204120C07219A831982EA
:10A5C0001A8892B242F040021A80F8BD334B596AA1
:10A5D0000A435A629DE700200246E1E72F4B1969C2
:10A5E0000A431A6195E72D4B196A0A431A6290E7EC
:10A5F00002F564424FF40010536A43F400135362AF
:10A6000027F0ECFC6359C6E702F584324FF4805022
:10A61000536A43F48053536227F0E0FC6359BAE76E
:10A6200002F500324FF48040136A43F48043136212
:10A6300027F0DCFC6359AEE702F5FE324FF4004030
:10A64000136A43F40043136227F0D0FC6359A2E776
:10A6500002F582324FF40050536A43F400535362C0
:10A6600027F0BCFC635996E702F568424FF480106E
:10A67000536A43F48013536227F0B0FC63598AE7AE
:10A68000987D00200038004000300140003C004030
:10A6900000340140005001400054014000380240A5
:10A6A000431C00F014812DE9F04F4FEAC00808EB7D
:10A6B00000039B00DFF8F4A25AF803B087B00AEB5E
:10A6C0000304BBF1000F00F0FF8014330AEB030119
:10A6D0000022DBF804704AF803204A608A60CA60EE
:10A6E0000346A56801900133D4F80C90DBB2002D2D
:10A6F00000F0EE801522EB71AA71B9F1000F00F0A5
:10A700000081162289F8062089F807309BF80E0090
:10A710002AF056FFBB8823F440731B041B0CBB803C
:10A72000284603F047FE484603F044FE1121284620
:10A7300003F02CFC1121484603F028FC0826642471
:10A7400004E00A203CB103F087F9013C284603F0FD
:10A7500083FE0028F5D0284603F026FE0A2003F0E9
:10A760007BF9284603F026FE0A2003F075F9013E26
:10A77000ECD1484603F018FE0A2003F06DF9284694
:10A7800003F012FE0A2003F067F9284603F012FED8
:10A790000A2003F061F9484603F00CFE019B08EB28
:10A7A00003040AEB84042846637C002B0CBF1221AF
:10A7B0003221042202F0D8FB637C002B0CBF122153
:10A7C00032214846042202F0CFFB704B9F4200F03A
:10A7D000B7806F4B9F4200F0BD806E4B9F4200F0F0
:10A7E000A580BB8801996C4A6C4C23F440731B0410
:10A7F0001B0CBB803B8888440AEB880A9BB243F061
:10A8000001039AF810103B80BD8802A8002918BFE8
:10A81000144627F0F3FB049A6148B2FBF4F325F0E9
:10A820003F05A0FB02122D04900C2D0C0543BD80AA
:10A830005C4C39884FF4967202FB00F284FB0240B4
:10A840009BB2D217002BC2EBA01221F0010108BF6E
:10A8500001230904013243F40043090C92B2398008
:10A860003A84BB833B889BB243F001033B803B8827
:10A8700023F4816323F002031B041B0C43F4806365
:10A880004FF480423B803A813B8823F080031B04D5
:10A890001B0C3B809BF810308DF8083000240123FE
:10A8A00002A88DF80B308DF809408DF80A4027F08A
:10A8B0005DFB9BF80F308DF8083002A88DF8094039
:10A8C0008DF80A4027F078FB07B0BDE8F08F70479D
:10A8D000B9F1000F48D0162289F8073089F8062010
:10A8E0009BF80E002AF06CFEBB8823F440731B0417
:10A8F0001B0C2846BB8003F05DFD484603F05AFD63
:10A9000018E79BF80E002AF05BFEBB8823F4407327
:10A910001B041B0CBB80284603F04CFD484603F08B
:10A9200049FD1121284603F031FB07E71E4A136A4F
:10A9300043F4000313624FF4000027F057FB50E785
:10A94000194A136A43F4001313624FF4001027F0FE
:10A950004DFB46E7144A136A43F4800313624FF435
:10A96000800027F043FB3CE79BF80E002AF028FE0E
:10A97000BB8823F440731B041B0C4846BB8003F0C8
:10A9800019FD484603F016FDD8E600BF005400400C
:10A9900000580040005C0040009F2400804F1200DF
:10A9A00083DE1B43D34D6210003802408035002007
:10A9B000F0B5C60033189B00254DEA585468A28AAA
:10A9C00083B092B20192019A2B4412F4706F1CBFB3
:10A9D00001221A75019B13F4E06F07460CD1A38A7C
:10A9E0003E4423F4706305EB86051B041B0C002218
:10A9F000A3826A7503B0F0BD238BA38823F4806320
:10AA00001B041B0CA380019B9B05E8D4238898059D
:10AA1000E5D42388D9050ED52388DA05FCD423880C
:10AA20009BB243F40073238023889B05FCD43846F3
:10AA3000FFF736FED3E723889BB243F400732380ED
:10AA4000A38823F440731B041B0CA380C7E700BF3B
:10AA500080350020F0B5037C012B83B005462DD056
:10AA6000022B31D1836913B11A689B885383C321A8
:10AA70006869FDF74BFE06236A4600216869FFF707
:10AA8000FBFCAB6913B11A689B8813839DF8040023
:10AA90009DF800609DF801109DF802409DF803208C
:10AAA0009DF8053041EA062143EA002342EA0422E8
:10AAB000012029876A87AB8703B0F0BD90F91400A5
:10AAC000461C01D0032802DD002003B0F0BDC70002
:10AAD000274E3A1806EB820251680029F4D06C7DAB
:10AAE0006400E4B294754FF0000E06244FF0430C5E
:10AAF00082F817C082F819E093761476537582F8BD
:10AB000014E08B88C2F820D09C05C2F81CD014D465
:10AB10000B88DA050CD44FF4805401E0013C1DD0C1
:10AB20000B889B05FAD40B889BB243F480730B808F
:10AB30008B889BB243F440738B80074406EB8702FB
:10AB40004FF4805401E0013C08D0537D002BFAD132
:10AB500006EB87073B7D002B98D0B5E7054A1388A5
:10AB600001339BB21380FFF79BFD2046ADE700BF8A
:10AB700080350020903B0020F0B5037A012B83B094
:10AB800005462DD0022B31D1036913B11A689B8879
:10AB90005383BB21E868FDF7B9FD06236A4600210F
:10ABA000E868FFF769FC2B6913B11A689B88138367
:10ABB0009DF804009DF800609DF801109DF802408A
:10ABC0009DF803209DF8053041EA062143EA002361
:10ABD00042EA04220120E9822A836B8303B0F0BD9C
:10ABE00090F90C00461C01D0032802DD002003B0C0
:10ABF000F0BDC700274E3A1806EB820251680029C3
:10AC0000F4D06C7B6400E4B294754FF0000E06241F
:10AC10004FF03B0C82F817C082F819E09376147657
:10AC2000537582F814E08B88C2F820D09C05C2F8D6
:10AC30001CD014D40B88DA050CD44FF4805401E0F6
:10AC4000013C1DD00B889B05FAD40B889BB243F4C2
:10AC500080730B808B889BB243F440738B800744D6
:10AC600006EB87024FF4805401E0013C08D0537D8D
:10AC7000002BFAD106EB87073B7D002B98D0B5E778
:10AC8000054A138801339BB21380FFF709FD204664
:10AC9000ADE700BF80350020903B0020F0B583B0C9
:10ACA000441C8DF8073001D0032802DD002003B0DA
:10ACB000F0BDC700244E3B1806EB83035D68002DF2
:10ACC000F4D04900C9B2997501240021DA755C7687
:10ACD00099761C765C751975A9880DF107028905AE
:10ACE000DA611A6214D42B88DA050CD44FF480543C
:10ACF00001E0013C1ED02B889B05FAD42B889BB227
:10AD000043F480732B80AB889BB243F44073AB80D9
:10AD1000074406EB87024FF4805401E0013C09D060
:10AD2000537D002BFAD106EB87073C7D84F00100B0
:10AD300003B0F0BD054A138801339BB21380FFF7BF
:10AD4000AFFC2046B3E700BF80350020903B0020D9
:10AD50002DE9F04F85B0019090F85500002840F0A3
:10AD60005386019A137C012B00F08F86022B12D19F
:10AD7000936913B11A689B885383019C6B216069A6
:10AD8000FDF7C4FC80216069FDF7C0FCA36913B125
:10AD90001A689B881383B14CB14DDFF8CC92B1484F
:10ADA000DFF8C8E24FF0640A4FF0100C4FF47A76E7
:10ADB000D9F80430C3F30803002B40F09585EFF376
:10ADC0001183002B40F090852168826800BF2368C2
:10ADD0009942F9D12F6806FB07F39B1AB3FBF7F3EF
:10ADE00006FB013101270091D9F80430C3F30803B1
:10ADF000002B40F0C383EFF31183002B40F0BE83A0
:10AE00002368816800BF22689342F9D1D5F800B069
:10AE100006FB0BF2521AB2FBFBF206FB0323009A6D
:10AE20009B1AB3F57A7FDFD3BAF1010AC0D1019A38
:10AE3000137C012B00F03386022B12D1936913B1DE
:10AE40001A689B885383019E68217069FDF75EFC38
:10AE500007217069FDF75AFCB36913B11A689B8822
:10AE60001383DFF804927F4EDFF800C24FF0640ACC
:10AE70004FF010084FF47A77D9F80430C3F3080381
:10AE8000002B40F04E85EFF31183002B40F04985F5
:10AE90002168B26800BF23689942F9D1286807FB8E
:10AEA00000F39B1AB3FBF0F307FB01310120009183
:10AEB000D9F80430C3F30803002B40F07C83EFF390
:10AEC0001183002B40F077832368B16800BF2268AC
:10AED0009342F9D1D5F800B007FB0BF2521AB2FB3E
:10AEE000FBF207FB0323009A9B1AB3F57A7FDFD3AB
:10AEF000BAF1010AC0D1019A137C012B00F0068639
:10AF0000022B12D1936913B11A689B885383019E57
:10AF10006B217069FDF7FAFB00217069FDF7F6FB04
:10AF2000B36913B11A689B881383DFF83C914D48CD
:10AF3000DFF838E14FF0640A4FF0100C4FF47A76E6
:10AF4000D9F80430C3F30803002B40F09384EFF3E7
:10AF50001183002B40F08E842168826800BF236833
:10AF60009942F9D12F6806FB07F39B1AB3FBF7F35D
:10AF700006FB013101270091D9F80430C3F308031F
:10AF8000002B40F03583EFF31183002B40F030832A
:10AF90002368816800BF22689342F9D1D5F800B0D8
:10AFA00006FB0BF2521AB2FBFBF206FB0323009ADC
:10AFB0009B1AB3F57A7FDFD3BAF1010AC0D1019AA7
:10AFC000137C012B00F09985022B12D1936913B1E8
:10AFD0001A689B885383019E6B217069FDF796FB6D
:10AFE00001217069FDF792FBB36913B11A689B8860
:10AFF0001383DFF874901B48DFF870E04FF00F0AFE
:10B000004FF0100C4FF47A76D9F80430C3F30803EC
:10B01000002B40F04C84EFF31183002B40F0478469
:10B020002168826800BF23689942F9D12F6806FB26
:10B0300007F39B1AB3FBF7F306FB013101270091DD
:10B04000D9F80430C3F30803002B40F0EE82EFF38D
:10B050001183002B40F0E9820AE000BF0C7D002044
:10B06000107D002010E000E000ED00E0087D0020F1
:10B070002368816800BF22689342F9D1D5F800B0F7
:10B0800006FB0BF2521AB2FBFBF206FB0323009AFB
:10B090009B1AB3F57A7FD3D3BAF1010AB4D10199DF
:10B0A00091F84F200B7C032A8CBF1A261826012BFF
:10B0B00000F04085022B12D18A6912B11368928880
:10B0C0005A83019F1B217869FDF720FB314678697F
:10B0D000FDF71CFBBB6913B11A689B881383DFF86B
:10B0E000CC92B148DFF8C8E24FF00F0A4FF0100CD5
:10B0F0004FF47A76D9F80430C3F30803002B40F0FC
:10B100008183EFF31183002B40F07C8321688268F8
:10B1100000BF23689942F9D12F6806FB07F39B1AF9
:10B12000B3FBF7F306FB013101270091D9F8043096
:10B13000C3F30803002B40F09582EFF31183002B3B
:10B1400040F090822368816800BF22689342F9D161
:10B15000D5F800B006FB0BF2521AB2FBFBF206FB6D
:10B160000323009A9B1AB3F57A7FDFD3BAF1010A61
:10B17000C0D1019A137C012B00F0D284022B12D192
:10B18000936913B11A689B885383019E1C217069CF
:10B19000FDF7BCFA18217069FDF7B8FAB36913B16D
:10B1A0001A689B881383DFF804927F48DFF800E277
:10B1B0004FF00F0A4FF0100C4FF47A76D9F80430A4
:10B1C000C3F30803002B40F03983EFF31183002B06
:10B1D00040F034832168826800BF23689942F9D126
:10B1E0002F6806FB07F39B1AB3FBF7F306FB01314D
:10B1F00001270091D9F80430C3F30803002B40F075
:10B200004E82EFF31183002B40F04982236881685E
:10B2100000BF22689342F9D1D5F800B006FB0BF2CB
:10B22000521AB2FBFBF206FB0323009A9B1AB3F5FA
:10B230007A7FDFD3BAF1010AC0D101990B7C91F872
:10B240004E60012B00F03E84022B12D18A6912B1AC
:10B25000136892885A83019F1A217869FDF756FA7C
:10B2600031467869FDF752FABB6913B11A689B88B9
:10B270001383DFF838914C48DFF834E14FF00F0AC0
:10B280004FF0100C4FF47A76D9F80430C3F308036A
:10B29000002B40F09B82EFF31183002B40F096824D
:10B2A0002168826800BF23689942F9D12F6806FBA4
:10B2B00007F39B1AB3FBF7F306FB0131012700915B
:10B2C000D9F80430C3F30803002B40F00582EFF3F4
:10B2D0001183002B40F000822368816800BF226840
:10B2E0009342F9D1D5F800B006FB0BF2521AB2FB2B
:10B2F000FBF206FB0323009A9B1AB3F57A7FDFD398
:10B30000BAF1010AC0D101990B7C91F85060012B70
:10B3100000F0CF83022B12D18A6912B11368928890
:10B320005A83019F19217869FDF7F0F93146786950
:10B33000FDF7ECF9BB6913B11A689B881383DFF83A
:10B340006C901948DFF868E04FF0640A4FF0100C79
:10B350004FF47A76D9F80430C3F30803002B40F099
:10B36000FD82EFF31183002B40F0F88221688268A0
:10B3700000BF23689942F9D12F6806FB07F39B1A97
:10B38000B3FBF7F306FB013101270091D9F8043034
:10B39000C3F30803002B40F0C381EFF31183002BAC
:10B3A00040F0BE8106E000BF10E000E000ED00E0EC
:10B3B000087D00202368816800BF22689342F9D18C
:10B3C000D5F800B006FB0BF2521AB2FBFBF206FBFB
:10B3D0000323009A9B1AB3F57A7FD7D3BAF1010AF7
:10B3E000B8D1019A137C012B00F07E83022B12D17D
:10B3F000936913B11A689B885383019E3721706942
:10B40000FDF784F910217069FDF780F9B36913B174
:10B410001A689B881383DFF80493BE48DFF8F8E2CC
:10B420004FF00F0A4FF0100C4FF47A76D9F8043031
:10B43000C3F30803002B40F0AD82EFF31183002B20
:10B4400040F0A8822168826800BF23689942F9D140
:10B450002F6806FB07F39B1AB3FBF7F306FB0131DA
:10B4600001270091D9F80430C3F30803002B40F002
:10B470007481EFF31183002B40F06F8123688168A2
:10B4800000BF22689342F9D1D5F800B006FB0BF259
:10B49000521AB2FBFBF206FB0323009A9B1AB3F588
:10B4A0007A7FDFD3BAF1010AC0D1019A137C012B54
:10B4B00000F01283022B12D1936913B11A689B8892
:10B4C0005383019E38217069FDF720F901217069CD
:10B4D000FDF71CF9B36913B11A689B881383DFF871
:10B4E0003C828C498C4F4FF00F094FF0100E4FF4F7
:10B4F0007A70D8F80430C3F30803002B40F066825A
:10B50000EFF31183002B40F0618222688E6800BF48
:10B5100023689A42F9D1D5F800C000FB0CF39B1BBD
:10B52000B3FBFCF300FB023300930126D8F8043090
:10B53000C3F30803002B40F02D81EFF31183002BA0
:10B5400040F028812368D1F808A000BF2268934208
:10B55000F8D1D5F800B000FB0BFCACEB0A0CBCFB3F
:10B56000FBFC00FB03C3009A9B1AB3F57A7FDDD383
:10B57000B9F10109BDD105B0BDE8F08FEFF3118835
:10B580008CF3128881680368DB0344BFCEF8007037
:10B5900081682368DEF800205FFA88F888F3118854
:10B5A000D5F800801A4406FB08F35B1AB3FBF8F3E6
:10B5B00006FB023333E4EFF3118E88F31288B1688F
:10B5C0003368DB0344BFCCF80000B1682368DCF8C3
:10B5D00000205FFA8EFE8EF31188D5F800E01A4441
:10B5E00007FB0EF35B1AB3FBFEF307FB02337AE4AF
:10B5F000EFF311888CF3128881680368DB0344BF82
:10B60000CEF8007081682368DEF800205FFA88F8C1
:10B6100088F31188D5F800801A4406FB08F35B1AFA
:10B62000B3FBF8F306FB0233C1E4EFF311888CF3AC
:10B63000128881680368DB0344BFCEF8007081681C
:10B640002368DEF800205FFA88F888F31188D5F8BF
:10B6500000801A4406FB08F35B1AB3FBF8F306FB01
:10B66000023314E5EFF311888CF3128881680368C4
:10B67000DB0344BFCEF8007081682368DEF8002049
:10B680005FFA88F888F31188D5F800801A4406FB21
:10B6900008F35B1AB3FBF8F306FB023361E5EFF343
:10B6A00011888CF3128881680368DB0344BFCEF8ED
:10B6B000007081682368DEF800205FFA88F888F35C
:10B6C0001188D5F800801A4406FB08F35B1AB3FB17
:10B6D000F8F306FB0233A8E5EFF311888CF3128828
:10B6E00081680368DB0344BFCEF80070816823687B
:10B6F000DEF800205FFA88F888F31188D5F800801A
:10B700001A4406FB08F35B1AB3FBF8F306FB02339B
:10B71000F1E500BF10E000E0087D002000ED00E052
:10B72000EFF311888CF3128881680368DB0344BF50
:10B73000CEF8007081682368DEF800205FFA88F890
:10B7400088F31188D5F800801A4406FB08F35B1AC9
:10B75000B3FBF8F306FB02333BE6EFF311888CF3FF
:10B76000128881680368DB0344BFCEF800708168EB
:10B770002368DEF800205FFA88F888F31188D5F88E
:10B7800000801A4406FB08F35B1AB3FBF8F306FBD0
:10B79000023382E6EFF3118A8EF312888A680B680F
:10B7A000DB0344BF3E608A682368D7F800C05FFAB5
:10B7B0008AFA8AF31188D5F800A09C4400FB0AF3AA
:10B7C0009B1AB3FBFAF300FB0C33CCE6EFF31182C8
:10B7D0008CF3128887680368D90303D50123CEF858
:10B7E000003087682368DEF80010D2B282F3118837
:10B7F0002A68194406FB02F3DB1BB3FBF2F306FBDA
:10B8000001315BE5EFF311828CF3128887680368DE
:10B81000D90303D50123CEF8003087682368DEF80A
:10B820000010D2B282F311882A68194406FB02F391
:10B83000DB1BB3FBF2F306FB013175E4EFF311827E
:10B840008CF3128887680368D90303D50123CEF8E7
:10B85000003087682368DEF80010D2B282F31188C6
:10B860002A68194406FB02F3DB1BB3FBF2F306FB69
:10B870000131BDE4EFF311828CF31288876803680D
:10B88000D90303D50123CEF8003087682368DEF89A
:10B890000010D2B282F311882A68194406FB02F321
:10B8A000DB1BB3FBF2F306FB0131FFF763BBEFF3E6
:10B8B00011828CF3128887680368D90303D50123AA
:10B8C000CEF8003087682368DEF80010D2B282F329
:10B8D00011882A68194406FB02F3DB1BB3FBF2F361
:10B8E00006FB0131FFF7AABBEFF311828CF312883C
:10B8F00087680368D90303D50123CEF80030876831
:10B900002368DEF80010D2B282F311882A68194445
:10B9100006FB02F3DB1BB3FBF2F306FB0131FFF77F
:10B9200061BAEFF3118288F31288B0683368D903E3
:10B9300003D50123CCF80030B0682368DCF8001090
:10B94000D2B282F311882A68194407FB02F31B1A4A
:10B95000B3FBF2F307FB0131FFF7A8BAEFF3118253
:10B960008CF3128887680368D90303D50123CEF8C6
:10B97000003087682368DEF80010D2B282F31188A5
:10B980002A68194406FB02F3DB1BB3FBF2F306FB48
:10B990000131F9E4EFF311828CF3128887680368B0
:10B9A000D90303D50123CEF8003087682368DEF879
:10B9B0000010D2B282F311882A68194406FB02F300
:10B9C000DB1BB3FBF2F306FB013149E5EFF3118614
:10B9D0008EF31288D1F808C00B68DA0303D501236F
:10B9E0003B60D1F808C023683A68F6B286F3118844
:10B9F0002E681A4400FB06F3A3EB0C03B3FBF6F32B
:10BA000000FB0233009390E501F046FC0446002859
:10BA100000F09F800068584900F13F4303F57E0322
:10BA20009A0A20258A5CA57102F01F06520901239B
:10BA30000021032A03FA06F3E17100F09780042A3B
:10BA400000F08F80022A7FD0A388029302A90023EE
:10BA5000039326F01BFD0199484B41F80C3F20460B
:10BA60002AF08CFAA388B3FA83F3C3F11F030122EF
:10BA700012FA03F33FF475A941490A681343019A86
:10BA80000B60137C012B7FF471A910468023417D4C
:10BA900090F914006B22FFF701F9FFF77CB910460B
:10BAA0000723417D90F914006822FFF7F7F8FFF7AC
:10BAB000D8B9084633461922497D90F91400FFF79A
:10BAC000EDF83CE4084633461A22497D90F914000B
:10BAD000FFF7E4F8FFF7CDBB10463822417D90F91F
:10BAE0001400FFF7DBF8FAE410461023417D90F9CB
:10BAF00014003722FFF7D2F88DE410466B22417D07
:10BB000090F91400FFF7CAF8FFF773BA10465346CE
:10BB1000417D90F914006B22FFF7C0F8FFF705BADA
:10BB200010461823417D90F914001C22FFF7B6F847
:10BB3000FFF739BB084633461B22497D90F91400B4
:10BB4000FFF7ACF8FFF7CBBA0E4A516C0B435364C6
:10BB50007AE70199094B41F80C3F2AF00FFAFFF7F9
:10BB600000B9084A116B0B4313636DE7054A116C6A
:10BB70000B43136468E700BFDC6F04080180000812
:10BB8000003C0140003802402DE9F04F8A4A4369E9
:10BB900083B09342019000F00D8188498B420CBF25
:10BBA000282130211A8822F040021204120C1A8037
:10BBB0001A8892B222F03802114319801A8892B280
:10BBC00042F040021A80012001F046FF019C20460D
:10BBD000FFF7BEF8A36913B11A689B885383019BD2
:10BBE000586940F2E93302E0002B00F0DB80028963
:10BBF000013B12F0020F9BB2F6D06A23838140F220
:10BC0000E93302E0002B00F0CD800289013B12F005
:10BC1000010F9BB2F6D0838940F2E93302E0002B9A
:10BC200000F0C5800289013B12F0020F9BB2F6D0F2
:10BC30001023838140F2E93302E0002B00F0B7804B
:10BC40000289013B12F0010F9BB2F6D08389019B60
:10BC50009B6913B11A689B881383594CDFF86CE118
:10BC6000DFF86C915748584F4FF0640A4FF0100CB2
:10BC70004FF47A75D9F80430C3F30803002B76D15A
:10BC8000EFF31183002B72D12168826800BF236813
:10BC90009942F9D1DEF8006005FB06F39B1AB3FB6D
:10BCA000F6F305FB013101260091D9F80430C3F306
:10BCB0000803002B40D1EFF31183002B3CD1236804
:10BCC000816800BF22689342F9D1DEF800B005FB1D
:10BCD0000BF2521AB2FBFBF205FB0323009A9B1AEC
:10BCE000B3F57A7FE1D3BAF1010AC3D1019B324A9D
:10BCF0005B69934207D0DFF8C4A0534514BF4FF0EF
:10BD0000080A4FF0000A1A8822F040021204120CAE
:10BD10001A801A8892B222F038024AEA020AA3F87C
:10BD200000A01A8892B242F0400201201A8003B0AB
:10BD3000BDE8F04F01F090BEEFF311888CF312884C
:10BD400081680368DB0344BF3E60816823683A680A
:10BD50005FFA88F888F31188DEF800801A4405FB42
:10BD600008F35B1AB3FBF8F305FB0233B6E7EFF316
:10BD700011828CF3128886680368D90302D50123E7
:10BD80003B60866823683968D2B282F31188DEF896
:10BD90000020194405FB02F39B1BB3FBF2F305FBE8
:10BDA000013180E713F022FB019B586934E713F05F
:10BDB0001DFB4CE72821F5E600380040003C004020
:10BDC0000C7D002010E000E0087D0020107D0020A8
:10BDD00000ED00E00220FCF70DBA00BF0220FEF7E4
:10BDE000E7BD00BF0120FCF705BA00BF0120FEF748
:10BDF000DFBD00BF0020FCF7FDB900BF0020FEF74B
:10BE0000D7BD00BF1549164B16480A6810B48C6898
:10BE10001549B2FBF4F203FB02F30360D1F888206A
:10BE2000124B134C42F47002C1F888201A680020AB
:10BE300042F001021A6098601A6822F0847222F4BB
:10BE400080321A605C601A684FF0006422F480222D
:10BE50001A60D8608C605DF8044B704700000020C9
:10BE600040420F00CC85002000ED00E00038024089
:10BE700010300024044B4FF4F0700A21022283E8B2
:10BE80000700FFF7BFBF00BF000000200D4B0121DE
:10BE90000022890710B4027203F1780402D51979DF
:10BEA000815401329C4203F1180308D0072A06DCB2
:10BEB00099798907F3D49C4203F11803F6D15DF810
:10BEC000044B70472C70040839230370704700BF7F
:10BED000012310B433213124322244704171C270E5
:10BEE00003720370037183705DF8044B704700BFE9
:10BEF0002322032302704370704700BF436A8269A4
:10BF0000D154436A0169826B01338B4228BF0023FD
:10BF10004362002A2FD0EFF31182502383F312885B
:10BF2000836B1968C9072CD470B45E686EB9456A12
:10BF3000816A8D4217D084690C44DC600ED9691A7D
:10BF400059608562002180F85C10196841F0010198
:10BF5000D2B2196082F3118870BC70470469611A0B
:10BF600059608662EEE7012380F85C30D2B282F33A
:10BF7000118870BC7047826DD36843F08003D36032
:10BF80007047D2B282F31188704700BF426B10B481
:10BF900062B1C36CC2684469D11A013B615C5DF84F
:10BFA000044B08BF1346C364C8B27047016A4369B3
:10BFB000C4685B5C0131A14228BF114601625DF893
:10BFC000044BD8B2704700BF836B13B190F85C008C
:10BFD0007047836A406A181AB0FA80F040097047C7
:10BFE000416A836A99420AD3CB1A816B026961B1B3
:10BFF0004968501E0B4483420AD2C01A7047026936
:10C000001144CB1A816B0029F2D1501EC01A70471F
:10C0100000207047436B43B1C26C5B6893422FBFF3
:10C02000981AC0689B1AC0187047C269036A9A427E
:10C030002FBFD01AC0688018C01A70470A4B30B59D
:10C0400003F1140493F900205D78072AC8BF143A5D
:10C05000811804330D7313F8025C855413F8012C16
:10C060000A76A342EED130BD5845040803682DE995
:10C07000F041DF691FB13B46BDE8F0411847002A97
:10C08000164611DD04460D460E4400E023689B6809
:10C09000204698470028F9D0236815F8011B1B6833
:10C0A00020469847AE42F1D1BDE8F081002325211A
:10C0B0002422017042708370C3707047038A2DE997
:10C0C000F0478589ADB21D4029D00F4606464FF096
:10C0D00000484FF00009B5FA85F328FA03F2D2437D
:10C0E00091B21B3B15403182042B16D8DFE803F0D8
:10C0F0003129211903007B6A002B32D003F1FF3A6A
:10C100001FFA8AFAC7F824903C6A34B123682046A3
:10C11000514698476468002CF8D1002DDBD1BDE86A
:10C12000F0873868716B036889B29847002DD2D1C7
:10C13000F5E77868B16B036889B29847002DCAD1DA
:10C14000EDE7B868F16B036889B29847002DC2D15A
:10C15000E5E7F868316C036889B29847002DBAD1D9
:10C16000DDE7F36A1FFA83FACEE700BF30B5044675
:10C17000806D61718389A26823F400531B041B0C3A
:10C18000838185B0A379009213F0040230D04FF47C
:10C19000805213F00203ADF8042056D1ADF80630FA
:10C1A0004FF480630022ADF8083011F00103ADF8C0
:10C1B0000C2028D1ADF80A3008238D07694648BF06
:10C1C000ADF80A3025F068FFA279A36DD10724D419
:10C1D00012F0080F9A8A1BD122F008021204120CE6
:10C1E0009A829A8992B242F400529A8105B030BD87
:10C1F00013F00203ADF8042024D04FF40055134689
:10C20000ADF80650CEE70423ADF80A300C23D4E78E
:10C2100092B242F008029A82E3E70D498B420FD0B6
:10C22000A1F548418B4209D00A498B42D0D1052063
:10C230000121FDF7B3FDA279A36DC9E70220F7E75D
:10C240000020F5E7ADF80630ACE74FF40053A5E762
:10C25000001001400014014010B50446806DA1603B
:10C26000838923F400531B041B0C8381A37984B0BE
:10C2700013F00402009135D04FF4805213F0020302
:10C28000ADF8042056D1ADF806304FF480636279E2
:10C29000ADF80830D1074FF00003ADF80A30ADF823
:10C2A0000C3045BF0423ADF80A3008230C2369463F
:10C2B000920748BFADF80A3025F0EEFEA279A36DD3
:10C2C000D1071FD412F0080F9A8A16D122F0080263
:10C2D0001204120C9A829A8992B242F400529A8104
:10C2E00004B010BD13F00203ADF804201FD04FF4CA
:10C2F00000511346ADF80610C9E792B242F00802A9
:10C300009A82E8E70D498B420FD0A1F548418B4254
:10C3100009D00B498B42D5D105200121FDF73EFD07
:10C32000A279A36DCEE70220F7E70020F5E7ADF88C
:10C330000630ACE74FF40053A5E700BF0010014002
:10C3400000140140022828BF022010B4084C094BF9
:10C35000207000EB8002C0EBC20207495DF8044B7D
:10C36000013003EB4203C0B20B6011F017BE00BFF7
:10C370008CA70020664D0020004D002008B519F064
:10C3800083FF13F05BFABDE8084019F065BF00BFFA
:10C390002DE98048013085B0C3B203938B4D8C4F9B
:10C3A0008C4C8D4E0A2302933220DFF8309229F014
:10C3B00027FB4FF4FA7A4FF0100C4FF47A70D9F84B
:10C3C0000430C3F30803002B40F0C180EFF3118366
:10C3D000002B40F0BC802968A26800BF2B689942FE
:10C3E000F9D1D7F800E000FB0EF39B1AB3FBFEF384
:10C3F00000FB01314FF0010E0191D9F80430C3F375
:10C400000803002B40F08780EFF31183002B40F0EE
:10C4100082802B68A16800BF2A689342F9D1D7F8BF
:10C4200000B000FB0BF2521AB2FBFBF200FB03233D
:10C43000019A9B1AB3F57A7FDFD3BAF1010ABED114
:10C44000039B002B40F0BD804FF47A7ADFF88C918B
:10C4500050464FF0100CD9F80430C3F30803002BFA
:10C4600040F09280EFF31183002B40F08D8029681B
:10C47000A26800BF2B689942F9D1D7F800E000FB11
:10C480000EF39B1AB3FBFEF300FB01314FF0010EDC
:10C490000191D9F80430C3F3080303BBEFF3118310
:10C4A000EBB92B68A16800BF2A689342F9D1D7F88D
:10C4B00000B000FB0BF2521AB2FBFBF200FB0323AD
:10C4C000019A9B1AB3F57A7FE3D3BAF1010AC2D17C
:10C4D000029B013B02937FF467AFFDF7B5F9EFF3E1
:10C4E00011888CF31288A1682368DB0344BFC6F867
:10C4F00000E0A1682B6832685FFA88F888F3118839
:10C50000D7F800801A4400FB08F35B1AB3FBF8F37A
:10C5100000FB0233D4E7EFF311888CF31288A16893
:10C520002368DB0344BFC6F800E0A1682B683268CB
:10C530005FFA88F888F31188D7F800801A4400FB66
:10C5400008F35B1AB3FBF8F300FB023370E7EFF379
:10C5500011828CF31288D4F808E02368D90303D53C
:10C5600001233360D4F808E02B683168D2B282F33B
:10C5700011883A68194400FB02F3A3EB0E03B3FBE6
:10C58000F2F300FB013135E7EFF311828CF31288EF
:10C59000D4F808E02368D90303D501233360D4F825
:10C5A00008E02B683168D2B282F311883A681944E6
:10C5B00000FB02F3A3EB0E03B3FBF2F300FB01312C
:10C5C00064E7184629F07EF83EE700BF0C7D0020A6
:10C5D000107D002010E000E0087D002000ED00E06C
:10C5E00038B5484B5A899989914224BF00225A8113
:10C5F000198ADA89914224BF0022DA81DA78CAB135
:10C60000072A41496AD091F85300404D0124002186
:10C610000A282C709C70D9715DD00C2807D0002A94
:10C620006CD0DFED3B7A072A0ED00A2862D0DFED0E
:10C63000397A09E0344A92F853000A2856D00C2877
:10C640005BD1D979DFED347A344C9FED350AA2788D
:10C65000002918BFF0EE407A062A04D8314901EBD0
:10C66000820191ED050A217979B1013A032A0BD8AB
:10C67000F7EE007A87EE800A36F02AFF2388984288
:10C6800028BF1846208038BD38BD9B781F4A07EE6A
:10C69000103A1178B8EEC77A67EE277A07EE101ACB
:10C6A000B8EEC77A27EE277AB4EEC70AF1EE10FA91
:10C6B000EADD80EE277AFDEEC77A17EE903A102B6E
:10C6C000A8BF1023012BB8BF0123DBB28B4238BFB8
:10C6D0000B46137038BDDFED147AA4E791F85300D0
:10C6E0000A2803D00C28ACD0D9799AE7D979DFEDA4
:10C6F0000E7AA9E7DFED0D7AA6E7D979DFED047AA6
:10C70000A2E700BFAC8D0020D0850020005400209F
:10C710006F1203396F12833A0AD7A339D059002018
:10C720006F120338584504085304E9380F506E3A25
:10C730002DE9F047AC4FAD4E19F0A6FDBE421ED21A
:10C74000DFF82C83DFF82C934446258862197DB1ED
:10C750004A450DD2052D0BD933886188C3F30B03ED
:10C76000994200F0E480144625886219002DEFD12B
:10C7700071683046143612F0EDFFBE42E4D39C4A95
:10C780001378A3F1170102290FD99A4911F8330040
:10C79000002840F0FB80D8000144497829B196492F
:10C7A00011F833300BB918231370944B5A78022ABE
:10C7B00000F2DD809249934802EB420201EB8201D4
:10C7C0001A780160022A00F2DB8002EB82018E4BB4
:10C7D000C2EBC10203EB4203998C5A8C8B4C914201
:10C7E000236001D300225A84894B9A78042A00F0EE
:10C7F000EE8032B91A88B2F5F07F84BF4FF4F07240
:10C800001A80844DFFF7ECFE2B68834A1A40002AF9
:10C8100000F0E680D80700F1D580590400F1CD8002
:10C820001A0700F1BC809B0400F1C0802AF018FEBA
:10C8300010B97A4810F0B6F94FF4007012F0C0FF4A
:10C840004FF4802012F0BCFF4FF4001012F0B8FF3C
:10C850004FF0007012F0B4FF4FF0806012F0B0FFA4
:10C860002FF04AFF002130226D4837F0EEFD20689E
:10C870002EF092FE6B4B256803F1500103E0043368
:10C88000994200F081801A78002AF8D19C78D878F3
:10C890008442F4D26449654B0A7028461D6031F029
:10C8A000F9F8634A63491079634A644B1160C822FE
:10C8B000642111FB0021002259609A60DA601A613C
:10C8C0005A619A61DA6183F8202083F8212027F0E9
:10C8D0003FF95B4B9FED5B5A1B885B4A9FED5B6AA0
:10C8E00055795B4C5B495C48086006EE903AF8EE7F
:10C8F000E66A1388C5EE265A07EE103A5388127975
:10C90000C4ED005A07EE903AB8EEC77A534BF8EEF2
:10C91000E77A1D725A7227EE067A67EE867ABDE8CC
:10C92000F04783ED017AC3ED007A19F095BC637985
:10C930009B077FF418AF716894F804A0304612F09A
:10C9400009FF3388BAEB133F04D01436BE42FFF41C
:10C95000FBAE14E773887068AA1FC3F30B039A42F7
:10C9600004F10601A8BF1A4636F072FCEDE700227A
:10C970005A701A78234822490160022A7FF625AFAF
:10C9800000221A70204B27E7012283E7D8000C18F9
:10C990006468002C7FF400AF17241470FCE6304864
:10C9A00012F00EFF2B689B047FF540AF2D4812F06C
:10C9B00007FF402012F004FF38E72B4812F000FF79
:10C9C0002B682DE7294812F0FBFE2B6825E79A8A91
:10C9D000B2F57A7FBFF415AF4FF47A729A8210E7FE
:10C9E00043F008032B6015E740060008900100089B
:10C9F00080580020B8720408E46804088CA700205E
:10CA000098A70020044D0020664D0020004D002016
:10CA1000D05900209C4E002009600002C4840020F0
:10CA2000B0200020483F00202C1D0020E4200020E2
:10CA30002CA7002012540020EC200020AC910020F4
:10CA400030260020C0C9FB483424002017B7D13855
:10CA50003426002098A100203661023D74A10020F8
:10CA60000160000209400002092000020860000283
:10CA7000024000080080000808B519F005FC12F01B
:10CA8000DDFE19F0E9FBFFF753FE0120BDE8084089
:10CA900011F084BA38B50C4C0C4DAC4206D261682A
:10CAA0002046143412F056FEAC42F8D3084A094B23
:10CAB000094C1460002209491A705A70084808602D
:10CAC000BDE838401DF042B990010008400600085A
:10CAD000004D00208CA70020664D0020044D002052
:10CAE00098A7002008B5FFF7D5FF19F0CDFB12F08D
:10CAF000A5FEBDE8084019F0AFBB00BFF0B50C299A
:10CB000034D8DFE801F0893333335E3333333433E1
:10CB100033330700048C9689B2F802E01788734D0E
:10CB200024F480542404240C0484038C8488818B92
:10CB300023F4005321F4E6411B0409041B0C46EACC
:10CB40000E06090C43EA063341EA0721A8429BB2CC
:10CB5000A4B289B200F09E8005F58065A84200F07D
:10CB6000998092688480818302640384F0BD048C80
:10CB70009589B2F802C0B2F800E05C4F24F48074EA
:10CB80002404240C0484038C8688818B23F4007392
:10CB90001B0421F073011B0C45EA0C04090443EA51
:10CBA0000423090CB8429BB2B6B241EA0E015CD034
:10CBB0004F4CA04259D0926886808183C26303841F
:10CBC000F0BD048C9589B2F802C0B2F800E0474E7F
:10CBD00024F010042404240C0484038C8788018B23
:10CBE00023F0200321F4E6411B0409041B0C45EA51
:10CBF0000C04090C43EA041341EA0E21B0429BB233
:10CC0000BFB289B25DD03A4CA0425AD092688780B8
:10CC1000018382630384F0BD048C9789B2F802E03B
:10CC20001688324D24F001042404240C0484038C5F
:10CC30008488018B23F002031B0421F073011B0C79
:10CC400047EA0E0709043B43090CA8429BB2A4B271
:10CC500041EA060125D005F58065A84221D09268F9
:10CC60008480018342630384F0BDD589148A578A86
:10CC700023F4006343EA05254FF6FF332B409588E4
:10CC800026F440563C4343EA052346EA04169BB289
:10CC9000B6B290E7158A24F4804444EA8514A4B21D
:10CCA0005FE7D689158A578A23F00803334324F4B3
:10CCB000407496883D4323F004032C433343A4B2CD
:10CCC000CDE7D489158A568A23F0800343EA0413FA
:10CCD0004FF6BF741C40938827F44067354344EAFD
:10CCE000031347EA85079BB2BFB28FE700000140FC
:10CCF000000401402DE9F04FC822002183B08A488A
:10CD00008A4CDFF84C928A4D8A4E8B4FDFF8448272
:10CD100037F09BFB89488A49DFF83CE2DFF83CC2E8
:10CD200000221359834200F0D480B3F1804F00F009
:10CD3000E480AB4200F0E380B34200F0E280BB420B
:10CD400000F0E180734500F0E080634500F0DF8093
:10CD5000434500F0DE80DFF808A2534500F0DB8099
:10CD60000AF5806A534500F0D8800AF5806A534579
:10CD700000F0D580AAF5983A534500F0D2800AF524
:10CD8000806A53457BD00AF5806A534508BF0D235E
:10CD900076D01832902AC4D1644C6A4E6A4F6B4DDB
:10CDA00004F1900802E01834A04565D0A379002B67
:10CDB000F9D023794FEA131909F1FF39B9F1030FBB
:10CDC00003F00F03EFD836F8190040FA03F2D20748
:10CDD000E9D54FF0010A0AFA03F3013B184035F098
:10CDE000C5FF17F80930184415EBC002DBD055F821
:10CDF0003000DFF870E1217A00F13F4303F57E0354
:10CE00009B0A1EF8033003F01F0E5B09032B0AFA7E
:10CE10000EFA60D0042B67D0022B51D09388009378
:10CE2000B3FA83F3C3F11F039BB2DA0800EB82026B
:10CE300003F00703D2F820E09B004FF00F0C0CFA30
:10CE400003FC2EEA0C0EC2F820E0D2F820E001FA32
:10CE500003F343EA0E0313626946002302221834E7
:10CE60008DF804208DF805308DF806308DF80730E8
:10CE700025F00CFBA04599D103B0BDE8F08F0C2341
:10CE800009EBC3034FF0010A1B7903F01F0B5B0989
:10CE9000032B0AFA0BFA0ED0042B07D0022B7FF4D7
:10CEA00078AF4B6C4AEA03034B6472E70B6B4AEAB8
:10CEB00003030B636DE70B6C4AEA03030B6468E73B
:10CEC000DFF87CE0DEF844304AEA0303CEF8443071
:10CED000A4E70023D4E7DFF868E0DEF840304AEA50
:10CEE0000303CEF8403099E7DFF854E0DEF8303045
:10CEF0004AEA0303CEF8303090E70123C0E702236B
:10CF0000BEE70323BCE70423BAE70523B8E70623FB
:10CF1000B6E70723B4E70823B2E70923B0E70A23FB
:10CF2000AEE70B23ACE700BFDC7D00202C700408CB
:10CF30000004004000080040000C004000000140D8
:10CF400000380240C0700408BC7004084C7B00200C
:10CF5000646F040800040140001000400014004009
:10CF600000400140DC6F040800286AD003682DE906
:10CF7000F04F03F13F4404F57E045F4EA40A0125FF
:10CF8000345D04F01F066409032C05FA06F559D038
:10CF9000042C00F0AC80022C59D08588B5FA85F0BD
:10CFA000C0F11F0080B2C40803EB840400F0070046
:10CFB000266A80000F27874026EA07062662276A2E
:10CFC00001F003068240701E3A430128C1F3810C30
:10CFD000C1F300182262C1F341113DD90024224659
:10CFE00001274FF0030E03E0102A04F1020426D0BB
:10CFF00007FA02F0A84302F10102F5D1D3F800C00C
:10D000000EFA04F0C04300EA0C0CC3F800C0D3F8D9
:10D01000008006FA04FC4CEA080CC3F800C0D3F800
:10D020000CC000EA0C00D860D3F80CC001FA04F080
:10D0300040EA0C00102AD86004F10204D8D1BDE8FF
:10D04000F08F70472D4C266C35432564A5E72B4C9B
:10D05000666C35436564A0E7002002464FF0010E80
:10D060004FF0030904E00132102A00F102003CD025
:10D070000EFA02F737EA0504F5D1D3F800A009FA51
:10D0800000F4E4430AEA040AC3F800A0D3F800B0AD
:10D0900006FA00FA4AEA0B0AC3F800A0D3F808A07F
:10D0A00004EA0A0AC3F808A0D3F808B00CFA00FA98
:10D0B0004AEA0B0AC3F808A0D3F804A02AEA070733
:10D0C0005F60D3F804A008FA02F747EA0A075F6036
:10D0D000DF683C40DC60DF6801FA00F401323C4369
:10D0E000102ADC6000F10200C2D1BDE8F08F034CD1
:10D0F000266B3543256350E7DC6F04080038024097
:10D1000003682DE9F04F03F13F4404F57E04604EBF
:10D11000A40A0125345D04F01F066409032C05FAF6
:10D1200006F500F0AF80042C00F0A780022C54D04C
:10D130008588B5FA85F0C0F11F0080B2C40803EB02
:10D14000840400F00700266A80000F27874026EA43
:10D1500007062662276A01F0030602FA00F0721E33
:10D160003843012AC1F3810CC1F300182062C1F3D6
:10D17000411137D90024224601274FF0030E03E066
:10D18000102A04F1020426D007FA02F0A84302F1A3
:10D190000102F5D1D3F800C00EFA04F0C04300EA52
:10D1A0000C0CC3F800C0D3F8008006FA04FC4CEA6B
:10D1B000080CC3F800C0D3F80CC000EA0C00D8601B
:10D1C000D3F80CC001FA04F040EA0C00102AD86031
:10D1D00004F10204D8D1BDE8F08F2E4C666C3543C3
:10D1E0006564A5E7002002464FF0010E4FF00309E9
:10D1F00004E00132102A00F102003CD00EFA02F7DE
:10D2000037EA0504F5D1D3F800A009FA00F4E443A5
:10D210000AEA040AC3F800A0D3F800B006FA00FA3C
:10D220004AEA0B0AC3F800A0D3F808A004EA0A0AE5
:10D23000C3F808A0D3F808B00CFA00FA4AEA0B0ABF
:10D24000C3F808A0D3F804A02AEA07075F60D3F860
:10D2500004A008FA02F747EA0A075F60DF683C406B
:10D26000DC60DF6801FA00F401323C43102ADC6024
:10D2700000F10200C2D1BDE8F08F064C266B3543A9
:10D28000256355E7034C266C3543256450E700BF02
:10D29000DC6F04080038024010B50409013C032C7F
:10D2A00017D80D4B33F8142000F00F0042FA00F3AA
:10D2B00013F001030DD0012303FA00F001381040F0
:10D2C00035F054FD054A064B125D104403EBC000D7
:10D2D00010BD002010BD00BFC0700408BC70040861
:10D2E0004C7B002001490248FEF7E8BE7C7E00200E
:10D2F0000004014001490248FEF7E0BE7C7E0020A8
:10D300000004014001490248FEF7D8BE547E0020C7
:10D31000000C004001490248FEF7D0BE2C7E0020E0
:10D320000004004002494FF08040FEF7C7BE00BF36
:10D33000047E002001490248FEF7C0BEDC7D0020CB
:10D340000000014001490248FEF7B8BEDC7D002024
:10D3500000000140F0B50468474DA30AAB426ED00F
:10D3600009D8B3F5801F66D0023DAB4258D14FF0CB
:10D37000700E022608E0414DAB4264D00135AB424D
:10D380004FD14FF0C00E04264779B0004FEA970CFA
:10D3900000295CD063460227A5899F4083190CEBC6
:10D3A00043032F4303F1040C354DBFB245F823105E
:10D3B00045F82C20A781EFF31181502282F31288C7
:10D3C000821905EBC202136963B313620433821935
:10D3D00005EBC202576917B11F6053690433821904
:10D3E00005EBC202976917B11F6093690433821974
:10D3F00005EBC202D76917B11F60D3690433002758
:10D40000CAB21F6082F31188304405EBC000036A82
:10D410005BB9A38923F001031B041B0CA381F0BD9E
:10D42000F0BDF0BD05EB0E03D1E7A3899BB243F03D
:10D430000103A381F0BD4FF0480E0126A4E74FF091
:10D44000980E0326A0E74FF0200E00269CE702234B
:10D45000BF0803FA07F7A389094D9BB223EA070324
:10D4600087190CEB470CA3810CF1040345F82C1031
:10D4700045F823209FE700BF030010004000100084
:10D48000DC7D002010B5036882480139834282B0F8
:10D4900089B200F0CA80A0F58060834200F0C580A8
:10D4A00000F58040834200F0B78000F58060834241
:10D4B00000F0B28000F58060834200F0AD80764CD1
:10D4C000188824686408B4FBF2F4013CA4B282B268
:10D4D000B3F1804F0AD07148834207D000F58060D5
:10D4E000834203D000F58060834202D122F07002B3
:10D4F00092B26B48834200F0A18000F580608342C5
:10D5000000F0A68022F4407200F56C4092B2834293
:10D510001A80D9621C854FD05E4A93424CD00122BA
:10D520009A821A8892B242F001021A80B3F1804FB7
:10D5300000F09880594A934200F0968002F580628C
:10D54000934200F0938002F58062934200F0908055
:10D5500002F58062934200F08D8002F58062934272
:10D5600000F08A8002F57042934200F0878002F555
:10D570007052934200F0848002F58062934200F082
:10D58000818002F5806293427ED0A2F59832934268
:10D590007CD002F5806293427AD002F58062934299
:10D5A00008BF0D2215D002A84FF0012340F8043D1A
:10D5B00024F0DCFC02B010BD0122002119869A8201
:10D5C0001A88384892B242F0010283421A80ADD1E3
:10D5D0000A46354B03EBC20301A85C798DF8044081
:10D5E000012300228DF805308DF807308DF80620D4
:10D5F00024F0BCFC1B2C08D02E2CDBD12B4B019330
:10D6000001A824F0B3FC02B010BD294B019301A87E
:10D6100024F0ACFC02B010BD1F4C18882468B4FB89
:10D62000F2F4013CA4B282B252E71B4C1888246881
:10D63000B4FBF2F4013CA4B282B257E701201A8095
:10D64000D9621C8598821A8892B202431A8071E7C7
:10D6500001201A80D9621C8598821A8892B20243EE
:10D660001A8063E70122B4E70222B2E70322B0E79F
:10D670000422AEE70522ACE70622AAE70722A8E7C4
:10D680000822A6E70922A4E70A22A2E70B22A0E7C4
:10D690000C229EE700040140CC85002000040040DD
:10D6A0000010004000000140646F04082C010001DC
:10D6B000190100012B4B98423CD0B0F1804F3BD078
:10D6C000A3F57C43984239D003F58063984237D064
:10D6D00003F58063984235D003F58063984233D0D8
:10D6E00003F58063984231D003F5704398422FD000
:10D6F00003F5705398422DD003F5806398422BD0E8
:10D7000003F58063984229D0A3F59833984227D037
:10D7100003F58063984207D003F58063984208BF01
:10D720000D2202D0002070470C220F4B03EBC203E6
:10D73000187970470022F8E70122F6E70222F4E7A1
:10D740000322F2E70422F0E70522EEE70622ECE7E7
:10D750000722EAE70822E8E70922E6E70A22E4E7E7
:10D760000B22E2E700000140646F04082DE9F04F4E
:10D77000013085B0C3B203930B4602918B4C8C4EA3
:10D78000002B00F09A8032208A4D8B4FDFF82C92CC
:10D7900028F036F94FF4FA7A4FF0100C4FF47A7003
:10D7A000D9F80430C3F30803002B40F0DE80EFF318
:10D7B0001183002B40F0D9802968A26800BF2B6834
:10D7C0009942F9D1D7F800E000FB0EF39B1AB3FBA6
:10D7D000FEF300FB01314FF0010E0191D9F8043046
:10D7E000C3F30803002B40F08780EFF31183002B75
:10D7F00040F082802B68A16800BF2A689342F9D16B
:10D80000D7F800B000FB0BF2521AB2FBFBF200FBA0
:10D810000323019A9B1AB3F57A7FDFD3BAF1010A89
:10D82000BED1039B002B40F0BD804FF47A7ADFF825
:10D830008C9150464FF0100CD9F80430C3F3080314
:10D84000002B75D1EFF31183002B71D12968A268E9
:10D8500000BF2B689942F9D1D7F800E000FB0EF326
:10D860009B1AB3FBFEF300FB01314FF0010E019157
:10D87000D9F80430C3F3080313BBEFF31183FBB9EA
:10D880002B68A16800BF2A689342F9D1D7F800B08D
:10D8900000FB0BF2521AB2FBFBF200FB0323019ACE
:10D8A0009B1AB3F57A7FE3D3BAF1010AC4D1029B84
:10D8B000013B0293002B7FF466AF05B0BDE8F08F0B
:10D8C000EFF311888CF31288A1682368DB0344BF4F
:10D8D000C6F800E0A1682B6832685FFA88F888F320
:10D8E0001188D7F800801A4400FB08F35B1AB3FBD9
:10D8F000F8F300FB0233D2E7EFF311888CF31288C0
:10D90000A1682368DB0344BFC6F800E0A1682B6868
:10D9100032685FFA88F888F31188D7F800801A44D3
:10D9200000FB08F35B1AB3FBF8F300FB023370E76C
:10D93000EFF311828CF31288D4F808E02368D9033E
:10D9400003D501233360D4F808E02B683168D2B2E4
:10D9500082F311883A68194400FB02F3A3EB0E032B
:10D96000B3FBF2F300FB01317FE7EFF311828CF39D
:10D970001288D4F808E02368D90303D50123336063
:10D98000D4F808E02B683168D2B282F311883A6883
:10D99000194400FB02F3A3EB0E03B3FBF2F300FB0D
:10D9A000013118E7184627F08DFE3EE710E000E051
:10D9B000087D00200C7D0020107D002000ED00E09F
:10D9C000204B5B68C3F3080330B4BBB9EFF311839A
:10D9D000A3B91D4B1D4C1868A16800BF1A6890427E
:10D9E000F9D11B4B1C684FF47A7202FB04F3591AED
:10D9F000B1FBF4F130BC02FB00107047EFF3118271
:10DA0000102383F3128811498C680B6813F4803F4C
:10DA1000104B02D0012018608C680B49D2B20D68FF
:10DA2000186882F311880A4B19684FF47A722844F7
:10DA300002FB01F31B1B30BCB3FBF1F302FB003014
:10DA4000704700BF00ED00E00C7D002010E000E01A
:10DA5000107D0020087D00202DE9F84F8046FFF75B
:10DA6000AFFF254E2549DFF8A0E0254A254D844625
:10DA700010274FF47A740120DEF80430C3F3080352
:10DA8000D3B9EFF31183BBB90B68D2F808A000BF7C
:10DA9000D1F800904B45F7D1D6F800B004FB0BF954
:10DAA000A9EB0A09B9FBFBF904FB0393A3EB0C03F5
:10DAB0004345E1D3BDE8F88FEFF3118A87F312886D
:10DAC000D2F808B01368DB0344BF2860D2F808B06E
:10DAD0000B68D5F800905FFA8AFA8AF31188D6F8B5
:10DAE00000A0994404FB0AF3A3EB0B03B3FBFAF386
:10DAF00004FB0933DAE700BF107D00200C7D002015
:10DB000010E000E0087D002000ED00E02DE9F04F7E
:10DB1000DFF830C1474A4849484E494D80461027F2
:10DB200018F1FF38C0F08480DCF80430C3F3080338
:10DB3000002B5CD1EFF31183002B58D10B68946854
:10DB400000BF08688342F9D1D6F800904FF47A708C
:10DB500000FB09FEAEEB040EBEFBF9FE00FB03EE7C
:10DB6000DCF80430C3F308034FF47A740120FBB9E6
:10DB7000EFF31183E3B90B68D2F808A000BFD1F826
:10DB800000904B45F7D1D6F800B004FB0BF9A9EB98
:10DB90000A09B9FBFBF904FB0393A3EB0E03B3F5EE
:10DBA0007A7FBDD2DCF80430C3F30803002BDFD04A
:10DBB000EFF3118A87F31288D2F808B01368DB03F9
:10DBC00044BF2860D2F808B00B68D5F800905FFA1F
:10DBD0008AFA8AF31188D6F800A0994404FB0AF364
:10DBE000A3EB0B03B3FBFAF304FB0933D5E7EFF325
:10DBF000118487F31288D2F808901368D80303D5EC
:10DC000001232B60D2F808900B682868E4B284F3F3
:10DC10001188D6F800A04FF47A7400EB030E04FBD1
:10DC20000AF3A3EB0903B3FBFAF304FB0E3E97E7F9
:10DC3000BDE8F08F10E000E00C7D0020107D00209A
:10DC4000087D002000ED00E030B4EFF311831022D6
:10DC500082F312880649074C0A68074801320025FA
:10DC60000A602560DBB2026883F3118830BC70471C
:10DC70000C7D0020087D002010E000E038B5264B28
:10DC80005C69636B73B1A36DA26BD2B1998A1A8878
:10DC9000C90592B201D5D20700D438BD4FF6F7724C
:10DCA0001A8038BDA36D99891A88890692B2EBD57E
:10DCB0009206E9D5E26AD2B19888216B80B290478A
:10DCC000E1E799891A880D0692B2DFD51006DDD5F5
:10DCD000A26A616A8A4219D0A1692569885C988024
:10DCE0000132B2FBF5F105FB1122A262CEE79B885F
:10DCF000E2696169DBB28B54E269E068A36D0132CD
:10DD0000B2FBF0F100FB1122E261BDE7DA6822F01C
:10DD10008002DA60BAE700BF5035002038B5264BE4
:10DD20009C68636B73B1A36DA26BD2B1998A1A8898
:10DD3000C90592B201D5D20700D438BD4FF6F772AB
:10DD40001A8038BDA36D99891A88890692B2EBD5DD
:10DD50009206E9D5E26AD2B19888216B80B29047E9
:10DD6000E1E799891A880D0692B2DFD51006DDD554
:10DD7000A26A616A8A4219D0A1692569885C988083
:10DD80000132B2FBF5F105FB1122A262CEE79B88BE
:10DD9000E2696169DBB28B54E269E068A36D01322C
:10DDA000B2FBF0F100FB1122E261BDE7DA6822F07C
:10DDB0008002DA60BAE700BF5035002038B5264B44
:10DDC0001C68636B73B1A36DA26BD2B1998A1A8878
:10DDD000C90592B201D5D20700D438BD4FF6F7720B
:10DDE0001A8038BDA36D99891A88890692B2EBD53D
:10DDF0009206E9D5E26AD2B19888216B80B2904749
:10DE0000E1E799891A880D0692B2DFD51006DDD5B3
:10DE1000A26A616A8A4219D0A1692569885C9880E2
:10DE20000132B2FBF5F105FB1122A262CEE79B881D
:10DE3000E2696169DBB28B54E269E068A36D01328B
:10DE4000B2FBF0F100FB1122E261BDE7DA6822F0DB
:10DE50008002DA60BAE700BF5035002070B4EFF3FB
:10DE60001186502383F31288836B1A68D20720D45B
:10DE70005D686DB9446A826A944217D08169114421
:10DE8000D9600ED9A21A5A608462002280F85C2000
:10DE90001A6842F00102F1B21A6081F3118870BC75
:10DEA000704701698A1A5A608562EEE7012380F89B
:10DEB0005C30F3B283F3118870BC704703685B6A0F
:10DEC00003B11847704700BF03681B6A03B11847C6
:10DED000704700BF03682DE9F041DF691FB13B4681
:10DEE000BDE8F0411847002A164611DD04460D46EC
:10DEF0000E4400E023689B68204698470028F9D02C
:10DF0000236815F8011B1B6820469847AE42F1D1E3
:10DF1000BDE8F08103689B69184700BF03685B692F
:10DF2000184700BF03681B69184700BF0368DB6818
:10DF3000184700BF03689B68184700BF03685B6809
:10DF4000184700BF03681B68184700BF38B50C4668
:10DF5000097849B1054601342B6828461B68984763
:10DF600014F8011B0029F7D138BD00BF064B53F848
:10DF700020302BB11A689B8851690B4201D1138361
:10DF800070475383704700BFD87C0020026802F1BD
:10DF90003F4303F57E032DE9F04F9B0A544DEB5CA4
:10DFA00003F01F055B090124032B04FA05F400F0BC
:10DFB0009980042B00F09180022B3ED001F00306E3
:10DFC000731E012BC1F3810CC1F300188588C1F3C6
:10DFD000411137D90024234601274FF0030E03E0F7
:10DFE000102B04F1020426D007FA03F0A84303F132
:10DFF0000103F5D1D2F800C00EFA04F0C04300EAE4
:10E000000C0CC2F800C0D2F8008006FA04FC4CEAFE
:10E01000080CC2F800C0D2F80CC000EA0C00D060B6
:10E02000D2F80CC001FA04F040EA0C00102BD060CA
:10E0300004F10204D8D1BDE8F08F2E4B5D6C2C4367
:10E040005C64BBE7002003464FF0010E4FF003096C
:10E0500004E00133102B00F102003CD00EFA03F76C
:10E0600037EA0504F5D1D2F800A009FA00F4E44338
:10E070000AEA040AC2F800A0D2F800B006FA00FAD0
:10E080004AEA0B0AC2F800A0D2F808A004EA0A0A79
:10E09000C2F808A0D2F808B00CFA00FA4AEA0B0A53
:10E0A000C2F808A0D2F804A02AEA07075760D2F8FD
:10E0B00004A008FA03F747EA0A075760D7683C400C
:10E0C000D460D76801FA00F401333C43102BD460CC
:10E0D00000F10200C2D1BDE8F08F064B1D6B2C434E
:10E0E0001C636BE7034B1D6C2C431C6466E700BF8D
:10E0F000DC6F0408003802402DE9F04F4A484B49D4
:10E100004B4B4C4C4FF0010A4FF002094FF0040802
:10E110004FF0080C4FF0100E20274026802530F8D5
:10E12000022B12F0010F03D01960A3F804A00833EA
:10E1300012F0020F03D01960A3F80490083312F014
:10E14000040F03D01960A3F80480083312F0080FFD
:10E1500003D01960A3F804C0083312F0100F03D0E5
:10E160001960A3F804E0083312F0200F02D0196000
:10E170009F80083312F0400F02D019609E80083350
:10E1800012F0800F02D019609D80083312F4807F56
:10E1900005D04FF4807B1960A3F804B0083312F463
:10E1A000007F05D04FF4007B1960A3F804B008335A
:10E1B00012F4806F05D04FF4806B1960A3F804B09F
:10E1C000083312F4006F05D04FF4006B1960A3F808
:10E1D00004B0083312F4805F05D04FF4805B1960FF
:10E1E000A3F804B0083312F4005F05D04FF4005BCD
:10E1F0001960A3F804B0083312F4804F05D04FF42F
:10E20000804B1960A3F804B00833D20B04D04FF44C
:10E21000004219609A80083301F58061A1427FF4C1
:10E220007EAFBDE8F08F00BFC07004080000024060
:10E230004C7B002000100240002855D0026802F1FB
:10E240003F4303F57E032DE9F04F9B0A544DEB5CF1
:10E2500003F01F055B090124032B04FA05F444D0E5
:10E26000042B00F09780022B44D001F00306731EAC
:10E27000012BC1F3810CC1F300188588C1F3411152
:10E280003DD90024234601274FF0030E03E0102B55
:10E2900004F1020426D007FA03F0A84303F10103B6
:10E2A000F5D1D2F800C00EFA04F0C04300EA0C0C1D
:10E2B000C2F800C0D2F8008006FA04FC4CEA080C50
:10E2C000C2F800C0D2F80CC000EA0C00D060D2F84E
:10E2D0000CC001FA04F040EA0C00102BD06004F1ED
:10E2E0000204D8D1BDE8F08F70472E4B1D6C2C4333
:10E2F0001C64BAE72B4B5D6C2C435C64B5E70020D3
:10E3000003464FF0010E4FF0030904E00133102BD8
:10E3100000F102003CD00EFA03F737EA0504F5D10C
:10E32000D2F800A009FA00F4E4430AEA040AC2F8A9
:10E3300000A0D2F800B006FA00FA4AEA0B0AC2F8C6
:10E3400000A0D2F808A004EA0A0AC2F808A0D2F88D
:10E3500008B00CFA00FA4AEA0B0AC2F808A0D2F890
:10E3600004A02AEA07075760D2F804A008FA03F7C6
:10E3700047EA0A075760D7683C40D460D76801FA7B
:10E3800000F401333C43102BD46000F10200C2D1F1
:10E39000BDE8F08F034B1D6B2C431C6365E700BF8A
:10E3A000DC6F04080038024010B1036882885A8389
:10E3B000704700BF10B1036882881A83704700BF9E
:10E3C00018B10368828809B95A8370471A83704765
:10E3D0000E4B1B8801463BB90D4B0E4A1B7810684B
:10E3E0000BB981F00101EBE70B4B5A691AB118B96F
:10E3F0001A68106058747047084A18681188084AEB
:10E4000092FBF1F20121026059747047E47C002014
:10E41000E67C0020E87C0020EC7C0020047D0020CD
:10E4200020A1070010B40A4B0A4A1C78012383403C
:10E43000234052F8200029B9B3FA83F149095DF865
:10E44000044BBDE7191C18BF01215DF8044BB7E769
:10E45000D47C0020D87C002030B1036882881B69FE
:10E460001A4214BF01200020704700BF2DE9F0417F
:10E470000B4E346873691C400FD0DFF828800127E9
:10E48000B4FA84F3C3F11F0307FA03F558F8230025
:10E4900003689847AC437561F2D1BDE8F08100BFD5
:10E4A000003C0140147D00202DE9F0410B4E346802
:10E4B00073691C400FD0DFF828800127B4FA84F379
:10E4C000C3F11F0307FA03F558F8230003689847C0
:10E4D000AC437561F2D1BDE8F08100BF003C014062
:10E4E000147D002038B50B4C23688BB15A68821A12
:10E4F000002A054604DA0CE05A68AA1A002A07DB4B
:10E500009A68226018461A6890472368002BF3D156
:10E5100038BD38BDE43E00202DE9F047C44B1C68EF
:10E5200062072DED028B03D4BDEC028BBDE8F087B2
:10E53000C04D2B78002BF7D06E6846F2A713861BD0
:10E540009E42F1D9DFF850936860B9F80070DFF8A7
:10E550004C83002F40F0A68198F80620AB689FED11
:10E56000B60ADFEDB60ADFF8F492013AB3FBF2F334
:10E5700007EE903AF8EE677AB7EE008A27EE800A47
:10E5800035F06EF8DFEDAE7A38EE400A20EE270A5D
:10E5900034F09EFFB8F80830DFEDAA6A07EE103AB3
:10E5A000EB68C01AB8EEC77A07EE900AA7EE668A43
:10E5B000B8EEE70AD9ED097AF8EEE77A20EE080A14
:10E5C00067EEA67AA7EE270A34F082FF9E4BC9F8C1
:10E5D000240002461860A30740F1AA81DFF8C0E2D8
:10E5E0009A4CDEED007A9FED9A5A2168F8EE677A30
:10E5F00027EE855A002900F0BB81964B07EE101AD2
:10E60000D3ED026AB8EEC77AF8EEE66A86EE878A3C
:10E61000914991ED004AB8F80C10D5ED054ADFEDAF
:10E62000895A95ED066A67EE847A06EE901A67EECF
:10E63000887A8A49B6EE004AF8EEE66AF0EE643A65
:10E64000E7EE843A66EEA56A91ED097A7E49F7EE27
:10E65000005A75EEE65AB8EEC77AA3EE856A77EEF1
:10E66000A47A27EE257AC5ED057AF0EE477AE6EE34
:10E67000267ABDEEE77AC5ED067A81ED007A784913
:10E680000978122900F05B810021196059609960B6
:10E690002160CEF80010002F7FF446AFE869EA61F0
:10E6A000121A07EE102ADFED6F6A6F4B07EE906AC1
:10E6B000B8EEC77AF8EE677A27EE267A40F2DC5297
:10E6C000C7EE276A0A21FDEEE67A17EE900A90421D
:10E6D000A8BF10469842B8BF184611F0D5FDB8F84B
:10E6E0000A309FED586AD5ED056A07EE103AB8EE8C
:10E6F000C77AF7EE007AE7EE467A05EE900AF8EE72
:10E70000E55A66EE866A67EEA57AE7EE267AB0EEFF
:10E71000670AC5ED057A34F0DBFE0521064611F0E7
:10E72000B3FD524A5249B2F90040086084EAE473EA
:10E73000A3EBE473B3F5487F74DAB2F9022082EAFE
:10E74000E273A3EBE273B3F5487F6BDA494B1B78B6
:10E75000002B40F01181484B3B4A1B681268474828
:10E760009B1AB3F5FA7FA8BF4FF4FA739842B8BF6B
:10E7700018460A2111F088FD414B1C68637A00FBA2
:10E7800003F00028B8BF7F30C211B2F5967F3D4B31
:10E79000A8BF4FF496729A42B8BF1A463A48E37E31
:10E7A000076895ED087ADFED396A911B01FB03F3E9
:10E7B000227F344E002B01FB0272B8BF1F335B1166
:10E7C000B2F5C81F3249A8BF4FF4C812B3F5967FFF
:10E7D000A8BF4FF496738A42B8BF0A46617F0260B1
:10E7E00007EE901A37EE087AF8EEE77A27EE267AE7
:10E7F000B34267EE877AB8BF3346002AB8BF02F546
:10E80000FF52FDEEE77AB8BF1F3203EB623317EE1B
:10E81000902A962A6FF09501A8BF96228A42ACBF33
:10E820009F1A5F1A1B4A85ED088A17607CE600BFB5
:10E83000A04C0020181F002008942537B1DC423E70
:10E84000D048874A6F12833AA44C0020ACA1002024
:10E85000BD3786359CA1002028A70020F451002058
:10E86000C84900200024744924FAFFFFAC4C002062
:10E87000A84C00202C260020242600200CFEFFFFA0
:10E88000004D0020D4FEFFFF1C2600200000003BAE
:10E890000000E7FF14260020EEBB002018A1002096
:10E8A000A8A10020374998F806A00A68AB689FED38
:10E8B000360ADFED360A002A0AF1FF3AB3FBFAF313
:10E8C0009246B8BF02F1070AA2EBEA0203EB020A82
:10E8D000BAF1000F5346B8BF0AF10703DB1007EE89
:10E8E000903AF8EEE77AC1F800A027EE800A34F0FB
:10E8F000B7FEF7EE007A77EEC07A9FED257A2B69A6
:10E9000067EE877A9A4518BF07F1FF33FDEEE77A85
:10E9100014BF9FB200274FF00003C5ED037A18BF64
:10E92000C5F810A0A9F800706B61AB61002252E637
:10E930009FED188ADFF870E0174C184B9FE695EDB5
:10E94000057AD5ED067ADFF864C02068996891FBF6
:10E95000F0F1BDEEC77AFDEEE77A17EE100A17EE7A
:10E96000909AACF80200ACF80010ACF804908BE67A
:10E970009FED088A094B4BE6094A0A4B12681C684E
:10E980000CE700BF1C00002008942537B1DC423E94
:10E99000D048874A00000000ACA100209CA10020C4
:10E9A00028260020004D0020A8A10020CC490020EE
:10E9B0002DE9F843304B1B685B0701D4BDE8F883B1
:10E9C0002E4C2F4D94F82490B9F1010F48D1EB69EA
:10E9D000284698472B69284698472B6A04F12C0053
:10E9E00004F128019847274B276B9B79A668E06ABA
:10E9F00007F101089845636B08BF84F8009003F1A4
:10EA0000010208BF4FF00008032A1FD01E496263AD
:10EA100094F8382041F82300FAB904EB870704EB97
:10EA20008803F863DA6BAB89C4F83080B61A3044D7
:10EA30000022A06084F82420002BBFD0134A0A2BA8
:10EA40001268B8BF0A231361BDE8F8830E4B012298
:10EA50009860002384F83820636326F0CFF9DCE760
:10EA60006B6928469847AB69284698470122EB898D
:10EA700084F82420E0E700BFA04C0020181F0020ED
:10EA8000F451002018A100207C5D002028A1002066
:10EA90002DE9F04F2DED028BB84BB94A1C7897B099
:10EAA00000F59C412031814609911160002C00F055
:10EAB0000085B44A1268904240F2E680B24A089259
:10EAC0001668B249B24ADFF80CA30791013C0492E0
:10EAD0001C7006F48056002E40F0E480AD4B1B788D
:10EAE000022B00F0F486042B00F05F87012B00F06E
:10EAF0001387A94B99459AF8023000F2B083002B96
:10EB000040F0B183A54B0993089B1E6816F480570B
:10EB100040F06B84DFF8C092049BB3F90620079B9A
:10EB20005C8BA242B4BF002401249D4B1B68D9001A
:10EB300040F1C280099B1B7813F0010300F0C380F1
:10EB40000799498C914240F3ED87002C40F0C28038
:10EB5000944D95F88821002A40F0BC80924A934950
:10EB6000106890F82D0000220A604A608A60904A7E
:10EB7000002840F0B0801070002B40F0B1808D4B29
:10EB80001A78002A40F0E1800799049D488BB5F976
:10EB90000070898BB5F902508742CCBF80260026D1
:10EBA00046F040038F42A8BF33469B0843F08006DF
:10EBB0008542C8BF3346049F43F040068D42B8BF2C
:10EBC00033469B08B7F90450B7F9066043F0800755
:10EBD0008542C8BF3B4643F040078D42B8BF3B4625
:10EBE0009B0843F080076F4D8642C8BF3B4643F009
:10EBF000400795F88AE18E42B8BF3B469E4501F03A
:10EC0000BE81A5F88C2185F88E216B4985F88A3163
:10EC10000E78002E01F0CE805F2B01F046816F2B25
:10EC200001F07581099B1B78DB0700F18E8095F858
:10EC30008E11002940F08980B5F98C31322B40F3D8
:10EC4000848095F88A210120572A85F88E0101F0E9
:10EC50008C84089B1B685C0740F1EE875A2A40F0C1
:10EC6000EB8795F89031002B41F0458695F892316D
:10EC700083F0010385F89231002B41F063860C206C
:10EC80000FF066F801F025B93F4B08931E683F4A24
:10EC90003F4B079206F480560493DFF838A1002E0C
:10ECA0003FF41CAF00213E4811F0BFFD00287FF467
:10ECB00015AF19F00FF911E773023FF53BAF099B50
:10ECC0001B7803F00103374D002285F88821002CC2
:10ECD0003FF444AF364A01211170002B3FF44FAF8F
:10ECE000F6067FF54CAF354B1B78DD063FF547AF99
:10ECF000002F7FF444AF2DF08DFC00287FF43FAF50
:10ED00002D4B1B78002B01F0FF852D4B9B78002CA1
:10ED100041F02A863BB12B4A2B4B12681B689B1A89
:10ED2000002BC1F2128610201E4D0FF011F80123A6
:10ED300085F8893123E70F200FF00AF8B5F88C31F8
:10ED400085F88E41FA3BA5F88C31089B1F4A1B6859
:10ED500006921F4C5F0700F192840DF1500BDFF813
:10ED60007C800A940023CBF804304546149319277D
:10ED700040F6330340F28336049C34E0E03E00204A
:10ED8000583D0020DC3E0020D08D002098840020DB
:10ED9000DCB900202E3E0020404B4C00D054002017
:10EDA000D0530020181F0020004D0020DC5100200F
:10EDB000CC2500205B4900202C1D0020FE4C0020AB
:10EDC0002C5400200C7D0020A4450020A04C0020E5
:10EDD000FC4C0020AC910020983F0020483F0020D0
:10EDE00004354D4524D0A878E978884217FB006E99
:10EDF000F6D295F801C00CF1040C17FB016034F950
:10EE00001C109942A8BF1946B1F5617FB8BF4FF4F5
:10EE100061718E45E4DA8842E2DB29782729DFD860
:10EE200058460435059311F0F1FC4D45059BDAD1A8
:10EE3000B54BB64A1B780A9C9BE8030082E80300A6
:10EE4000002B40F00581B24B1F78002F00F0738338
:10EE50000121AE4811F0E9FC002840F019819AF830
:10EE60000330002B40F01481228822F001039BB272
:10EE70009A42238009D0A74B02251421FF220E209D
:10EE80001D7059709A700EF063FF02219F4811F0B7
:10EE9000CCFC002800F0188401200DF021FD23880F
:10EEA0009E0740F1C386DFF884A2DFF884B29AF8A7
:10EEB0000010DBF804009D0708BF81F00201C1F3D8
:10EEC0004001FFF77DFA2421904811F0AEFC30B9E3
:10EED000099A1378590744BF23F004031370069B63
:10EEE0001B6813F00A0F1ED00521884811F09DFC05
:10EEF000002800F0FE8523885F0740F17A8706210D
:10EF0000824811F092FC002800F0EE8523885E060E
:10EF100040F15D8707217D4811F087FC002840F013
:10EF20008B85069B1B689D0600F17A8326887748AF
:10EF30000C2111F07AFC002800F0C68046F48073A2
:10EF4000B342238009D0734B02251421FF220E20E7
:10EF50001D7059709A700EF0FBFE6F4B1B78082BDA
:10EF600000F0BE800E2B00F0BB80089B1B685D0587
:10EF700046D56A4B1B79002B6FD01421634811F0E2
:10EF800054FC00286DD12AF0F1FD01200EF0E8FDBF
:10EF9000002835D0DFF89C8100254FF0CC0902E035
:10EFA000DDB2022D2CD809FB05F76B1C58F8076061
:10EFB000002EF5D1032290F9023002960192C27818
:10EFC000574951F822200092184632463346012113
:10EFD0000EF0BCFB034605EB450000EB001005936B
:10EFE00053B1314608EB8000CC2235F02EFA059B58
:10EFF00048F807300135EDB228F0C0FC0028D0D128
:10F00000099B1B78D80740F197809AF80010454A71
:10F01000454DDBF80000012301F0010113702B7056
:10F02000FFF7CEF9069B1B685A0700F1F98017B06D
:10F03000BDEC028BBDE8F08F98F8022098F8033001
:10F040009A42C0F0E88508F10408A8453FF4FBAEF9
:10F0500098F800102329F6D1EEE7099B1B78D90711
:10F0600091D54FF40F7026F0A9F80028C8D00EF003
:10F0700055FB4FF40F7026F043F80028C0D00EF077
:10F080004DFB4FF40F7026F03BF80028EFD1B7E7A7
:10F09000069B1B689B077FF5E7AE2388DF0740F1DF
:10F0A0001F8723F0020292B29A4222803FF4FBAE05
:10F0B000184B1421FF2202250E201D7059709A70E2
:10F0C0000EF046FE2388EEE626F480739BB2B34230
:10F0D00023807FF438AF104B1B78082B7FF442AFAE
:10F0E000228822F040039BB29A4223803FF43DAF36
:10F0F000084B02251421FF220E201D7059709A70B2
:10F100000EF026FE31E700BFF4590020D053002056
:10F1100087A70020183A002080580020B04A00201D
:10F120003871040838260020D1540020D47C0020F7
:10F13000D87C002054780020BE4B1E78002E65D16C
:10F14000BD4B1B68002B61D0DFF84083DFF8409394
:10F1500018F8030C99F804704146A8F103052DF046
:10F160002FFA002800F0F684002F40F0478505F1C3
:10F17000080168792DF024FA002841F03C83AF495A
:10F18000A87A2DF01DFA002800F0F784022F41F034
:10F190002E83AB49E87B2DF013FA002841F023833E
:10F1A000A849287D2DF00CFA002800F0F784042FE0
:10F1B00041F01583A449687E2DF002FA002841F041
:10F1C0000A83A249A87F2DF0FBF9002800F0F784FC
:10F1D000062F41F0FC829E4995F823002DF0F0F9AE
:10F1E000002841F0F0829B4995F828002DF0E8F9BD
:10F1F000002800F0F784082F41F0D682964995F850
:10F200002D002DF0DDF9002840F0F784934B01220A
:10F210001A7032F0E1FE069B1B685A077FF507AFB4
:10F2200003202DF005FA002800F0C186238813F092
:10F2300008047FF4FCAE08200DF06AFB049E8848A9
:10F24000884D8949894A8A4BF68800682E80086073
:10F2500014601C6017B0BDEC028BBDE8F08F13B9D1
:10F2600001238AF80230834B09931B201D789AF8FA
:10F2700021402DF0DDF9012C05F00108814600F058
:10F28000428605F0020305939AF820307A4EDFF8A3
:10F2900004B27A4F052B00F29B80DFE813F08B005D
:10F2A00081000600C900FD00BE00012C04BF05233B
:10F2B0008AF82030B8F1000F12D0079B3088B3F9DC
:10F2C00018100022134661F30F0260F31F4261F32E
:10F2D0000F03049861F31F43036003234260059307
:10F2E000674DDAF814202B689A4280F0288547F29F
:10F2F00030520323CAF81C208AF8203002200DF077
:10F300001FFB18F0E7FD2A68DAF81C3013440422CA
:10F31000CAF818308AF82020012C40F097862B6814
:10F32000DAF818209A4253D29BF8000018B92DF051
:10F330007FF900284CD13B6823F002033B602A6828
:10F340007388642101FB03234FF480600022CAF814
:10F3500010308AF820208AF803200DF0C1FA9AF8BC
:10F36000203097E72DF06AF9012807D1444D7388C2
:10F370002A68642101FB0323CAF81030B9F1000F99
:10F3800002D0B379002B4AD1012C21D03C4DDAF8C0
:10F3900010202B689A42C0F04E8601238AF8203054
:10F3A000012C3AD0F379012B78D02DF0C7F89AF8D8
:10F3B00020306FE7B8F1000FD4D14FF48060B9F17D
:10F3C000000F00F0FF820DF0A3FA0023CAF81030FE
:10F3D000059B002B3FF498AB18460EF0B9FC089B38
:10F3E0001E6816F480573FF495AB1D21254811F097
:10F3F0001CFA00287FF48EAB234B03F1500903E085
:10F400000433994500F0D8851A78262AF8D19978DE
:10F41000DA789142F4D2FFF77FBB194D8FE72DF0D8
:10F420008DF803224FF47A738AF82020CAF81C3032
:10F43000134D63E7D1540020D4540020E839002054
:10F44000ED390020F2390020F7390020FC39002086
:10F45000013A0020063A00200B3A0020382600200E
:10F46000A44C002018260020242600201C26002062
:10F4700014260020D05400202CA70020F84C002097
:10F480000C7D0020D0530020483F0020DE390020B2
:10F490001C0000202C1D00208C4D3DE72DF04EF867
:10F4A000032240F6B8338AF82020CAF81C30874D72
:10F4B00024E7874F3B78002B01F0B580854BDFF8C0
:10F4C0004C82DFF84CB2DFF84CA2079345465E460B
:10F4D000049099460EE019F804109847032C28DC94
:10F4E00088B93B782AF8020F01349C4205F10405E3
:10F4F00080F21681072CE1B23046DBF80430EADDF9
:10F50000984700B2EDE738F824206B88801A4FF452
:10F510007A719B1A01FB00F040F6CA0290FBF3F0EF
:10F520000844904240F2EE23A8BF10469842B8BF6C
:10F53000184600B2D5E7DFF8E0B1DFF8E081664DAC
:10F540000BF15A064FF0010959461BF8010C2DF03A
:10F5500037F8F8B19BF804009BF802309BF803E001
:10F5600000EB400105EB8101013BD1F89C2103EB4D
:10F570004303434493420DD095F8C82181F898E1A4
:10F5800009FA00F022EA0000C1F89C31C1F8A0712C
:10F5900085F8C8010BF1060B5E45D5D14F494B4AA2
:10F5A0004F4B504D09681B78D2F800900A91059393
:10F5B000A5F5CC7B00266B6863B31F7857B3AA68A8
:10F5C000A9EB0202002A0ADB9BF8C8210121B14005
:10F5D00022EA010209F5FA718BF8C821A960059A9F
:10F5E000C2B12A7859780432D2B2002940F0A08200
:10F5F00007990498098B30F9122001F1C800824262
:10F6000040F3EB849BF8C8119A7841FA06F3D807C7
:10F6100040F183850136042E05F10C05CBD117E4AA
:10F62000314B1B78980704D5304D2B7D042B00F20D
:10F630001585268816F0300F3FF479AC10200DF0B8
:10F640004FF920200DF04CF9294B268800221A7022
:10F65000284A2948294F2A4D00211160294A39603A
:10F660000023296041608161036083604361C3615D
:10F6700013605160936053619161D36157E4164DFB
:10F6800095F892315BB1099B1B78DE0707D5049B87
:10F69000B3F90620079B5B8B9A4200F3308511215A
:10F6A000194811F0C2F8002800F02B8295F8963125
:10F6B0002BB995F8903113B93223A5F89431012371
:10F6C00085F89631FFF749BB2388EAE40C7D0020DA
:10F6D0001040002098840020181F0020044D0020B6
:10F6E000D9900020B0200020FE4C00208C5D00202E
:10F6F000EC470020D848002088480020A0250020A2
:10F7000094260020B0480020D05300202440002040
:10F71000D4A7002012200020F538002088450408D6
:10F72000DDF81090A94AAA4908921268A1FB091BAA
:10F7300042F2010111404FEA9B1B0F9100F0DE8164
:10F74000A44DA548A54CA6492E78007826700870CF
:10F750001EB1A3490E7886F00106A24D0F2185F84F
:10F760002011002B00F057839F4B079C0E93B4F899
:10F7700024E0B4F826C0079CCDF82CC01846248B92
:10F7800000789A4B12949A4C0D9004940446A3FB73
:10F7900000035B0803EB4303E31ADBB295F8218116
:10F7A0000A9302F4805205F592700BF59673119549
:10F7B00097F800A0DFF878C28D4C0C917546DDF803
:10F7C0003CE01392002106930596CDF84090059BEE
:10F7D000002B00F05782874B33F911301FFA83F961
:10F7E000A9454FEA410203D30B9EB14540F29782EF
:10F7F0005CF821309B4580F04E82A35EBEF1000F85
:10F8000040F06C8201315145A35200F10600DEDB6D
:10F810000C9A119D784B85F820210F2A0CBF0122EC
:10F820000022DDF8409085F821811A7000F0FA82FC
:10F830006948DFF800A26A49704D01220270042075
:10F840000A700DF07DF82B68DAF80810DAF8042059
:10F85000CAF80C305B1A934284BF00238AF8213027
:10F860003C78089B1E68002C00F0E186079A644DE6
:10F87000B2F824E0178B5E4916F48056284640F013
:10F88000F68232460EE0437803EB830303EB8303F7
:10F8900003F2EE239BB20132A24221F8023B00F1B7
:10F8A00002000ED015F81230002B00F03C82022B23
:10F8B000E9D001320B8821F8023BA24200F102009C
:10F8C000F0D10E9A137801331370FFF704B9079A39
:10F8D0000499537DD27D013B31F913301AB1C3F540
:10F8E0003B6308331BB2A3F57A7307EE903A9FEDA2
:10F8F000457A454AF8EEE77A40F2FF3167EE877ABB
:10F90000FCEEE77ACDED057ABDF814308B4228BFC6
:10F910000B461380FFF7EDB8324DD5F88431A9EBD3
:10F920000303002BFFF6E5A8384A394B527C0799B0
:10F9300033F812308A7DDFED376A9FED376AC97D73
:10F940009BB207EE102A07EE903AB8EEC77AF8EEAF
:10F95000E77A27EE267A67EE867A099AC5F8842137
:10F96000C7EE876A40F2FF32FCEEE67ACDED057A0B
:10F97000BDF81430934228BF134609B1D31A9BB285
:10F980002648274D0178274C35F81160226825F864
:10F990001130921B134401311B4D236001F00F0203
:10F9A0001B0902702B80FFF7A4B8FEF709F81E4B65
:10F9B0001E4A1B68C31A9342C2BF134B00221A800F
:10F9C000FFF797B80CF08CFFFFE400BFD08D00204C
:10F9D000D34D6210343D0020F0000020D99000206B
:10F9E000F1000020181F0020FD3E0020ABAAAAAAAB
:10F9F000DCB9002014200020D2A700200C7D0020BC
:10FA0000584000206F12833FA09100205C7D0020B1
:10FA10007C7D00200000C842000080442F3E002072
:10FA2000343E0020303E00204824002060E31600D1
:10FA3000003F0020AC910020C94AB2F90030002BF1
:10FA4000B8BF5B42B3F5E17FBFF66BAAB2F90230F3
:10FA5000002BB8BF5B42B3F5E17FBFF662AAC14B92
:10FA600093ED057AD3ED077AD3ED096A93ED030A96
:10FA700077EEA67A30EE070AF7EE000AB0EE007ACB
:10FA8000E7EEC70A30EE000A10F01CFCB6EE008A62
:10FA900020EE488A9FEDB40A38EE000AFDEEC07AE7
:10FAA00017EE903A2033402B40F226839FEDAF0AA9
:10FAB000AF4DDFEDAE7A85ED000ABDEEC87AC5ED3B
:10FAC000017A17EE103A2033402BC5ED027A00F28E
:10FAD0006B85B0EE480A10F06BFB0A2085ED030A37
:10FAE0000EF036F9FFF71DBA40200CF0F9FEFFF7D3
:10FAF00011BA04200CF0F4FEFFF701BA9D490E780C
:10FB000026E695F89031002B3FF427A9099B1B7836
:10FB100013F0010302BF012285F8903185F891218D
:10FB2000FFF71BB9944D012285F88821FFF7D2B861
:10FB3000012900F0DC849BF8C8210123B340013681
:10FB40001343042E8BF8C83105F10C057FF433AD57
:10FB5000FFF77EB908F1050168792CF031FD002826
:10FB60003FF40DAB012F40F0468605F10D01A87A58
:10FB70002CF026FD002840F03A868049E87B2CF0E6
:10FB80001FFD00283FF40CAB032F40F02C867C496E
:10FB9000287D2CF015FD002840F021867949687EEB
:10FBA0002CF00EFD00283FF40CAB052F40F013861F
:10FBB0007549A87F2CF004FD002840F008867349A1
:10FBC00095F823002CF0FCFC00283FF40CAB072F29
:10FBD00040F0F9856E4995F828002CF0F1FC0028DA
:10FBE00040F0E2856B4995F82D002CF0E9FC0028E7
:10FBF0003FF40CAB092F3FF409AB0926334603EB66
:10FC000083031D44644B6978AA7889F804601970ED
:10FC10005A70FFF7FBBA614810F007FE00283FF466
:10FC200012A914200EF094F8FFF70DB902200CF081
:10FC30006FFE2388FFF737B95D2A00F073825B2AD5
:10FC400000F0F9845E2A00F05385562A00F05485AE
:10FC5000972A00F0AD85A72A00F02F85504C238805
:10FC60009B0740F0FA84A2F1B703072B00F27982D8
:10FC7000DFE813F0680277027702770275027702F5
:10FC800073027102002D48D05CF821309B454FEA89
:10FC90004102FFF4B2AD434B424E9B5C06EB0209BE
:10FCA000002B00F0D780022B47D199F8013003EBED
:10FCB000830303EB830303F2EE239BB20329DFBF2D
:10FCC000012606FA01F90C9E26EA0906CEBF1BB2F0
:10FCD0001BB20C96BEF1000F3FF494AD0A9E20F8C3
:10FCE0001630B8F1000F03D10D9E022E7FF68AADBB
:10FCF0000388B0F80290B0F804804B4498442A4B33
:10FD00000FFA88F883FB0863284EA3EBE87326F804
:10FD100002801BB24FF0010874E52B464A00069E94
:10FD20004CF821606AE5D3B2022B04D9032B7FF48F
:10FD3000C0AD7346AFE53B46ADE5A35ABEE71C4BED
:10FD40001B78002B7FF4D3AAB8F1000F3FF4CFAAA1
:10FD5000012C7FF43DAB9AF82030FFF79BBA00BF2F
:10FD6000AC4C0020641C0020DB0FC93F00000000E9
:10FD7000A0000020D9900020181F0020ED3900209D
:10FD8000F2390020F7390020FC390020013A002028
:10FD9000063A00200B3A0020D8540020D05300200F
:10FDA000FC4C00205840002056555555842000201A
:10FDB000BC2500203146C04810F037FD002800F077
:10FDC000BA8085F88F6118F0B3FCFEF72BBF43F0C3
:10FDD0004002934222803FF49DA8B84B0225142193
:10FDE000FF220E201D7059709A700DF0B1FFFFF7C1
:10FDF00091B843F00402934222803FF480A8AF4BB5
:10FE000002251421FF220E201D7059709A700DF0EA
:10FE10009FFFFFF774B8AA4BAA4A0E9201221A70EC
:10FE2000A94B04931B21A44810F0FFFC00287FF489
:10FE3000FFACDFF8C0A2A54DDAF80C202B68CAF899
:10FE400008309B1AC82B00F2FA83089B1E6806F440
:10FE5000805636E5CBB2022B40F24683032B7FF46B
:10FE60006CAF129B139E002E08BF2B4626E7002284
:10FE70000FE0437803EB830303EB830303F2EE23EA
:10FE80009BB20132A24221F8023B00F102003FF492
:10FE900018AD15F812301BB1022BEAD00B88F0E731
:10FEA000D3B2032BFAD83B46EBE7B2F5FA7FFEF666
:10FEB0004CAF95F88E31002B7EF447AF099B1B7831
:10FEC000012213EA020485F88E213EF434AF18F0C3
:10FED00001F87F4B0693089B7E4C1B68FEF73ABFE8
:10FEE00043F00102934222803FF4DBA8734B1421BC
:10FEF000FF2202250E201D7059709A700DF028FF08
:10FF00002388FFF7CEB800230593FFF7BDB9B2F5FC
:10FF1000FA7FFEF61AAF95F88E21002A7EF415AF0F
:10FF2000099B1B78012185F88E11D90700F1728396
:10FF300018F0FEFBCDE7099B674A1B781060D807D5
:10FF40007EF575AE654B1B78002B3EF4FEAE9AF83D
:10FF50000330002B7EF4F9AE95F88F310133DBB21C
:10FF6000032B85F88F317EF6F0AE5D4B5B7813B9CD
:10FF7000002C7EF4EAAE17F0ADFFFEF753BE594AEF
:10FF800059491068B5F98C21C66981FB06018911B0
:10FF9000F617701A00F5FF407F3082423EF735AE0B
:10FFA000891B0A4412B2A5F88C21FEF72EBE082048
:10FFB0000CF096FCFFF73BB84C4A079BD488049A98
:10FFC0001B8BB2F90620191B8A4271DD23449A4229
:10FFD000B4BF00240124FEF7A8BDC8398A425ADA0A
:10FFE0009BF8C8119A7841FA06F3D9073FF512AB8E
:10FFF000524201200B920DF0D1FF7B1E0B9A162B63
:020000040801F1
:1000000000F21981DFE813F0F9011E02E001470256
:1000100034025B02CB01B6019F0188017101170117
:1000200047025C015B02CB01B601460130011A01B7
:100030000501ED00D7002CF081FA032240F6B83319
:100040008AF82020CAF81C30FFF758B92A68DAF875
:100050001C301344CAF81830FFF7BAB90A202CF044
:10006000E7FA26880746002800F0A282F10640F150
:100070008D831F4D95F8D071002F7EF458AF0D2061
:100080000DF066FE012385F8D0312688002F7FF41D
:10009000DFAAFEF74CBF9BF8C8310122B24023EA29
:1000A000020309F5FA728BF8C831AA60FFF7B2BAF9
:1000B0000124FEF73ABD00BFD0530020183A0020BB
:1000C000D2A70020FD3E0020DCB900200C7D0020DE
:1000D000A04C0020FC4C0020A8450020D990002016
:1000E0002C54002028A10020D34D621010A700201E
:1000F000181F0020AC91002010F05AF8D8E400211D
:10010000C94810F092FB00287FF4C9AA322385F871
:100110009201A5F89431FFF7C2BA002A0CBF012062
:10012000022067E7C14B00220120C149C14C0B608E
:10013000C14B227006930DF031FF089BBF4C1B682A
:10014000FEF708BE012018F0C3FFBB4B0693089BC7
:100150001B68FEF7FFBD0220F5E70320F3E7002050
:10016000F1E7792A00F0C1837A2A00F0B8839E2A49
:1001700000F0AE839D2A00F07783AE2A00F06D83F5
:10018000AD2A00F06383EF2A00F05D83FD2A00F0C2
:100190004883FB2A00F00184FE2A00F0FB83F72A43
:1001A00000F0CD837B2A00F0BF83089BA24A1B6826
:1001B0000692FEF7CFBDDBF8CC01DFF8848290F821
:1001C000361098F8023011446429A8BF642121EA4E
:1001D000E17180F83610002B40F0E8832BF03CFBF7
:1001E000A9E4DBF8CC01DFF8588290F8371098F8D2
:1001F00002301144FE29A8BFFE2121EAE17180F8F6
:100200003710002BEAD016202CF05CFADBF8CC017A
:10021000E4E70A98DFF8288241781144B1F5967F27
:10022000A8BF4FF4967121EAE171417098F802304D
:10023000002B40F0B583DBF8CC01CFE7DBF8CC0135
:10024000DFF8FC8181781144C829A8BFC82121EAC0
:10025000E171817098F80230002BBFD014202CF08F
:1002600031FADBF8CC01B9E7DBF8CC01DFF8D0815B
:1002700041781144C829A8BFC82121EAE171417021
:1002800098F80230002BA9D013202CF01BFADBF8D1
:10029000CC01A3E7DBF8CC01DFF8A481017811449D
:1002A000C829A8BFC82121EAE171017098F802307D
:1002B000002B93D012202CF005FADBF8CC018DE74F
:1002C000DFF87C810A9898F802304179114464295A
:1002D000A8BF642121EAE1714171002BABD00E204F
:1002E0002CF0F0F9DBF8CC0178E7DBF8CC01DFF893
:1002F0005081017A98F802301144C829A8BFC8215A
:1003000021EAE1710172002B3FF468AF0B202CF061
:10031000D9F9DBF8CC0161E7DBF8CC01DFF820810B
:10032000C17998F802301144C829A8BFC82121EA30
:10033000E171C171002B3FF451AF0A202CF0C2F9DA
:10034000DBF8CC014AE7DBF8CC01DFF8F4808179F7
:1003500098F802301144C829A8BFC82121EAE171E8
:100360008171002B3FF43AAF09202CF0ABF9DBF898
:10037000CC0133E7DBF8CC01DFF8C480417998F891
:1003800002301144C829A8BFC82121EAE171417196
:10039000002B40F00F83112F7FF454AF1EE7DBF8E2
:1003A000CC01DFF89C80017998F802301144C8290B
:1003B000A8BFC82121EAE1710171002B40F0DF8262
:1003C000102F7FF455AF09E70A99DFF874800F7991
:1003D0001744642FA8BF642727EAE7770F712CF032
:1003E0008BF998F80230002B3FF425AF03203946F3
:1003F0002CF068F9DBF8CC01F0E60A98DFF84080D1
:1004000001781144FA29A8BFFA2121EAE1710170AB
:1004100098F80230002B3FF40EAF01202CF052F977
:10042000DBF8CC01DAE600BFD0530020664D002097
:10043000004D00208CA70020A04C0020FC4C002088
:10044000864E00200A98DFF884848178114464295C
:10045000A8BF642121EAE171817098F80230002B75
:100460003FF4E9AE02202CF02DF9DBF8CC01B5E623
:100470000A98DFF85884C17998F80230114481F362
:100480000801C171002B3FF4D6AE05202CF01AF9FB
:10049000DBF8CC01A2E60A9BDFF83084997998F862
:1004A000020011446429A8BF642121EAE171997115
:1004B000002840F087820D2F7FF404AFBBE6DBF805
:1004C000CC01DFF80884C17898F802301144C829BB
:1004D000A8BFC82121EAE171C170002B40F03C8225
:1004E0000F2F7FF4DBAE79E6129BFFF7E7BB049991
:1004F00031F912209978B2F5617F4FF4966393FB3E
:10050000F1F36CDB40F633019142A8BF11460C2F8A
:10051000A1F5617191FBF3F100F07181182F7FF467
:100520000AABC9B2C8290B46A8BFC823DBF8CC0167
:10053000C27DDFB297423FF4FEAA9A1ADFF88C839D
:10054000C77548BF0732D71098F802300137FFB29D
:100550003BB9002F3FF4EFAA38460DF01FFDFFF71F
:10056000EABA18202CF0AEF8F3E7C34BC3491A6877
:100570004FF47A73B3FBF2F3C3EB431203EB820243
:10058000089B1B68D2001F06A1F8A82000F1A180DB
:10059000BB4A0692126855077EF5DBABB94ABA4CE6
:1005A0000A211180FEF7D6BBB0EE670AFFF795BAB5
:1005B000F20600F1DD800B202CF03AF8002840F024
:1005C000A180B30600F11D81B04D95F8D031002B0C
:1005D0003FF455AD002F7FF43BA8FEF7A8BC0C2FCD
:1005E00040F0CE8000273946A94B0B915B78BB4287
:1005F0003FF4A1AADFF8D482384618F069FD98F8D4
:1006000002300B991BB1C9B20C202CF05BF80137FA
:10061000FFB29EE79F49089B0A60994A1B680692B1
:10062000994CFEF797BB9C4A0792FFF77BB806F4FC
:100630008056FFF746B9994B0122022075E5984A8A
:10064000089B1E68136823F004031360012306F45B
:1006500080568AF82130FFF734B90023BB2A14935F
:1006600000F0DC80B72A00F0D580BE2A00F0D080F0
:10067000BD2A7FF476AD4FF6FE718A4A8048D6894E
:1006800006909089334401449181D38115F0FCFD9B
:100690000FF0D4F815F0E0FDFCF74AF801200DF05A
:1006A0007DFCB5F88C21089BFA3A00211B68A5F85F
:1006B0008C2185F88E11FEF74DBB7B49089B0A788B
:1006C0006F481B68069042F004020A706E4CFEF7F9
:1006D00041BB754A127896077FF55AAF734A127D6F
:1006E000042A7FF655AF19F0CBFB089B1B684FE738
:1006F0006F4B0222032018E5FCF7BEF995F88A211A
:10070000FFF7A6BA6B4A6C4B528993ED007A07EE5D
:10071000902AF8EEE77AB0EEC77AB4EEE77AF1EE17
:1007200010FA7FF54EAF93ED017AB0EEC77AF4EE92
:10073000C77AF1EE10FA7FF744AFB3063FF544AF46
:1007400020200CF0E5F895E80C005C490A600846AA
:1007500041F8043F2DF048F9594B01221A704B4DD6
:1007600095F8D031002B00F012812688FEF770BF7B
:1007700010200CF0B5F8524B26881F7001271AE79D
:10078000182F7FF4D8A900210B46CFE610200CF0DB
:10079000BFF820200CF0A4F84A49081F2DF024F9D6
:1007A000474B02221A70DAE708263346FFF727BACA
:1007B0003349454A089B06914FF4C8711B68118064
:1007C000314CFEF7C7BA07263346FFF718BA06269C
:1007D0003346FFF714BA05263346FFF710BA04264E
:1007E0003346FFF70CBA03263346FFF708BA022652
:1007F0003346FFF704BA01263346FFF700BACFB2FB
:10080000F2E620200CF06CF82D4B00221A70A6E7BF
:10081000022132E719464FF6FE732EE719460223EE
:100820002BE70021012018F077FBB5F88C21089BFD
:1008300013491B680691963AA5F88C21002285F889
:100840008E21FEF787BA00210846ECE7FF21002041
:1008500021F067FE95F88A2195E40121002021F01E
:1008600060FE95F88A218BE40021FF2021F059FEDB
:1008700095F88A2181E400BFC08D0020D08500203A
:10088000A04C0020EEBB0020FC4C0020181F0020D4
:100890008CA70020A845002098840020B44D00209B
:1008A000F84C00200C540020FE4C00208C5D0020F1
:1008B000024E00207C480020C04A00202C2400204A
:1008C000EC470020E4470020F0BB0020864E0020CB
:1008D0000021012021F025FE95F88A214AE43C4AB6
:1008E000137A43F0010313725FE4394A137A23F059
:1008F0000103137259E4374B85F8901185F8910183
:100900000693354CFEF7BCBE002C3EF40CAA334DCA
:1009100095F88931002B3EF432A90DF0FDF9002342
:1009200085F88931FEF72BB94FF4FA61022018F0EF
:10093000F3FA284B0693089B1B68FEF70BBA0021BD
:10094000042070E70B20FEF79BB9244D17F0C2FA84
:1009500085F88941FEF713B90F200B922BF0B2FEF8
:10096000DBF8CC010B9ABBE5002BD0D01C491D4A0B
:1009700009684FF47A7000FB03131360C7E7102077
:100980000B922BF09FFEDBF8CC010B9A18E50127A8
:10099000FFF775BB0021032045E70021022042E755
:1009A00015202BF08FFEDBF8CC0117E417202BF07D
:1009B00089FE40E411200B922BF084FEDBF8CC0181
:1009C0000B9AE8E40D200B922BF07CFE0B9A72E55B
:1009D00000490020A04C0020FC4C0020181F0020E3
:1009E0000C7D0020A44500202DE9F047C74C63682A
:1009F00020469847002800F0C380C54B1B78012291
:100A0000042B84F83C2000F0BD80B4F91610B4F932
:100A10001820B4F91A3021636263A363BD4B1B88AD
:100A2000002B69D0BC4DD4ED0C7AD5ED004A95ED84
:100A3000050A95ED015A95ED067AD5ED035A95ED27
:100A4000026AF8EEE76AD5ED047AA4EEA60AA5EEEE
:100A5000267A67EEC07AA5EEC07AE6EE267A85EDB4
:100A6000057AC5ED067A32F033FDD4ED0D6AD5ED89
:100A7000094A95ED0E0A95ED0A5A95ED0F7AD5EDD6
:100A80000D7AD5ED0C5A95ED0B6A2063F8EEE66A07
:100A9000A4EEA60AA5EE267A67EEC07AA5EEC07A85
:100AA000E6EE267A85ED0E7AC5ED0F7A32F010FD6E
:100AB000D4ED0E6AD5ED124A95ED170A95ED135A4D
:100AC00095ED187AD5ED167AD5ED155A95ED146A8F
:100AD0006063F8EEE66AA6EEA40AA6EE857A67EEF3
:100AE000C07AA0EE657AE6EE867A85ED177AC5EDD6
:100AF000187A32F0EDFCA063884FA17F884822F07D
:100B0000A9FF3B88002B40F08480864ED6F8D45154
:100B1000854B1B685B0743D4B5F90070216B636B91
:100B2000A06B824A824E92ED026AD2ED006AD2ED4B
:100B3000015AC91B2163B5F90270DB1B6363B5F968
:100B400004703568C01B07EE900AB8EEE75A07EE4E
:100B5000901AB8EEE77A07EE903AF8EEE77A36EEBA
:100B6000056A36EE877A77EEA57A0135A06382EDC5
:100B7000026A82ED007AC2ED017A3560BDE8F08745
:100B8000BDE8F0876B4BB4F91600B4F91810B4F94E
:100B90001A2018802063598061639A80A2633DE720
:100BA000B6F89421322A00F08880002A66D196F89F
:100BB0009131002BB0D06048D6F8F0215F4980FB1E
:100BC0000273D217C2EB23122A80D6F8F42180FBDD
:100BD0000273D217C2EB23126A80D6F8F831A78AC3
:100BE00080FB0302DB17C3EB2213DB1BAB8000236C
:100BF000CB6086F8913115F047FB0EF01FFE15F023
:100C00002BFBFBF795FD01200DF0C8F9D6F8D45168
:100C100082E7444E226BD6F8D451B3F5C87F4FF02B
:100C2000000323632B80398818BFD6F8D801B7F8A2
:100C3000008008BF0020B1F5C87F18BFD6F8DC31AE
:100C4000616B02440B440020B8F5C87F6063C6F8AE
:100C5000D821C6F8DC31688052D0D4F838E0D6F814
:100C6000E011A0637144B8F1010FA880C6F8E0114B
:100C700068D008F1FF38A7F8008049E7D6F8F001FE
:100C8000236B00210344C6F8F03121632980D6F894
:100C9000F401636B61630344C6F8F4316980A36BAC
:100CA000D6F8F801A1630344012AC6F8F831A980F7
:100CB00075D0013AA6F8942179E72B8820491F487E
:100CC000276BA6F8E4310023B5F802E0B5F804C0BC
:100CD000C0684B608B602363C6F8F0712B80616B3A
:100CE000C6F8F41163636B80A16BC6F8F811A363B7
:100CF000A6F8E6E1A6F8E8C1C6F8EC01AB80D8E7B3
:100D0000A36BC6F8E031A063A880B2E7B44C002022
:100D1000C8490020F0540020F4540020F0BB00200B
:100D2000E44C0020181F0020D08D002068A1002076
:100D300064A10020CC4900201F85EB510C540020F9
:100D400008210020DFF88CC0DFF884E0C8328CFB7B
:100D500002A9C833D217C2EBE9128CFB03A9DB1737
:100D6000C3EBE913C8316B802A808CFB013CA28A5B
:100D7000CB17C3EBEC139B1AAB80CEF80C0015F02D
:100D800083FA0EF05BFD15F067FAFBF7D1FC4046E5
:100D90000DF004F9B7F80080D6F8D45169E70B20BC
:100DA00086F8961186F890210CF0D2FFD6F8D4512F
:100DB000074BB6F8E421B6F8E671B6F8E801D6F8C4
:100DC000EC112A806F80A880B6F89421D96070E772
:100DD0000C5400201F85EB512DE9F0478C4B1B78FC
:100DE000DB07074644D58B4B8B4D1C788B4E012C73
:100DF00059D01CD3022C07D189498A4A0988128804
:100E0000914201D901241C70EB7AE3B12B89D3B153
:100E1000854B1B78BBB10CF021F9002800F09B80BA
:100E20002B7B83422CBF0121002131700CE07C49D7
:100E30007E4A098810886A7B801A8842E2DAEB7A57
:100E40000024002BE2D131782A79632A06D8022CBB
:100E5000774E00F0BA803378002B5DD1754AAB7ABB
:100E60008C4238BF0C461470002B4CD1BDE8F08783
:100E70006B4B694D19885B88E878CB1A83EAE3727B
:100E80008142A2EBE3721DD32B788B421AD3614BC4
:100E90001C78E01E012861D96749097802294FD0E2
:100EA000012C5E4EA5D15F4A5D491288687B098896
:100EB000121A914239DD5D4A12888A42A4D2002476
:100EC0001C70A1E7B1EB400FE1DC524B1C78E11E36
:100ED000012940F29480022ADEDC57494F4E0878FF
:100EE000DFF84481DFF844C1DFF838E10021032452
:100EF000022834701C7088F80010ACF80010AEF8AE
:100F0000001081D11FE0012C71D0022C0BD10720E1
:100F1000BDE8F0470CF01CBF7068381A474B984288
:100F200058DD72709AE7BDE8F08702241C706BE709
:100F3000022AD2DD4049097802294FF0040464D125
:100F40003949364E09783E48022ACCBF0022012298
:100F5000C28081804BE70221317075E7022A9BDC59
:100F600095F800C091FBFCFC0CF1010CBCF1080FE2
:100F7000DFF8B4A0304EA87895F801E096F800802C
:100F80002A4CDFF8A090254EA8BF4FF0080C8AF835
:100F900000C01FFA8CFA10FB0AF01EFB0AFE80B29A
:100FA000DFF88CA02080A9F800E000244FF0640E48
:100FB000B8F1020F34701C70CAF804408AF801E0DE
:100FC0007FF439AF0FFA8CF1BDE73078A0B9012377
:100FD00077603370C2F164021A4B00FB02F083FBAE
:100FE0000023C017A0EBA3506430707036E70820D0
:100FF000BDE8F0470CF0ACBE7368F81A8EE7032C1E
:1010000096D10D49097802299AD0044EFCE600BF1A
:10101000D054002050270020844C00205627002068
:10102000A84A002054270020BE4A00205227002052
:10103000FC250020A6910020C84900207F9698003A
:10104000CC4900206BCA5F6B08B501210220FDF777
:10105000E9F9094B1B7803F00503052B08D00021A3
:101060000120FDF7DFF900210846FDF7DBF9FEE777
:101070002AF05CFEF3E700BF4C3500202DE9F04F6D
:10108000BC4B1E788BB0002E40F08180BA4BBB4C1D
:101090001D78BB4FDFF80CB305F00105A4F10A0978
:1010A00054F80A0CB8B14FF0CC0808FB0698FCF7CE
:1010B00045FF80B154F80A0CFCF738FF14F8023CE5
:1010C000024683B924283BD075B354F80A0CFCF7C8
:1010D00035FF0028EED10136032E04F1CC04DFD118
:1010E0000BB0BDE8F08F012B2ED0022B33D0032B99
:1010F00040D0042B00F06981052B00F05781062BAE
:10110000E3D114F801ECBEF1000F00F0DC81BEF178
:10111000010F00F01F8201360023032E04F8023C69
:1011200004F1CC04BCD1DBE7232A54F80A0C00F00C
:101130008281944B93F832309342B8D1F8F784FB14
:10114000012304F8023CC0E74D2800F0678100232A
:1011500004F8023CB9E700233C2804F8023C00F004
:1011600057813E28B1D10122032304F8012C04F851
:10117000023CAAE7C028EAD80021042304F8050CA1
:1011800004F8040C04F8061C04F8023C9DE77E4BAE
:1011900018680028A4D00EF03FFADFF80CA27B4DAF
:1011A000DFF8F891DAF80000FCF7C8FE002897D0C5
:1011B000DAF80000FCF7BAFE09281BD03F2819D046
:1011C0002B68002B67D1042800F0BE810C2800F0AA
:1011D000CA807F28E6D0A0F12002D2B25E2AE1D8F0
:1011E0000BB92028DED05A1C09F803002A601CF035
:1011F0003FFFD7E72C68002C5AD1654FA34607F56F
:101200002478BBF1000F08BFBB4610374745F8D123
:10121000BBF1000F00F05281103FDBF800003A688C
:10122000065D135D9E42204402EB040140F04481C0
:10123000661E4E4422460BB9FD2A5CD906F8013FD2
:1012400001322A6010F8013F11F801EF9E45F2D0FB
:101250000AB15F4512D04F481CF012FF5F4508D31A
:101260005BF8100B1CF00CFF09201CF001FFBB45C4
:10127000F6D949481CF004FF2A680024944291D210
:10128000661E4E4416F8010F1CF0F2FE2B68013466
:101290009C42F7D386E70C2865D00A2834D00D2865
:1012A00032D07F2800F0BE80FF2B3FF67BAF92E765
:1012B000374E002706F52478BB4602E01036464537
:1012C0000DD02246316848460EF002FD0028F5D1C7
:1012D000B346002FF2D1374610364645F1D13B4692
:1012E0005F469B46002B98D1002F3FF45BAF294807
:1012F0001CF0C6FEB4E7511C202009F8020029604A
:1013000009F801300A46A4E71CF03BFF23212348DB
:1013100033F0B2F8002800F01581A0EB0900286036
:1013200090B1431E19F80310202940F0308109EBD9
:10133000030243B112F8011D202903F1FF304FD100
:101340000346002BF6D12B604FF4807200214846F3
:1013500033F07BF8074B1B78002B3FF4C1AE0E48EF
:101360001CF08EFE1EE70E481CF08AFE0A481CF098
:1013700087FE17E787A70020D05400205E78002062
:10138000181F0020C4840020143A00208C3B002049
:10139000884E0408A47A0408AC7A04088C3A002029
:1013A000B47A0408D0450408883A002014F8063CB2
:1013B00014F8051C994273D814F8043C83427FF456
:1013C000C6AE062304F8023C9BE614F8043C04F87D
:1013D000030C5A40052304F8042C04F8023C74E67C
:1013E0002B606C4C002204F5247809F8032002E0FD
:1013F0001034444550D02168484613F0C3F9002802
:10140000F6D0444548D2E368984700232B609BE719
:10141000032204F8013C04F8022C56E6022304F8E7
:10142000023C52E6013B00225B482B6009F8032096
:101430001CF026FEB6E6594B5949DB78594ADFF8CD
:1014400090E11060003318BF01230B70564B574AD0
:10145000CEF80030564BC7F800224FF0400E012165
:1014600087F808E2C7F8FC01C7F8040287F80952B8
:10147000504819701DF054FA4F481CF001FE4FF40B
:1014800000600BF05DFA4D4B93F83230232B3FF4A4
:1014900055AE14F8023C32E649481CF0F1FDB4E7C1
:1014A00014F8041C08EB03005140013304F8041C39
:1014B00004F8063C827208E62246C9E64148103F1D
:1014C0001CF0DEFDCCE69BE80F000DF1280C0DF1C1
:1014D000080888E80F004CF824ED14F8053C14F8CF
:1014E00003AC0694624623444FF0010C414606A823
:1014F000ADF822E00793ADF820A08DF824C002F0EB
:101500009BFE40B1029A304B03924146A4F10A007F
:1015100002930BF0B1FFDDF80480002304F8023CD5
:10152000B8F1000F3FF4D7AD54F80A0C0CF02CF8CA
:10153000013654F80A0CC047032E04F1CC047FF4A2
:10154000AFADCDE52868EBE6204811F0C1FF0BB048
:10155000BDE8F08F14F8053C14F8032C06942344DE
:1015600007936E2A4FF0000308930993ADF82020EB
:101570007FF4D1AD06A80EF02AFC06A80EF01CFCE4
:1015800006A80EF019FC06A80EF016FCC3E50346EB
:1015900027E700BF884E0408DC7A04088CA70020E7
:1015A000B8270020883A0020182100206DC00008CC
:1015B00087A70020E07A0408AC7A0408C4840020DD
:1015C000C07A0408A47A0408F8BB00208C3A0020F2
:1015D000143A00202DE9F04F2DED028B95B0064610
:1015E00028F0C4FA9C4B1D7825B115B0BDEC028BD8
:1015F000BDE8F08F994B1B685A05F6D5DFF8A89225
:10160000D9F80020002A00F02381954CD4F8283125
:1016100003F5F43348339E42C0F01A81914F94F899
:101620002C313968C4F82861013384F82C318B07D8
:1016300001F1858511F0140F41F0668594F82C3185
:1016400013F0070801F0DA85282B874B029301F08D
:1016500056875E209047854B1B78002B6BD0804CC3
:10166000834AD4F83431F31A934201F20F84DFF83D
:101670003CA29AF80080B8F1000F33D1DFF8009255
:10168000D9F80000FCF75AFCC0B201280ED9022894
:10169000784F42F040803B78002B42F0E681D4F84E
:1016A0003C31F31AB3F57A6F82F0528272480768C0
:1016B000002F40D09AF80030BBB9704BD9F8000029
:1016C0001B689B781E3B012B4FF0020142F2DF8129
:1016D00004301AF06DFF012200238AF8002084F8FC
:1016E000483126E0644807682FB3D4F8443140F607
:1016F000B732F31A93421ED994F84031002B02F00E
:101700000080013BDBB284F84031002B01F06E8693
:1017100017F8011B94F84821076094F8493158489C
:101720000A440133006884F8482184F84931FCF701
:1017300009FCC4F84461534A029B12781B68012AD1
:1017400003F101030C9301F0CB824F4B1B787BB16B
:10175000DFF85C91D9F8003053B1414C029BD4F8CA
:101760005C21D3F800B0ABEB0202632A01F2E68100
:10177000DFF8408198F800A0BAF1020F01F012865C
:101780003C4F97F87430032B01F0A8843F4B1B7833
:1017900073B13F4D2B685BB1314CFCF711F9D4F8B4
:1017A0006831039044F61F62C31A934200F22C8101
:1017B000384B1B78002B7FD1374B1B7843B1284C1B
:1017C000D4F8B83203F50043E8339E4281F0FE823C
:1017D000324B1B78002B3FF408AF214E304C314D7B
:1017E00006F2C1272068FCF7A9FB00283FF4FDAEF4
:1017F0002068FCF79BFB2B7880465A1E33B120688B
:101800002A70FCF79BFB0028F2D1EEE60322394652
:10181000781E32F000FE96F8C03296F8C12286F8A3
:10182000C38283F47F4383F0FF039B1A1FFA88F877
:101830009BB2B8EB132FD5D196F8C222DBB29A42F5
:10184000D0D1781E1AF0D6F82B7818442870C9E742
:10185000054B0293FFE600BF87A70020D08D002034
:1018600064210020A04C00200C7D00206A92002002
:101870003F0D030024000020184D0020144D0020CF
:10188000104D00206B920020789200208092002062
:1018900084920020F0920020019300208A92002080
:1018A0009092002094920020D89100201C4D00209E
:1018B0007C4C0020CE3E0020474C2278002A41F08C
:1018C0000682DFF83C9199F80040002C79D1434D15
:1018D0002878002842F05480414C424DD4F8B02280
:1018E0002978414B93FBF1F313449E42FFF464AF1C
:1018F00094F8B4323D4AC4F8B062D75CFB0702F1F9
:10190000F981B80702F19281790702F13F823A0723
:101910004CD5374BDFF8EC800D930DF15009A3F156
:101920003D0249F8202D0021A3F1400203F8401C9C
:1019300002231121517093704846D8F800100EF020
:1019400055FA4846D8F804100EF050FAB8F80E30A0
:10195000284903EBC3039B00053381FB0321DB17FD
:10196000C3EBA10189B248460EF057FAB8F810301F
:1019700003EB8303590089B248460EF04EFA1E4B22
:101980001B789B0743BFB8F8081001F57A7189B23C
:101990004FF47A7148460EF040FA0C9B98F81420E8
:1019A000591C0C9148461A7028F086F894F8B43205
:1019B0002978013393FBF1F201FB123384F8B4323E
:1019C000FAE60E4D2F6E002F41F0D485044B89F8B6
:1019D0000070C3F8B062EFE65C920020F89200203D
:1019E0006421002000930020A0860100FC920020CA
:1019F0001C92002067666666FE4C0020089300205B
:101A0000F99200208C5D002094F86E31002B41F09B
:101A10006185DF4B1B6803F00802002A48F603418A
:101A20004AF60B404BF60F4249F6074704BF024601
:101A30000F4613F0040F4FF0190118BF17469B060D
:101A400084F86E1103D547F4804747F020070BF068
:101A5000F7FAC7F30909002842F0D881CD4B9B79EA
:101A6000002B42F02A83984664204FF0FF3A4FF053
:101A7000000C0C970D97ADF83CC0CDF842C0CDF8E6
:101A800046C0CDF84AC0CDF83890ADF83E80ADF8EC
:101A900040A08DF84E000CAF0FCFDFF808E384F8BC
:101AA00005C0AEE80F0097E80F00AEE807002EF87B
:101AB000023B71464FF0010C1B0CFE271F20C82271
:101AC00001F81E39A770A27184F807C0E07094F87D
:101AD0007E01207180F0F10383EA0313DAB2130967
:101AE00083F0E70343EA022383EAC2031BB283EADB
:101AF0000312D2B2C3F3072383EA121343EA022389
:101B000083EAC2031BB283F0C80282EA0212D2B295
:101B1000C3F3072383EA121343EA022383EAC203CF
:101B20001BB283EA0C0787EA0717FFB2C3F3072249
:101B300082EA171242EA072200EB0C0382EAC70787
:101B40000EEB0C0084F87E31278011F8013B7B40BE
:101B500083EA0313DBB21A0982EA172242EA03225C
:101B600082EAC3031BB29FB281422780EDD183F08A
:101B70007C0383EA0313DBB24FEA131E8EEA172EAF
:101B80008EEA032E8EEAC30E0FFA8EFE1FFA8EF92E
:101B9000DFF814C2A4F800905FFA8EFE4FEA19290C
:101BA00084F8289084F827E00CF5D37804F1220A11
:101BB000DCF80000DCF80410DCF80820DCF80C305D
:101BC00047460FC70CF1100CD445B846F0D1DCF8ED
:101BD00000003860704F9CF8043088F8043007F13A
:101BE000270884F8CDE184F8CE9117F8011F286802
:101BF000FCF7A8F9B845F8D194F86F21002A41F014
:101C0000FD836649029B08781B680A2184F86F11DE
:101C1000002801F09B85DFF894E10128BEF8001050
:101C2000059142F251820228BEF8028002F0C3817F
:101C3000BEF804100491032802F05A820428BEF86A
:101C400006A002F050820528BEF8087002F0478214
:101C50000628BEF80AC002F03F820728BEF80C1022
:101C600001D0BEF80E2094F87EB10C938BF03003B7
:101C700083EA0313DBB24FEA131E494884F804B029
:101C80008EF07A0E4EEA032E00888EEAC303DFF848
:101C900020E1C0EB00208EFB009E8644C0171BB2E3
:101CA000C0EB6E200690C3F3072E83EA0310059B5A
:101CB000C0B24FF0000963F30F098EEA10130593C9
:101CC0004FF0000E049B68F31F4967F30F0E4FF0AF
:101CD0000008002763F30F0861F30F07059BCDF899
:101CE00034906CF31F4E62F31F474FF0000C9DF8C9
:101CF0001820CDF83CE06AF31F48CDF838801097E3
:101D00008DF844C08DF8452043EA00230DF13008DA
:101D100083EAC007B8E80F003FB287F0C80989EA34
:101D20000919DFF880E084F805C05FFA89F9C7F384
:101D30000727AEE80F0087EA191747EA092398E852
:101D4000030083EAC9031BB283F023074EF8040B98
:101D500087EA0717FFB2C3F3072282EA1712704619
:101D600042EA072282EAC70720F814190BF1010B97
:101D70004FF0230CFE211622C82384F87EB1278061
:101D800084F807C00EF1020EA170E270A37111E099
:101D9000A04C0020844C00200B230020D4A700205E
:101DA000A09100206C21002066210020DCB90020D9
:101DB0000308208010F8013B7B4083EA0313DBB269
:101DC0001A0982EA172242EA032282EAC3031BB2FB
:101DD0009FB270452780EDD183F0F40383EA0313AB
:101DE000DBB24FEA131E8EEA172E8EEA032E8EEA1E
:101DF000C30E0FFA8EFE1FFA8EFCD64FA4F800C059
:101E00004FEA1C295FFA8EFE84F81EE084F81F90CA
:101E10007968BA683868FB6807F5D37CACE80F00CE
:101E200038697969BA6904F2C518ACE8070004F2A8
:101E3000A71784F8C59184F8C4E117F8011F286832
:101E4000FCF780F8B845F8D194F87231002B41F0D6
:101E50005183C14F3B681922980684F8722140F1E2
:101E60000E83BE4BDFF800831B78990741F1928601
:101E700098F81430042B8CBF4FF003094FF002097F
:101E8000FBF79EFDB8F81030B8F808200C9003EB73
:101E900083035B00ADF84A304FF47A70D8F8003015
:101EA0008DF84C900E93B8F80E1098F814E0D8F80E
:101EB00004308DF84DE000FB02F24FF0000A4FF0C5
:101EC000FF300DF13009CDF834A010920F93ADF82A
:101ED00048101190CC46BCE80F00DFF890E2AEE865
:101EE0000F009CE80F00AEE807007246182122F8A8
:101EF0001C39E17194F87E1184F805A081F0780313
:101F000083EA0313D8B2030983F0F60343EA0023FC
:101F100083EAC0031BB283EA0310C0B2C3F30723F2
:101F200083EA101343EA002383EAC0031BB283F061
:101F3000C80080EA001C5FFA8CFCC3F3072080EA2B
:101F40001C1040EA0C2080EACC0000B280F018039C
:101F500083EA0313DBB2C0F3072080EA131040EAE0
:101F6000032080EAC30301F1010CFE204FF01E0A9A
:101F70004FF0C80BA0700EF1020E217184F87EC1E3
:101F8000238084F803A084F806B0184612F8011BD9
:101F9000414081EA0111C9B20B0983EA102343EAE7
:101FA000012383EAC10109B288B272452080EDD1D4
:101FB00081F0180181EA0111C9B20A0982EA1023ED
:101FC00083EA012383EAC1031BB29AB261492280EA
:101FD000DBB2120A04910692059384F8272084F854
:101FE00026308E4601F5D37B04F1220ADEF800008C
:101FF000DEF80410DEF80820DEF80C30DC46ACE831
:102000000F000EF1100ED645E346EFD1DEF80000CA
:10201000CCF800009DF81430DFF854A184F8CC31DE
:102020009DF8183084F8CD31D3461BF8011F28687D
:10203000FBF788FF4A4B5B45F7D1FBF7C1FCD8F8AB
:1020400000103B68B8F808200591D8F804100691F4
:1020500013F0140F4FF47A7101FB02F141F01D856A
:102060000F4694F87EB10C908BF06A003D4BDFF880
:1020700004E1B3F90420109780EA0010C0B203090C
:1020800083F0D50343EA002383EAC0031BB283EA4B
:102090000310C0B2C3F3072383EA101343EA0023FB
:1020A00083EAC0031BB28EFB020E05980D90D21777
:1020B0004FF00008C2EBAE0206980E9083F0C80CF9
:1020C0000F91ADF84A20ADF84480ADF84680ADF8E8
:1020D00048808CEA0C1CCE465FFA8CFCC3F30727C1
:1020E000BEE80F0087EA1C1747EA0C2787EACC07EF
:1020F000DFF878C084F804B03FB2ACE80F0087F096
:1021000021039EE8070083EA0313DBB2C7F3072726
:1021100087EA13170BF1010E47EA03278CE8070043
:1021200087EAC30384F87EE14FF0210B4FF0FE0EE7
:102130001C27C8220CF10C0C84F8058084F807B029
:1021400084F802E0ACF11C01E7701846A27123800C
:1021500012E000BF66210020A04C0020FE4C0020B1
:1021600031230020AC4C00208C5D00206C2100202D
:102170000B2300206766666611F8012B424082EA55
:102180000212D2B2130983EA102343EA022383EA3C
:10219000C20212B290B261452080EDD182F0680295
:1021A00082EA0212D2B24FEA121B8BEA102383EAB0
:1021B000022B8BEAC20B0FFA8BFB1FFA8BF3DB4F60
:1021C00023805FFA8BFB1B0A059384F8253084F883
:1021D00024B007F5D37C04F1220838687968BA681E
:1021E000FB68E646AEE80F0010374745F446F4D1E9
:1021F0003B88AEF800309DF81430CD4F84F8CAB15A
:10220000D04684F8CB3118F8011F2868FBF79AFEF6
:102210004745F8D194F87EC1C64A84F804C08CF0D2
:10222000EB0383EA0313D9B20B0983F0C50343EA36
:10223000012383EAC1031BB283EA0310C0B2C3F3D4
:10224000072181EA101141EA002181EAC00109B2A7
:102250000CCA81F0C80787EA0717FFB24FF0000EDB
:10226000C1F307210D93CDF838E081EA17130C92E2
:1022700099E8070043EA072383EAC7030FFA83F8C4
:10228000AD4B84F805E088F0310783E8070087EA62
:102290000717FFB2C8F3072383EA171343EA07239C
:1022A00083EAC703277A607AA27AE17A94F80CE08D
:1022B00094F811801BB25F4087EA0717FFB2C3F39F
:1022C000072383EA171343EA072383EAC7031BB2F2
:1022D000584080EA0010C0B2C3F3072383EA10130A
:1022E00043EA002383EAC0031BB25A4082EA021089
:1022F000C0B2C3F3072282EA101242EA002282EA45
:10230000C00212B2514081EA0111C9B2C2F30723DF
:1023100083EA111343EA012383EAC1031BB28EEA65
:10232000030E8EEA0E1E5FFA8EFEC3F3072383EAC6
:102330001E1343EA0E23677BA07BE17B227C83EAAA
:10234000CE031BB25F4087EA0717FFB2C3F3072330
:1023500083EA171343EA072383EAC7031BB25840F3
:1023600080EA0010C0B2C3F3072383EA101343EAE4
:10237000002383EAC0031BB2594081EA0111C9B2AC
:10238000C3F3072383EA111343EA012383EAC1035A
:102390001BB25A4082EA0212D2B2C3F3072383EA85
:1023A000121343EA022383EAC2031BB288EA03083A
:1023B00088EA08185FFA88F8C3F3072383EA18133A
:1023C00043EA082383EAC803A17CE27CDFF8748136
:1023D0001BB2594081EA0111C9B2C3F3072383EA52
:1023E000111343EA012383EAC1031BB25A4082EA74
:1023F0000212D2B2C3F3072383EA121343EA022381
:1024000083EAC2031BB283F0270787EA0712D2B21E
:10241000C3F3072787EA121747EA022787EAC207AA
:102420003FB20CF10103BAB25FFA87F94FF0310CF9
:10243000FE200C2184F87E31C8234FEA122E228020
:1024400084F807C0A070E170A37184F81490049F11
:1024500084F815E07968BA68FB683868B7F810C086
:10246000A8E80F0028F803CB84F8BBE184F8BA9100
:102470001AF8011F2868FBF765FDD045F8D194F8DC
:102480007671002F41F031802C4B94F87E81B3F9A6
:102490000010B3F90220B3F904309FED296A677187
:1024A00007EE103A029B1B680C9388F06A0383EADC
:1024B000031306EE901AD9B20B0983F0D50343EA51
:1024C000012383EAC1031BB283EA03115242C9B25A
:1024D00007EE902AC3F3072383EA111343EA01238B
:1024E000F8EEE77AF8EEE66AB8EEC77A83EAC10357
:1024F0001BB267EE867A66EE866A27EE067A0020C1
:1025000083F0C80ECDED0E7ACDED0D6A8DED0F7A0C
:102510001090119012908EEA0E1C0DF130095FFAA6
:102520008CFCC3F3072EB9E80F000DE066210020F4
:102530002F230020E04700206C210020AC4C00201D
:1025400088C3E43A0C2300208EEA1C1E4EEA0C2EAF
:102550008EEACC0EDFF888C40FFA8EFEACE80F00CE
:102560008EF01E0799E8070087EA071A5FFA8AFAD1
:10257000CEF3072787EA1A1747EA0A278CE80700ED
:1025800087EACA071C214FF0050A4FF01E094FF0D9
:10259000FE0EC82208F10103E17084F876A184F8E8
:1025A000079084F802E0ACF11001A2710CF10C0C60
:1025B00084F80480278084F87E3111F8013B7B4049
:1025C00083EA0313DBB21A0982EA172242EA0322E2
:1025D00082EAC3031BB29FB261452780EDD183F02D
:1025E000270383EA0313DBB21A0982EA172282EA7D
:1025F000032282EAC3031BB21FFA83FCDFF8E483E1
:10260000A4F800C05FFA83FE4FEA1C2C84F825C0B2
:1026100084F824E008F5D37904F1220AD8F8000000
:10262000D8F80410D8F80820D8F80C304F460FC757
:1026300008F11008D045B946F0D1E04FB8F80030A5
:10264000A9F8003007F1240884F8CAE184F8CBC166
:1026500017F8011F2868FBF775FCB845F8D194F806
:1026600077A1BAF1000F40F03A87D54B1B680522DD
:1026700084F877219A0641F17380D24ADFEDD27A4D
:10268000D18907EE101AB8EEC77A13F0140F27EEAF
:10269000277A01F0C084CD4BDFEDCB6AD3ED007A11
:1026A000F8EEE77A67EEA67A94F87EC1C84BC94A7D
:1026B000B3F90410B2F90620C74FC8488DED0D7A62
:1026C0008CF0220383EA03135FFA83FE4FEA1E13A2
:1026D00083F0590343EA0E23B2F5FA6F83EACE037F
:1026E0001BB2A8BF4FF4FA6283EA0318B2F57A7FEF
:1026F0005FFA88F8C3F3072EB8BF4FF47A72A2F5D9
:102700007A728EEA181E642303FB02F34EEA082E47
:1027100087FB03278EEAC80EDA17C2EBA71280FBED
:1027200001300FFA8EF7CB174FF0000BC3EBA0036D
:1027300087F0C8080DF13009CDED0E7AADF84220D2
:10274000ADF84030CDF830B0CDF83CB0CE4688EA98
:102750000818BEE80F005FFA88F8C7F3072787EA72
:10276000181747EA082787EAC8089D4FDEF800E0F7
:1027700084F804C00FC70FFA88F888F04A0383EA88
:102780000310C0B2C8F3072383EA10133A460CF1D2
:10279000010143EA002383EAC00342F810E9002064
:1027A0004FF04A084FF0FE0C4FF0140E84F87E11E3
:1027B000C82160712380043784F8078084F802C040
:1027C00084F803E0A171184612F8011B414081EA28
:1027D0000111C9B20B0983EA102343EA012383EAFA
:1027E000C10109B288B2BA422080EDD181F0140152
:1027F00081EA0111C9B24FEA111E8EEA102E8EEA4B
:10280000012E8EEAC10E774B0FFA8EFE1FFA8EFC58
:102810001F464FEA1C2B5FFA8EFE84F81DB084F829
:102820001CE0596838689A68DB68A4F800C007F5AE
:10283000D37CACE80F0038697969B7F81880049741
:10284000ACE8030004F2A717ACF8008084F8C3B129
:10285000B84684F8C2E104F2C31B18F8011F2868C7
:10286000FBF770FBC345F8D15F4B604A1B781278C9
:10287000013B12F00100DBB214BFC0214021172B35
:1028800003D85B4A134493F80CA05A4B1A88930759
:102890001ABF002341F01001012312F4027F18BF78
:1028A000022312F0100F18BF062312F0200F18BFDA
:1028B0001023002841F03C814FF0030894F87EC1BA
:1028C0000C938CF0460383EA0313DAB2130983F006
:1028D000920343EA022383EAC2031BB283EA031092
:1028E000C0B2C3F3072282EA101242EA002282EA4F
:1028F000C00212B282F0C80E8EEA0E1E00235FFAEA
:102900008EFE0320C2F307228DF834A08DF83780A5
:1029100082EA1E128DF835308DF836108DF83800A9
:1029200042EA0E2899E8070088EACE0E0FFA8EF8E0
:10293000DFF8ACA0E37188EA0819AAE803005FFA9F
:1029400089F9C8F3072888EA191848EA092181EAB1
:10295000C90994F808808AF800200FFA89F988EAF2
:10296000090282EA02185FFA88F8C9F3072282EAAC
:10297000181242EA0822607AA17A94F80B906371E7
:1029800082EAC80212B2504080EA0010C0B2C2F31C
:10299000072282EA101242EA002282EAC00212B240
:1029A000514081EA0111C9B2C2F3072282EA111231
:1029B00042EA012282EAC1021EE000BF0B2300208E
:1029C000A04C00208C5D00200AD7233CA44C0020A2
:1029D000AC4C0020DCB90020D34D621067666666FF
:1029E0006C2100206621002080580020D054002057
:1029F000E0450408FC4C002012B289EA020989EA89
:102A000009195FFA89F9C2F3072282EA191242EA28
:102A1000092294F80C80607BA17B84F804C082EAD0
:102A2000C90212B288EA020888EA08185FFA88F830
:102A3000C2F3072282EA181242EA082282EAC80296
:102A400012B2504080EA0010C0B2C2F3072282EAFC
:102A5000101242EA002282EAC00212B2514081EA18
:102A60000111C9B2C2F3072282EA111242EA01221D
:102A700082EAC102E17B94F8109013B281EA03026A
:102A800082EA0212D2B2C3F3072383EA121343EAA3
:102A9000022383EAC2031BB289EA030282EA02121A
:102AA000D2B2C3F3072383EA121343EA022383EA71
:102AB000C2031BB283F0320282EA0212D2B2C3F323
:102AC000072383EA121343EA022383EAC2031BB2F9
:102AD0009AB24FF0FE085FFA83FE0920C8210CF17C
:102AE000010C84F802804FEA1228E070A17184F88A
:102AF0007EC1228084F8128084F811E0049B18685B
:102B000059689A68B3F80CB00AF5CC7CACE80700B9
:102B10000AF5D47A8CF80290ACF800B084F8B88149
:102B200084F8B7E117F8011F2868FBF70BFABA45DC
:102B3000F8D1039BC4F86831FEF73ABEDFF83C8356
:102B4000BF4FDFF83CA3412019F0D4F9B8F90220B7
:102B500087FB0230D217C2EBA00080B219F0AEF9A9
:102B6000B8F9002087FB0230D217C2EBA00080B278
:102B700019F0A4F9B8F9042087FB0230D217C2EB90
:102B8000A00080B219F09AF99AF80010D9F8000064
:102B9000FBF7D8F994F8608118F0010700F033844E
:102BA000A84F3A68910640F18180A74ADFF8D482A5
:102BB0001278920740F1678798F81420042A8CBF96
:102BC000032302230393472019F094F9D8F8000057
:102BD00019F040F9D8F8040019F03CF9B8F80E20C3
:102BE0009A49D9F80000A1FB0232C2F347121146FC
:102BF0000492FBF7A7F99AF800003968049A11F0DB
:102C0000140F82EA00028AF8002040F09786B8F894
:102C10000820642000FB02F019F01CF998F81470E9
:102C2000039BD9F8000043EA8707FFB23946FBF758
:102C300089F99AF80020D9F80000574039468AF8F7
:102C40000070FBF77FF994F86081B8F1000F2DD187
:102C50007F4F4F2019F04EF9386819F0FBF878686B
:102C600019F0F8F8404619F0F5F80121D9F80000FC
:102C7000FBF768F9744A9AF800701278D9F80000E6
:102C800002F00108414687F001078AF80070FBF75F
:102C900059F99AF80020D9F8000088EA0202114692
:102CA0008AF80020FBF74EF994F86081694AC4F86D
:102CB0005CB108F10103DBB2A2FB0312D20802EB04
:102CC0008202A3EB420384F86031FEF751BD624BF0
:102CD00062491868FBF7FEF800232370FEF7F1BD88
:102CE0005F4F386800283EF430AD4FF0000ADFF83F
:102CF00098815C4CAB465546FBF720F9F8B1F5B925
:102D00004FF00109AA463868FBF710F983B27E2B11
:102D100000F05D8398F80120002A49D194F84C1105
:102D2000B1B11B2B84F84C2100F02B830D2B45D027
:102D3000386888F80190FBF701F90028E3D1AA462A
:102D400050460CAA48495D4619F0EEF8FEF7FDBC66
:102D50007D2B00F0F18494F8502122B180F0200303
:102D6000DBB284F8501194F84B21062A10D8B4F83D
:102D70004E1138681944A4F84E11A118013281F897
:102D8000543184F84B21FBF7D9F80028BBD1D6E7A2
:102D9000B4F84E2188F8019013449BB21A0A52FAF3
:102DA00083F3FF2BA4F84E31386802D12F4DA3E7EF
:102DB0003868FBF7C3F80028A5D1C0E73868A4F845
:102DC0004E21FBF7BBF800289DD1B8E794F8BC3240
:102DD000C4F8B862012B40F2988494F8BD222449CB
:102DE000981801EB8001013202F001024F6A84F869
:102DF000BD22BFB11F4D0D950DF15009123DA52308
:102E000049F8205D802284F8103115233146484668
:102E100084F8112184F81231B847002840F0F68375
:102E200094F8BC32144A013382FB0312A2EBE37222
:102E300002EB42029B1A84F8BC32FEF7C9BC00BF09
:102E400067666666A04C0020FE4C00201F85EB5193
:102E5000E0470020CDCCCCCCF49200201C92002086
:102E60000C4D002064210020AE220020B82200205A
:102E7000E04504088922002056555555AC4C0020E9
:102E8000804C00208C5D002024000020C54AC64BE9
:102E900092F80BE0029AD4F8381110681B88C34AE4
:102EA000401A4FF47A71DFB201FB0EF11B0A9777DB
:102EB000177588424FF00007D377537597701771D5
:102EC00080F00F84BA4BDFF814C31B68B949BA4FBE
:102ED0000868DFF80C9389683F688CFB038EDB176A
:102EE000C3EB6E1303F5FA739BB293761B0AD3768A
:102EF00089FB00A389FB01A9C017C917C0EBA30078
:102F0000C1EBA90107F5EA43DFF8D8E210773033C7
:102F1000001282F8201009121B12DFF8CC829EF8F2
:102F200000E0507782F821108CFB0790F917C1EB75
:102F3000601182F82330A14B98F814A083F81AA0EE
:102F4000783130371EF0020F82F8241082F8227098
:102F500000F0C483D8F800E0994AD8F80400DFF8FC
:102F60008CB282FB0E714FEAEE77C7EBA151039151
:102F700082FB0092C117C1EBA25203990BFB01E146
:102F800001EB410149000F460BFB020B0497B946C8
:102F90000BEB4B0B8B4F4FEA4B01059187FB099BCA
:102FA00087FB01194FEAA949CDF81C90B8F80E909B
:102FB0000399B8F8088002EB820209EBC90902EB19
:102FC0008202089201EB81074FEA89020599039278
:102FD00007EB8707049A0697CF17C10F099104984A
:102FE00079494FEAAB4BD2174FEADE7E83F809E00E
:102FF000ABEB020E01FB1E020798069908F5FA7862
:10300000BAF1050F1FFA88FAA0EB0708059F6E4872
:1030100083F815A04FFA8EF909EB8109414600FBB0
:1030200018789DF8240098730898684FDFF8C0E17D
:1030300049B201EB80018CFB020B4FEAE272049271
:10304000039ABEF800E08CFB08C087FB02C74FEA7A
:10305000E27C049AC2EB6B1203925D4A1FFA89F973
:103060001288ADF8102083F80A90039A83F813E0D1
:1030700089B24FEAE8784FEA112BC8EB6010CCEB2D
:10308000A7174FEA1A284FEA192C4FEA222A9DF86F
:103090000C2083F810B04FEA202983F80BC0D973B5
:1030A000C7F3072C4FEA1E2134BF4FF0320B4FF00D
:1030B000330B1A739DF8102083F80DA0587483F811
:1030C000129083F81680DF7183F808C0197583F8B1
:1030D0001BB01A77C4F83461FEF7C9BADFF814914F
:1030E000D9F80000FAF71AFF00283EF44FABD9F8E0
:1030F00000000121FAF70EFF0222002387F8742056
:1031000088F80030FEF742BB5E209047D9F80030C7
:1031100030209847284BD3F800805FFA88F026F0DB
:1031200031FCC8F3072026F02DFC94F82C3113F065
:10313000030800F0B783D9F80020FEF781BADFF862
:10314000B8809FED248A4FF0240A5E2090475046B5
:10315000D9F800309847204BF8EC016A9B8A07EEBB
:10316000103AF8EEE66AB8EEC77A0AF1010AC6EE3E
:10317000877A5FFA8AFA67EE887AFDEEE77ACDED14
:10318000027ABDF908B05FFA8BF026F0FBFBCBF3B7
:10319000072026F0F7FBBAF1270F00F0ED80D9F8F1
:1031A0000020D2E7B04A0020A84A002098920020D0
:1031B000A44C0020944C0020A84C0020C492002075
:1031C0006BCA5F6B83DE1B4340420F00D34D62101E
:1031D0003048002000007A44B44C00201F85EB5199
:1031E00067666666FE4C00208C5D0020806967FF84
:1031F000084D0020E83F0020E44C00205E2090476E
:10320000D9F8003002209847FF2018F079FB0378A6
:10321000FF2B00F0358490F901304FEAE3785FFA34
:1032200088F8D8B226F0AEFB404626F0ABFBD9F8C2
:1032300000305E209847D9F8003003209847FF20DF
:1032400018F05EFB0378FF2B00F01584B0F908300E
:10325000D8B2C3F3072826F095FB404626F092FB30
:10326000C84B1B78042B7DD0DFF854B3B4F82E1173
:103270009BF80020DFF834A391FBF2F302FB131359
:103280009BB2BAF80010A4F82E314FEA03181FFAC7
:1032900088F8642303FB01235200B3FBF2F348EAEE
:1032A0000328C3F303225E20D9F800301FFA88F800
:1032B00048EA02089847D9F80030062098475FFA94
:1032C00088F026F05FFB4FEA182026F05BFBAE4942
:1032D000B4F82E214B7ABAF800A00132012BA4F8E1
:1032E0002E2100F082864A7B0AEB8A031FFA83FABA
:1032F000002A40F02784D9F800305E209847D9F89A
:1033000000303A209847A14BA3FB0A384FEA5818DF
:103310001FFA88FB5FFA8BF026F034FB4FEA1B2084
:1033200026F030FBD9F800305E209847D9F80030FD
:103330003B209847642303FB18A39BB294480533B2
:1033400080FB0320DB17C3EBA000C0B226F01AFB02
:10335000002026F017FBDFF86C8298F80630002B6F
:1033600040F0AD833B68980600F1058294F82C315B
:10337000D9F80020FEF768B93968D9F80020FEF7BF
:1033800059B93868FAF7DAFD00287FF4D1AC38680B
:1033900084F84A9188F80190FAF7D0FD00287FF46C
:1033A000B2ACCCE4FAF70CFB7A4B1B68A0EB030B36
:1033B00040F6B8339B4500F2B481774B1A793A2A2C
:1033C00000F03C85002388F80030FEF7DFB938684C
:1033D00084F84AA184F84BA184F84C9188F801A0A4
:1033E000FAF7ACFD00287FF48EACA8E494F84811FD
:1033F00094F8493169484A1CFEF793B9013A84F8B8
:103400006F21FEF721BD664A1288D30513D4D0067A
:1034100000F14183910600F1D585530600F1028643
:10342000100700F10286D10700F1418612F0020F69
:103430000CBF04270C275B495B4A0B78D27803F05A
:1034400001030AB143F002035320039318F052FD25
:10345000564A128802EB820202EB8202900080B28E
:1034600018F02CFD002018F029FD514A514912880E
:10347000D9F80000C2EBC212520081FB02311144A4
:103480004FEAE278C8EB61285FFA88F84146FAF71C
:1034900059FD9AF80020039BD9F800001F4388EAE1
:1034A000020800218AF80080FAF74CFD3946D9F865
:1034B0000000FAF747FD9AF80020D9F800007A409A
:1034C000D2B211468AF80020FAF73CFD94F86081E8
:1034D000FFF7BBBB013B84F86E31FEF78DBB0AF1F1
:1034E000FF3A84F877A1FFF724BB013F84F8767197
:1034F000FFF7B5B8013B84F87231FEF7C0BF4FF05B
:10350000000A5E201F6884F82CA19047D9F800308B
:10351000DFF8B48017209847504626F033FA264B40
:10352000A3FB07239B0BA8FB03125209C2EB021259
:10353000A3EB8203D8B226F025FAD9F800305E203A
:103540009847D9F80030182098471C4BA3FB072355
:103550009B09A8FB03125209C2EB0212A3EB8203E0
:10356000D8B226F00FFA504626F00CFAD9F800200F
:10357000FEF76FB80024DFF8548027464FF0500A5A
:1035800029E000BFA6910020B04A00201F85EB5122
:1035900067666666D43E0020BC3E0020104D0020C9
:1035A000FC4C0020D0540020AC910020A84A002000
:1035B000A09100200308208073B2E745D34D62102C
:1035C000BE4A0020844C002089888888ED9A030830
:1035D000DBB283F3118815F804B0601C5946284407
:1035E00018F036FB002840F0A2810BF101031C44C7
:1035F000EFF311838AF312882A6E9442E8DB0022EB
:10360000DBB22A6683F31188FEF7E0B90C9EAE4266
:103610004FF000014FD941F2210015F8013B81EA3A
:1036200003235A0013F4004F80EA020192B289B2D8
:1036300008BF11464A0080EA020311F4004F99B214
:1036400093B218BF0B46590080EA010213F4004FF1
:1036500089B293B208BF0B465A0013F4004F80EAB8
:10366000020192B289B208BF11464A0080EA020301
:1036700011F4004F99B293B218BF0B465A0013F4DD
:10368000004F80EA020192B289B208BF11464B0096
:1036900011F4004F80EA03029BB292B208BF1A46AF
:1036A000530080EA030112F4004F9BB289B208BFB5
:1036B0001946B542B1D148460CF0D3FBA1490C9D47
:1036C000A1486D1A152DA8BF15252A462FF0C0FD5B
:1036D0009E4A94F8BC321570FFF7A4BB2D22DA760F
:1036E000F8E49B4B02991B780968C4F83811013B38
:1036F000012B3FF6E7AB1021022391701371FFF706
:10370000E1BB18F08BFFFEF714B8924A02EB83027C
:10371000576AFFF76EBB18F071FF01233B70FDF78E
:10372000C5BF8D4AB2F8623100210133A2F862317F
:1037300088F80010FEF72AB8386884F85091FAF734
:10374000FDFB00287FF4DFAAFFF7F9BA01468446A3
:10375000074682460490804605900246FEF783BAEB
:103760009FED7E7A13F0140F08BFF0EE477A7EF4D7
:1037700092AFFEF799BFDFF8FCA19AF800309907E5
:1037800000F10C82DFF8F0810027BB46D9F8003049
:103790005E209847D9F8003001209847584626F017
:1037A000F1F8384626F0EEF8D9F800305E20984758
:1037B000D9F8003009209847002026F0E3F80020CF
:1037C00026F0E0F8B8F8123098F81470B3F5967F48
:1037D0000AD994F82C2102F00F02072A04D842F2E9
:1037E0000F779F4228BF1F46D9F80030DFF88CB111
:1037F0005E209847D9F80030052098479BF808309C
:10380000002B00F0EB83A7F1200307EE903A9FED29
:10381000547AF8EEE77AF6EE006A67EE877ABEEE43
:10382000007AF5EEC07AF1EE10FA58BFB0EE667A83
:1038300077EE877AFDEEE77ACDED027ABDF9087072
:10384000F8B226F09FF8C7F3072026F09BF89AF805
:10385000002000230A930B93930700F1258194F82D
:103860003031012B00F02081BBF90030DFED3D6AE3
:1038700007EE103ABBF9023007EE903AB8EEC77A7D
:10388000F8EEE77A27EE267A67EEA67ABDEEC77ADB
:10389000FDEEE77A0CA88DED0C7ACDED0D7A26F0D1
:1038A00093F863E53049D4F82821304B8A421868F0
:1038B00040F23A8180EAE073A3EBE0732C4A1BB23A
:1038C00082FB03124FEAE37BCBEB621B4FF06408F1
:1038D00008FB1B380FFA88F80FFA8BFB5FFA88FA9F
:1038E0005FFA8BF2C8F30728CBF3072BD9F8003027
:1038F00002925E209847D9F8003010209847029A2B
:10390000104626F03FF8584626F03CF8D9F800302B
:103910005E209847D9F8003021209847504626F07D
:1039200031F8404626F02EF894F82C3103E4414655
:103930003A2018F0E9F80743FFB256E60B4A106840
:10394000FFF76AB974220020643C0020793C002013
:10395000A6910020E045040864210020000000003A
:10396000E4380E3F0050C3473F4B4C00A44C0020AE
:103970001F85EB51FE4C00208C5D0020B04A0020DA
:10398000CC49CD4B0093A1F13F07CC4BCC4A0B91D6
:1039900001F8404C0CA8CB490A970CF039FB0A9F60
:1039A0007B1C0A933C700A9B2922591C0A911A70AD
:1039B0000A9BEA22591C0A911A700A9BC822591CB8
:1039C0000A910CA81A702EF0D7FC00F101080CA97E
:1039D00042460A982FF03CFC0A9A02EB0803013396
:1039E0000A9302F808400A9B5A1C0A921C700A9B10
:1039F0005A1C0A921C700A9B5A1C0A921C700A9B41
:103A00005A1C0A921C700A9B5A1C0A921C700A9B30
:103A10005A1C0A921C700A9B5A1C0A921C700A9B20
:103A20005A1C0A921C700A9B5A1C0A921C700A9B10
:103A30005A1C0A921C700A9B5A1C0A921C700A9B00
:103A40005A1C0A921C700A9B0122991814A80A9108
:103A50001A7050F8283DDB1B3B7026F02DF89A4B6E
:103A60002C70C3F8B062FDF7A7BEC4F83C6187F8BC
:103A70000080FDF71BBE4FF000084046FFF7EBBB90
:103A80004046FFF7CFBB01230393FFF79CB8FAF73B
:103A900041FAFDF720BE3427CDE48C4B1F6807EBBD
:103AA00087077F00FEF7DDBA98E80C0001210AA81D
:103AB00084F830110A920B9325F086FF56E4D9F86A
:103AC0000030DFF828A2DFF820B25E209847D9F84E
:103AD000003028209847DAF800308BFB032BDB17E7
:103AE000C3EBAB0B5FFA8BF025F04CFFCBF3072059
:103AF00025F048FFD9F800305E209847D9F800300B
:103B000004209847B8F80830002B40F05E82DAF8BD
:103B1000083083F310085FFA88F025F033FFC8F30C
:103B2000072025F02FFF1DE4C246C3464246DDE6CE
:103B3000674AD278002A0CBF4FF004084FF00508FE
:103B4000FEF7BCBE9BF800309AFBF3FAFFF7D3BB3D
:103B50000123D9F800003B70FAF7E8F90746D9F8D5
:103B60000000FAF7E3F97F067DF4A0AD8A2800F0A3
:103B70008D828E287DF49AAD9AF80030002B7DF46A
:103B8000B1AD5448544B03602D2384F8403107688D
:103B9000FDF790BD4FF00109FEF772B9DFF85081D3
:103BA000D9F800304D4F5E209847D9F800301120E9
:103BB0009847B8F80E204FF4F36B0BFB02F287FB2B
:103BC0000237D217C2EB6737F8B225F0DBFEC7F336
:103BD000072025F0D7FED9F800305E20984719203D
:103BE000D9F800309847B8F80E303D4A0BFB03F384
:103BF00082FB0301DB17C3EB611382FB0321DA179E
:103C0000C2EB6112642101FB1233D8B225F0BAFE77
:103C1000002025F0B7FE9AF80030B8F808709A072F
:103C20007FF5B2AD5FFA87FB3F0AAFE5214A2D4B26
:103C30000D920DF15008A2F13D0048F8200D1988B1
:103C4000DFF8A890A2F1400300204FF00A0E02F81E
:103C5000400C082283F801E040469A700CF0DDF831
:103C6000D9F800302049DA1781FB0313C2EBA30314
:103C700099B240460CF0D1F809F0F0F9D9F8089063
:103C80000C9B4FEA1942591C0C911A700C9B4FEA7D
:103C90001922591C0C911A700C9B5A1C0C9283F817
:103CA00000900C9B5A1C0C921870404625F004FFA3
:103CB000FDF72ABE1C92002092A70020347B040846
:103CC0003C7B0408487B040864210020A44C0020AD
:103CD000AC910020184D00209892002089B5F8146E
:103CE0001F85EB51A84A002067666666944C002049
:103CF0008C5D0020DFF884939FEDCF8AB9F9023004
:103D0000CE4A0D9207EE903AF8EEE77A0DF15008A0
:103D100067EE887AA2F14003FDEEE77AA2F13D0159
:103D200048F8201D02F8400C0822CDED027A5A70A6
:103D30001E229A70BDF8081040460CF06EF8B9F9D2
:103D4000003007EE903AF8EEE77A404667EE887A60
:103D5000FDEEE77ACDED027ABDF808100CF05DF8C3
:103D6000B9F9043007EE903AF8EEE77A404667EE8C
:103D7000887AFDEEE77ACDED027ABDF808100CF0F6
:103D80004CF8404625F098FEFDF7BBBDAB4B0D93BC
:103D9000A3F1400900222121A3F13D0A03F8402CA0
:103DA00089F8021089F80120CDF830A028F032FC03
:103DB000A34BA44A1B88A44900280ABF11464FF010
:103DC00003084FF004085A0500F12181D80700F1DB
:103DD0002F8103F002039D4A002B1CBF4FF0030804
:103DE000114642469A482FF033FA0AEB080314A80A
:103DF000984A013340F8203D9B1A00220AF8082017
:103E000089F8013025F058FEFDF781BD924B934AA9
:103E10001B88927903EB830303EB83034FEA830848
:103E20001FFA88F8002A00F045818D4B1B680FFAB5
:103E300083FA09F013F940B2FDF719BE997803939C
:103E4000184613F0FDF900287FF4BCAA8249854F7B
:103E5000834A09888448854CF961DFF82492116807
:103E600003689268F962B4F86211C7F86CB0FB633A
:103E7000FA64D9F80000F965F8F7CCF88346002811
:103E80007DF47FAC5146D9F80000FAF743F8039B64
:103E900094F86421DB780493642A4FF0040387F8D4
:103EA000743040F02B8194F86531DFF8D8A1072BEE
:103EB00008BF84F865B194F86521069207EB021BF0
:103EC000DBF80410059108462EF056FADBF80830AE
:103ED00003935FFA80FB18462EF04EFAC3B20BEB49
:103EE0000300069A0599059308308AF8070022F026
:103EF0000F008AF80A0002F00F0203EBCB008AF8E9
:103F00000D208AF80E005A460AF10F002FF0A0F992
:103F1000059B03990BF109001A460AF106031844A0
:103F20002FF096F99AF8073003F1010BD3B1013B5A
:103F30005FFA83FC0CF1080CDFF84CE1D4440AF181
:103F40000700002310F8011B59408B00CA0883EAC0
:103F5000410302F018024B404EFA02F253408445EE
:103F6000DBB2EFD1424A04980BF802302FF01EF971
:103F700094F865310022013384F8653184F86421B6
:103F80009AF802305BB11AF80510D9F80000F9F779
:103F9000D9FF01359AF80230EDB2AB42F3D894F86C
:103FA00064310322013384F8643187F8742088F87F
:103FB0000020FFF795B811469446174692460492A2
:103FC000FDF751BE2427FFF736BA09F047F825F070
:103FD000D9FC002025F0D6FCFFF7C4B9F8B225F0D3
:103FE000D1FC380A25F0CEFC31E4D9F800305E204F
:103FF0009847D9F80030392098475FFA8AF025F0C1
:10400000C1FC4FEA1A2025F0BDFCFFF7A4B94FF020
:1040100003081849E5E6138907EE903AF8EE677A47
:10402000FEF742BB1027FFF706BA2027FFF703BAB7
:1040300011494FF00408D4E658A08B411C9200208F
:10404000FC4C0020187B0408207B0408307B04080B
:10405000DF910020DD910020A84A0020844C002040
:10406000944C002024000020A44C00206421002057
:10407000CE6F0020247B0408287B0408AC4C002071
:10408000E83F0020C86F00200007090E614B1B6845
:1040900098067DF50BAB9AF80030002B7DF422AB2F
:1040A0005D485E4B03602D2384F840316FE508279F
:1040B000FFF7C1B94FF0FF33B9E6594B8046B3F96A
:1040C00000A06420FDF7D3BC1146944617469246E3
:1040D00004929046FDF7C7BD1146FDF7C4BD1146D9
:1040E0009446FDF7C0BD114694461746FDF7BBBD8B
:1040F0001146944617469246FDF7B5BD97F87530C0
:10410000DFF82CA1474905951A0704BF0133DBB23C
:10411000072B28BF01234FEA031B07EB0B02107C80
:1041200000228AF80A2011F800C05FFA8BF203928D
:104130000AF10D02039D07EB0B012843BCF1010FAF
:104140001070C96802F101000ED9ACF10205EDB2A0
:1041500005F1020E9644024602F8011B72454FEA31
:104160001121F9D101352844BB4421F0600201330B
:104170009BF81110DBB20A43082B027000F1010218
:1041800044D04FEA031B07EB0B00264D007C264969
:1041900015F800C0039D511A05F1100E01EB0C0536
:1041A00006955FFA8EF50395069D132DC2DD059DDC
:1041B000DFF880E0C9B28A1DD2B242F040008AF82E
:1041C000070002F1010BCAB14A1DD2B208325244B3
:1041D00003920EF1010C00221CF8010B50408200EA
:1041E00082EA4002C1084240104801F0180140FA3A
:1041F00001F14A4003996145D2B2EDD104980BF820
:104200000E2087F875302EF0D1FFB9E60649059DDE
:10421000511ACDE7A04C0020184D0020C492002078
:10422000944C0020E0450408D56F00200007090EDB
:10423000C86F0020CE6F00202DE9F04F95B0B0F987
:1042400008500D81EDB2442D00AF0C46904600F0B1
:104250004484064643D9812D00F07D8300F2988086
:10426000542D00F0CC8040F2D6806E2D00F00384F7
:10427000802D40F0D380764B93F800A00AF1020A1B
:104280001AF0FF0A00F09780724BDFF8F481724E4B
:10429000DFF8F0B19A4403F101090A2516E0322D46
:1042A00001F0FD82A5F13C00C0B2132841F2FE826C
:1042B00000232268511C216015702268D14502F14B
:1042C00001012160137076D019F8015B0A2DE6D147
:1042D000BBF80030FF2BA8BFFF23DBB2E9E7052DB9
:1042E00000F0E98320D8022D00F0818040F2128393
:1042F000032D00F0B783042D40F0908057492046ED
:104300002A460BF069FD002120460BF0AAFD226829
:104310000021531C0125236028462B465437117079
:104320006381BD46BDE8F08F242D5ED040F2A882A7
:10433000282D00F05983382D70D10A68484B01258B
:10434000511C2160157022680521501920601170E0
:1043500022680A215019206011702268002150192A
:10436000206011702268197850192060117022683D
:104370005978501920601170226899785319236078
:104380002B461170284654376381BD46BDE8F08F37
:10439000A02D18D040F29382B82D00F06183FE2D3D
:1043A0003CD1304D05F1080635F8021B20460BF0D4
:1043B00058FDAE42F8D101252B462846543763817B
:1043C000BD46BDE8F08F284B084619680BF032FD5A
:1043D000264B204619680BF02DFD254B1968204609
:1043E00001250BF027FD2B46E7E7224BF6E70422D9
:1043F0002149204601250BF0EFFC2B46C2E70B6854
:1044000000215A1C2260197022680125531923606B
:104410002B461170B6E7522D3FF479AF214628465E
:1044200007F0A0F903460028C5D1742D00F085825D
:10443000772D29D13268716891421EBF531C3360B9
:1044400011780E4A08BF194620462DF057FDB2E7F5
:10445000A9490020144604080027002092A7002044
:10446000514D0020CC490020107AFF1F147AFF1F05
:10447000187AFF1F9C4E0020B47B0408851D040899
:104480006766666628270020F52D01F06783762D84
:1044900000F02B83472D01F09E82292D336801F017
:1044A0008182392D01F04B82212D01F05B827168F0
:1044B0000B3DCA1AEF2D00F2778401A050F825F0C9
:1044C0008D530108A94D0108A94D0108A94D010806
:1044D000A94D0108A94D0108A94D0108A94D0108E0
:1044E000A94D0108A94D0108A94D0108A94D0108D0
:1044F000A94D0108A94D0108A94D0108A94D0108C0
:10450000A94D0108A94D0108A94D0108A94D0108AF
:10451000A94D0108A94D0108A94D0108A94D01089F
:10452000C5530108A94D01086B530108A94D0108A5
:10453000EF540108A94D0108A94D0108A94D010832
:10454000C7540108A94D010851540108A94D01089B
:104550001F540108A94D01082B550108A94D010858
:1045600019550108A94D0108BD510108A94D0108BF
:104570006B510108A94D0108A94D0108A94D010879
:10458000A94D0108B7430108A94D01086D5801085C
:10459000A94D0108A94D010853580108A94D01086A
:1045A000854B0108A94D0108A94D0108A94D010835
:1045B000A94D010807580108A94D0108A94D010896
:1045C000A94D010813580108A94D01081D53010800
:1045D000A94D0108A94D0108DF520108A94D0108A4
:1045E000A94D0108A94D0108A94D0108A94D0108CF
:1045F000A94D0108A94D010871520108A94D0108F2
:1046000021570108A94D010867560108A94D010865
:10461000B9550108A94D010851550108BF570108B6
:10462000A3570108A94D0108A94D0108A94D01088A
:10463000A94D0108A94D0108A94D0108A94D01087E
:10464000A94D0108A94D0108A94D0108A94D01086E
:10465000A94D0108A94D0108A94D0108A94D01085E
:10466000A94D0108A94D0108A94D0108A94D01084E
:10467000A94D0108A94D0108A94D0108A94D01083E
:10468000A94D0108A94D0108A94D0108A94D01082E
:10469000A94D0108A94D0108A94D0108A94D01081E
:1046A000A94D0108A94D0108A94D0108A94D01080E
:1046B000A94D0108A94D0108A94D0108A94D0108FE
:1046C000A94D0108A94D0108A94D0108A94D0108EE
:1046D000A94D0108A94D0108A94D0108A94D0108DE
:1046E000A94D0108A94D0108A94D0108A94D0108CE
:1046F000A94D0108A94D0108A94D0108A94D0108BE
:10470000A94D0108A94D0108A94D0108A94D0108AD
:10471000A94D0108A94D0108A94D0108A94D01089D
:10472000A94D0108A94D0108A94D0108A94D01088D
:10473000A94D0108A94D0108A94D0108A94D01087D
:10474000A94D0108A94D0108A94D0108A94D01086D
:10475000A94D0108A94D0108A94D0108A94D01085D
:10476000A94D0108A94D0108A94D0108A94D01084D
:10477000DD570108A94D01084F51010825510108D5
:10478000A94D0108A94D0108A94D0108A94D01082D
:10479000A94D0108A94D0108A94D0108A94D01081D
:1047A000A94D0108A94D0108A94D0108A94D01080D
:1047B000A94D0108974F0108454F01080D4F010809
:1047C000A94D01086D4E0108114E0108F54D010873
:1047D000A94D0108DB4D0108B950010891500108AD
:1047E000D54B0108DF4B0108A94D010861500108B4
:1047F000A94D0108A94D01083750010809500108C9
:10480000F54F0108B34D01088B4D0108614D0108BA
:10481000354D0108A94D0108A94D0108A94D010810
:10482000A94D0108A94D0108A94D0108A94D01088C
:10483000A94D0108A94D0108A94D0108A94D01087C
:10484000A94D0108A94D0108A94D0108A94D01086C
:10485000154D0108A94D0108A94D0108BD4C0108DD
:10486000A94D0108A94D0108A94D0108594C01089D
:10487000A94D0108A94D0108A94D01083F4C0108A7
:10488000202D7FF4CBAD0B68AB4D591C6A782160AD
:104890001A7023682A78591C21601A702368AA7834
:1048A000591C21601A70298920460BF0DAFA236816
:1048B0006A79591C21601A702268A97929E5822D2C
:1048C0007FF4ACAD0B689D4A9D4D11789A4A581CF7
:1048D00020601970118920460BF0C3FA994B2268A9
:1048E0001B88FF2B02F10101A8BFFF232160137079
:1048F000A96881F3100189B220460BF0B2FA296849
:1049000001F30F0189B220460BF0ABFA8E4B2268FF
:104910001978FEE4012D7FF481AD0B680022591C4B
:1049200021601A7023685A1C22601D70226825219C
:10493000531C23602B46117024E532687168914244
:104940001EBF531C33601178804A08BF19462046A9
:104950002DF0D4FA2FE57E4B1E78033616F0FF06B5
:104960003FF429AD7B4BDFF814821E4403F1010AAA
:104970004FF00A0920E0B9F1500F00F08D87B9F12E
:10498000320F00F0A987A9F13C00C0B2132840F211
:10499000BD870025294623685A1C2260204683F8DB
:1049A00000900BF05EFA294620460BF05AFA564565
:1049B0003FF401AD1AF8019BB9F10A0FDBD1664B48
:1049C0009D68196805EB85054FF6FF736D009D42E4
:1049D000A8BF1D469942A8BF194625EAE57521EAF8
:1049E000E171ADB289B2D6E70B68DFF894915B4E06
:1049F000591C022221601A7023684FF006085A1CC5
:104A0000226083F8008023680A22591C21601A70F2
:104A1000236801255A1922601D70B9F8001020463C
:104A20000BF01FFAB9F8021020460BF01AFA2368AF
:104A30005A19226083F80080236850225919216096
:104A40001A7023680022591921601A703188204693
:104A50000BF007FA718820460BF003FA2B4691E41D
:104A60003F4BBBE40B685A1C0A601D700B685A1C54
:104A70000A601D704BE4334B0A681B88304DFF2BD6
:104A8000A8BFFF23511C21601370A96881F3100196
:104A900089B220460BF0E5F9324B204619880BF01D
:104AA000E0F9296801F30F0189B2204601250BF0D6
:104AB000D8F92B4666E40B222B4920460BF08CF9E3
:104AC00008222A4920460BF087F9012507222849A8
:104AD00020460BF081F92B4654E4002A3FF46BACDE
:104AE000244B136001252B464CE43268511C316085
:104AF0001278002A01F01581102A01F06E811E46FD
:104B0000194625686B1C236020462A700BF092F929
:104B1000314620460BF08EF9174B204619680BF0F2
:104B200089F9204600210BF09CF9002120460BF06A
:104B300098F9FFF7ECBB00BF844C0020BE4A002070
:104B4000944C0020A84A0020A6910020911D040842
:104B5000A949002024460408B4260020E8260020A5
:104B6000E8380020A0910020BC7B0408C87B040822
:104B7000D47B0408A9B4010824260020F8260020CC
:104B8000FC5300205A1C3260A84A1B78DFF8D08200
:104B900013700023C8F8003030460BF0F6F8336885
:104BA000D8F80020A249A34D10435A1CC8F80000B1
:104BB00032601B780B7230460BF0FEF828603046EE
:104BC0000BF0FAF8686030460BF0F6F8A860304653
:104BD0000BF0F2F830460BF0EFF8FFF7ECBB0D2AC4
:104BE00040F0E2805A1C32601D78072D00F2DC8014
:104BF000DFF8709230464FF00C080BF0DDF808FB40
:104C000005F809EB0805A88030460BF0D5F8E880D8
:104C100030460BF0D1F8336828811A46591C3160B0
:104C200012F8021BA97232605B78EB7230460BF00F
:104C3000ACF8012549F808002B46FFF7A3BB7E4BD3
:104C40001B78DB0700F1B0800125F7F797FBF7F73A
:104C50006FFD2B46FFF796BB30460BF0ADF833687F
:104C6000B8851A46591C316012F8021B326087F869
:104C70002E105A7887F82F20DA1C32609A7887F83D
:104C800030201A1D3260DA7887F831205A1D3260E0
:104C90001B7987F8323007F12C000023BB860AF01D
:104CA000E5FF664A664B1268801A4FF0010561F114
:104CB0000001C3E906012B46FFF764BB5A1C3260B2
:104CC0001A780F2A70D8991C3160C2EBC2025D4974
:104CD00058788854D81C30600A4499785170191D4E
:104CE0003160D9789170591D31601979D170991D51
:104CF000316059791171D91D31609979517103F180
:104D000008013160DB79937101251AF085FC2B468F
:104D1000FFF738BB30460BF04FF8DFF83481A8F8C6
:104D20000E0030460BF048F80125A8F80C002B4681
:104D3000FFF728BB19465A1C3260434A11F8020B90
:104D40001070316059785170D91C31609978917028
:104D5000191D3160DB78D37001252B46FFF712BB9C
:104D600030460BF029F8DFF80081A8F81000304633
:104D70000BF022F8A8F8120030460BF01DF80125C0
:104D8000A8F814002B46FFF7FDBA1A46591C3160EB
:104D900012F8020B3260DA1C597832609A7825F0EA
:104DA00097FA00287FF407AB4FF0FF352B46FFF74B
:104DB000E9BA1A46591C3160244912F8020B0870EE
:104DC000326023495A788A70DA1C3260214A9B7813
:104DD000937001252B46FFF7D5BA174B1B78D807E0
:104DE0003FF5E9AA0125F7F77DFEF7F7A1FC2B4671
:104DF000FFF7C8BA104B1B78DA073FF5DCAA164A52
:104E00001378012543F0040313702B46FFF7BABA59
:104E1000094B1B78D9073FF5CEAA104B4FF4C87247
:104E200001251A802B46FFF7ADBA00BF805800203D
:104E300098840020F8350020D05400200C7D0020FC
:104E400028240020FC370020DC450020AC8D002009
:104E50000C5400201C540020FE4C0020F0BB00200D
:104E60009C4E00203C370020D0590020092A9BDDB1
:104E7000DFF8EC831A46591CD8F80050316012F85C
:104E8000021B297032605A78AA70DA1C32609A7854
:104E9000642A03F10401A8BF64226A713160DA78E0
:104EA000642A03F10501A8BF6422AA7131601A794E
:104EB000EA719A1D32605A79642A03F10701A8BF8A
:104EC00064222A7231609A79EA7003F10802326032
:104ED000DB792B7130460AF06FFF726833686881A6
:104EE000D11A00290CDD591CD8F800003160521A83
:104EF000002A1978417203DD9A1C32605B78437096
:104F0000012527F0F9FB2B46FFF73CBAC14A106890
:104F1000DA1C01462133951E356012F8035C0D70D2
:104F2000551E356012F8025C4D70326012F8015C5B
:104F30008D7003329A4201F10301ECD126F08CFC12
:104F4000FFF739BA5A1C32601A78B349002A00F0C8
:104F50004B870A7842F00202981C0A70AF4D30600D
:104F60005B782B7530460AF010FF286030460AF057
:104F70000CFF686030460AF01FFF288130460AF0B7
:104F80001BFFA74AE8811378012543F00203137041
:104F90002B46FFF7F7B9C2F34705122D3FF604AFD2
:104FA000C5B107F1500307F12A0903EB450AC846CA
:104FB000AAF1260A30460AF0FFFE28F8020FC24581
:104FC000F8D1984B39F8022F23F8022FC845F9D1B0
:104FD000112D09D8944A6B00023B13440021223260
:104FE00023F8021F9A42FBD1904A01231D461370F9
:104FF000FFF7C8B9874B8E4918684E2201252EF05D
:1050000027F92B46FFF7BEB919465A1C3260894A68
:1050100011F8020B1070316059785170D91C316051
:105020009B78937030460AF0C7FE834B0125D880E9
:105030002B46FFF7A7B930460AF0BEFEDFF8F8812D
:10504000A8F8000030460AF0B7FEA8F80200304683
:105050000AF0B2FE0125A8F804002B46FFF792B92A
:10506000DFF8009299F80030002B3FF4A4A9DFF894
:10507000F881002530460AF09FFE26F043FD99F89E
:105080000030A8EC010A01359D42F3DBFFF793B92C
:105090005A1C32601878060600F12D87674B1B7882
:1050A000DD073FF588A9032828BF00200125F7F771
:1050B00049F92B46FFF766B95A1C3260304693F81F
:1050C00000A00AF062FE814630460AF05EFE054608
:1050D00030460AF05AFE804630460AF06DFE3046F1
:1050E0000AF06AFE30460AF072FEBAF1000F00F0D4
:1050F000B886BAF1100F7FF45EA9514BC3F8049043
:105100009D60B8F1000F02D04E4BC3F800804E49AD
:105110004E4B0222081F01251A7028F065FC2B4611
:10512000FFF730B95A1C4A4932600A781B78002AC6
:1051300040F0B18604220A70464A9B001380F8F7BB
:105140003FFC3F4B012518622B46FFF71BB9DFF8E8
:105150001C8100233046C8F800300AF016FE0125F5
:10516000C8F800002B46FFF70DB90721B2FBF1F19B
:10517000C1EBC105521B7FF417AEC9B201F1FF3973
:105180005FFA89F900293FF416A9DFF8CCA009F1EC
:10519000010915465A1C326093F900102E4B4FF04E
:1051A000000893F902208A4203F1080300F0BE854B
:1051B00008F10108B8F1060FF3D1F5E55A1C326089
:1051C0001A780E2A3FF6F0AD991C31605D78032DF8
:1051D0003FF6EAAD2148062101FB02F1421803F136
:1051E000030E5571C6F800E09D784554191D3160D5
:1051F000D9785170591D316019799170991D3160BC
:105200005979D170D91D31609B79137101252B46D5
:10521000FFF7B8B8004D0020FE4C00208C5D002048
:10522000EA4700205A3D00205C3D0020803D0020E0
:10523000947104080454002010A70020D0540020CA
:10524000282400202426002030240020EC470020C1
:105250002E3E0020A0910020C4840020F4380020BD
:10526000044D0020A9490020683A0020E8380020B9
:10527000C14B1B68002B3FF49EA828F0ADFCFF2813
:105280003FF499A830460AF097FD3F2840F2158672
:10529000DFF81483002588F8005033687268A8F896
:1052A0000400D21A012A7FF786A81A46591C3160D9
:1052B00012F8021B88F8021007F150003260002239
:1052C0005D7800F8242D28F059FC97F82C30AB427B
:1052D0003FF471A8284628F075FCFFF76CB8A74A80
:1052E0001278012A3FF667A818465A1C3260DFF888
:1052F000BC8210F8022B88F80220DA1C891A306070
:1053000001295878326040F3CB8530460AF054FDCD
:105310000125A8F800002B46FFF734B85A1C32606C
:1053200093F80080B8F1110F3FF63EAD9A1C326041
:10533000934D5B7805F8183030460AF03DFD40F695
:10534000CA039842A8BF184640F2EE23984205EBE4
:105350004801B8BF18460125A0F2EE222B461920BD
:1053600092FBF0F24A70FFF70DB8DFF84482002399
:10537000C8F8003030460AF008FDD8F800300125A2
:105380000343C8F800302B46FEF7FCBF7D49102AC6
:1053900013464FF0000228BF10230A604A608A605B
:1053A000CA600A74002B3FF406A83268013913441E
:1053B0000132326012F8010C01F8010F9A42F7D164
:1053C000FEF7F9BF5A1C32601D78132D3FF6ECAC86
:1053D0009A1C326058787B622CF0CAFD00283FF49A
:1053E000E3AC7B6A684A017802F82510D91C316069
:1053F00002EB850299785170191D3160D97891704E
:10540000591D31601B79D370002027F0B5F85F4B30
:1054100080F00100012518702B46FEF7B3BF5C4DEC
:1054200005F1400830460AF0C7FC3368A5F8800053
:10543000591C1A46316012F8021B85F8821032603E
:105440005B7885F883300435A845EBD1FEF7B3BF10
:105450005A1C32604F4D1B782B7230460AF0ACFC60
:10546000A88330460AF0A8FC288330460AF0A4FC42
:1054700032686883531C33601278EA747268D31AF6
:10548000032B00F3CA843368D11A05290EDD5A1C98
:1054900032601B78EB7230460AF077FC3368E860C4
:1054A0005A1C32601B782B7433687268D21A002A37
:1054B0007EF781AF5A1C32601B7885F821300125B8
:1054C0002B46FEF75FBF581C3060334A1D781570BD
:1054D000091A00297EF76FAF991C31605B780033A1
:1054E00018BF0123012553702B46FEF74BBF3046F2
:1054F0000AF062FCDFF8BC80C8F8000030460AF011
:105500005BFCC8F8040030460AF056FC0125C8F8D8
:1055100008002B46FEF736BF5A1C32601D4A1B7826
:10552000537501252B46FEF72DBF591C31601D78A0
:105530001F2D3FF639AC052A7FF436AC30460AF011
:1055400024FC134B43F8250014F000FCFEF733BF96
:105550001A46591C3160114912F8020BC8703260AA
:105560000F495A784A71DA1C32600E4A9B78D37020
:1055700001252B46FEF706BFD4540020844E0020A0
:1055800058400020E8530020483F00202C1D0020F8
:105590005C8F002098840020805800200C5400204C
:1055A00018A100201C540020D8540020864E002052
:1055B0009C4E0020F835002030460AF0FDFB3046B6
:1055C0000AF0FAFB30460AF0F7FB30460AF0FFFB20
:1055D0003368C34D1946581C2A68306011F8020B15
:1055E00082F82C003160597882F83610D91C31606D
:1055F0009B7882F8373030460AF0E9FB30460AF0F3
:10560000E6FB30460AF0E3FB3046D5F800800AF0AE
:10561000D3FBA8F83A003046D5F800800AF0CCFB5E
:1056200033687268A8F83800D11A01290ADD591CBC
:105630002A6831601B7882F82E3030460AF0C7FBAA
:1056400033687268D31A032B0BDD3046D5F800801F
:105650000AF0B2FBA8F8320030462E680AF0ACFB24
:10566000B08628686AE45A1C32609D4DDFF8988243
:105670001B7888F805303046D5F800900AF09CFB7E
:10568000A9F820003046D5F800900AF095FB726822
:105690003368A9F81E00D11A072919DD30460AF02F
:1056A0008BFBA8F80A0030460AF086FBA8F80C002D
:1056B0003046D5F800900AF07FFBA9F8220030466A
:1056C000D5F800900AF078FB33687268A9F82400D6
:1056D000D11A03290BDD30460AF06EFBA8F80E0044
:1056E00030460AF069FB33687268A8F81000D21AD5
:1056F000002A05DD591C2A6831601B7882F82630A3
:10570000F6F76EFF22F0A4FB764B1B68002B00F02F
:1057100070832868012525F02DFD2B46FEF732BE4B
:105720001A46591C3160DFF8E08112F8021B88F834
:10573000021032606C495A780A70DA1C32606B4D84
:105740009A782A711A1D3260DB78092BA8BF0923C9
:105750003046AB700AF030FB336872682880D11A8B
:10576000012905DD30460AF027FB33687268E881BD
:105770009A4207D05A1C32601B78003318BF0123AD
:1057800088F80730F6F72CFF336872689A423EF4C7
:1057900012AE5A1C32601B78EB7001252B46FEF7C7
:1057A000F1BD5A1C32601B78002B00F02D834FF4A2
:1057B0000040012507F0C4F82B46FEF7E3BD4C4A34
:1057C000127812F001017FF4EFAA5A1C32601878A7
:1057D000012513F0A1FB2B46FEF7D4BD1A46591C38
:1057E000316012F8025B3260DA1C587832609978C6
:1057F000002D00F08B83012D7EF4DDAD13F04CFC09
:105800002B46FEF7BFBD01250BF046FA2B46FEF7EF
:10581000B9BD1A46591C374D316012F8021B297167
:1058200032605B786B7130460AF0C6FA33682880C4
:105830005A1C32601B78AB7130460AF0BDFA3368EF
:1058400068805A1C32601B78EB7101252B46FEF7ED
:1058500099BD294A03F108010133336013F8010CA3
:1058600002F8010F8B42F7D1FEF7A5BD1A46581C6E
:105870003060224812F8025B857032605D784570B6
:105880008A423EF498ADDA1C32601D4A9B7813744C
:1058900001252B46FEF776BD1A4BFFF791B83388EA
:1058A000FF2BA8BFFF23DBB2FEF703BD16F028F8DD
:1058B00000283EF4FDAC03780A2B3ED8B0F9023044
:1058C00088FB0312DB17C3EBA2039BB2FF2BA8BF1D
:1058D000FF23DBB2FEF7EDBC98E82200FFF772B8B9
:1058E000004D00207C58002000540020D05900209A
:1058F000D05400202CA70020978400202C54002096
:1059000028240020EC260020AC8D002015F0F8FFA4
:1059100000283FF43EA803780A2B3FF63AA8B0F9D6
:105920000430B0F9061003EB830383F3500521EA3A
:10593000E171ADB289B2FFF72EB80023C9E75A1C56
:1059400032601A780A2A00F0D28130460AF03FFA13
:1059500030460AF03CFA012530460AF038FA2B4668
:10596000FEF710BD1A46591C3160BE4D12F8021BDD
:10597000697032605A782A70DA1C32609B78AB709A
:1059800030460AF019FA33682881591C1A463160EA
:1059900012F8021B697132605B78AB7101252B46EE
:1059A000FEF7F0BC5A1C32601B780A2B00F099817C
:1059B000502B7FF40CA930460AF0FEF9DFF8BC82C8
:1059C000A8F8000030460AF0F7F90125A8F802000F
:1059D0002B46FEF7D7BC726835687B623046551B94
:1059E0000AF0D3F9052D38627B6A00F26E818026B9
:1059F000B346012594E80600521A103AB242B8BFE5
:105A00001FFA82FB984A396A92683A61521A9345A2
:105A1000396A7B622046FA6088BF1FFA82FB0AF06F
:105A200009FA7B6A002B00F02F81002D40F0F380F3
:105A30002368C7F800D05D71C0B00533C7F808D03F
:105A4000FB61BBF1000F00F008823B6A3A699342A8
:105A500080F01E82AA463E6A7D627C6080255446A4
:105A6000FB681C1B804BB4F5807F28BF4FF480740B
:105A70009B6832199A4288BF9C1B0BF081F8224622
:105A8000BC68304621460AF041FFF969B86104EB71
:105A9000000C0B787B6164452ED2DFF8E4910CF1A9
:105AA000FF3C04F1FF3E1EF8013F09EB830219F8A9
:105AB00023405688ECB100234FF4004204F1FF3834
:105AC00016424FEA520202D00878284308706D0847
:105AD00006D10AF1010A4D701FFA8AFA01318025B8
:105AE000D34503D8F44533D8984531DC01339C4283
:105AF000E6D1F445D7D1F9617B6ABA6913449BB208
:105B0000D3457B6206D97B6A3A6A1C46D6183B6944
:105B10009E42A5D37C68802D1CBF0AF101031FFAA9
:105B200083FA0AF1020189B220460AF09AF9236841
:105B3000796A01255A19226020461D700AF091F9F0
:105B40002368534423602B46D7F800D0FEF71ABCD5
:105B5000FB697C681A463B7D1370DCE7336872682A
:105B60009A4240F00881414BFF221A704FF0000A20
:105B70003F4D12F073F9514620223E4885F800A0AF
:105B80002EF063FC87F82CA097F82C30072B00F23E
:105B90002981DFF8F090374E524697F82C3003EB0E
:105BA000430309EBC3035B7CE3B197F82C3003EBB1
:105BB000430309EBC30320215B699BB197F82C30A9
:105BC00003EB430309EBC303586946F82200F8F7D7
:105BD00033FB2B7856F82300F8F7ECFB2A780132D8
:105BE000D2B22A7097F82C300133DBB287F82C3010
:105BF00097F82C30072BD0D92368591C21601A70D4
:105C0000B8F1000F3EF4D7AB1B4BC8F800300125AC
:105C10002B46FEF7B7BB144B3A6A9B68D4F800904A
:105C20005A449A4272D93A6AA3EB02080AF0A8FFD2
:105C300042464946386A0AF069FE236803442360F5
:105C4000002D3EF4B8ABB042BEF6B5AB002100E08B
:105C5000236801305A1CB04222601970F8D1FEF757
:105C6000AABB00BF844C002060170020282400201D
:105C7000113A0020FC36002099220208E826002074
:105C80003446040810590020002DC4D1594620463E
:105C90000AF0E7F823685A1C22601D709E4B2668A4
:105CA0009D683B6A0BEB0302AA4200F216810AF0E0
:105CB00067FF5A463146386A0AF028FE23680125F4
:105CC000034423602B46FEF75DBB30460AF074F8B0
:105CD000326871687B6A9142834675D106461D46DB
:105CE00088E630460AF068F8DFF8648268E69A1CB5
:105CF00032608A4A59781170D91C31609978517094
:105D0000191D3160DB789370FEF755BB0AF038FF40
:105D10005A464946386A0AF0F9FD2368034423606D
:105D200091E77F4B93E84200FEF7EBBE0AEBC80B0E
:105D300030468BF802100AF03FF832682AF8380033
:105D40001346511C316013F8021B8BF803103360AB
:105D500053788BF80430D31C336093788BF806307B
:105D6000131D33600135D2788BF80520A9457FF4E7
:105D700011AAFEF720BB5A1C19463260694811F877
:105D8000022B027031605B784370042A03D9FF2A2A
:105D90007EF4BDAAEAE664490978994205D8022A48
:105DA0007EF4B5AAFF2B7EF4B2AA236801255A1906
:105DB00022601D70B8F1000F3EF4FDAA5B4BC8F8DD
:105DC00000302B46FEF7DEBA511C316012781D46BA
:105DD000131C064618BF01230CE6524B59689E68F7
:105DE000FEF78FBE524607E70A7802F0FD02FFF782
:105DF000B3B84F484F49504A504B036001250B60E0
:105E000013602B46FEF7BEBA4D4A1368012523F4F2
:105E1000004313602B46FEF7B5BA304609F0CCFFBD
:105E2000A884304609F0C8FF33687268E884D11A44
:105E300003297FF729AB1A46591C316012F8021B5F
:105E4000A97732605B7885F82030304609F0B4FFDE
:105E5000336872686884FFF717BBDA46C7F824B066
:105E60005FE62F4B1020C3F800905D6006F038FD10
:105E7000344A137843F001031370B8F1000F3EF475
:105E80009AAA314B0125C3F800802B46FEF77ABA57
:105E90007D62AA4645E6042A7EF48DAAFFF74CB936
:105EA0002A4A99781288012512FB00F22B4692FBB0
:105EB000F1F2A8F80020FEF765BAC50800F0070364
:105EC00001350133EDB2DFF88C802846194688F899
:105ED000013015F099FCFFF7DEB93B6AED1A0AF0C4
:105EE0004FFE2A463146386A0AF010FD2368034403
:105EF0002360FEF760BA00F07F00032828BF00206F
:105F0000012513F0E5F82B46FEF73CBA012525F0F4
:105F100027FB2B46FEF736BA60170020514D0020B4
:105F2000E047002028240020A9490020B5B401083A
:105F3000B4A1002008A2002008A6002093EE0108CA
:105F4000F84C0020FE4C002024260020DCBB002062
:105F5000FC530020D85400202DE9F04F2DED0C8B80
:105F6000DFF8A89395B0D9F80430049048469847D4
:105F7000002875D0B9F8A850002289F85120002DCA
:105F800041F0F685D9F84830B9F93C60B9F93800E4
:105F9000D9F82050B9F93A10D9F82440DFF870A3A5
:105FA000F71A87EAE772A2EBE772B2F5804FD9F8E9
:105FB0002820DCBFC9F848603346401B091B9B1AE8
:105FC000C9F82C00C9F83010B54899F85210C9F832
:105FD00034301DF03FFDDAF80030990041F1298797
:105FE000D9ED0C5ADFF82CB3D9ED0B7AAD4A9BED05
:105FF000406ADBED416A9BED427ADBF80C311268B6
:10600000B8EEE58AD9ED0D5AF8EEE77AF8EEE58AB2
:10601000013377EE867A38EE268A78EE878A9342C5
:10602000CBED407A8BED418ACBED428ACBF80C3137
:1060300002F073849C4B02931E78142E03F0D283DB
:10604000DBF814214FF00008062A01F22483DFE870
:1060500012F09F1760186B167118A60A3117CB162D
:10606000914BDFF8B0B21C780293072C01F06683E5
:106070009BF82131069353B1581E8BF82101012C56
:1060800001F08B8615B0BDEC0C8BBDE8F08F874B13
:106090005B79002B01F0C883854B1B78013BDBB299
:1060A000072C8BF8213102F0F98400230893814AF0
:1060B000DBF82C31D2ED006A7F4A9FED806AD2F87E
:1060C00000A07F4A0592049ADBED4AAA7D4F9BED22
:1060D000499A9FED7DAADFED7DBA9FED7DCA9FEDC8
:1060E0007DBADFF834827C4ECBF82C21D31A07EE30
:1060F000903AF8EE677AB7EE007AC6EE279A07F183
:106100001C0300240793754B0393254677EE6A8A98
:1061100068EEA68AF4EEC78AF1EE10FA88BFF0EEB8
:10612000478A6F4B97ED008A2344D3ED007AF5EE52
:10613000407AF1EE10FA17D06A4B234493ED007ABF
:1061400078EE476AB0EEE66AF4EEC67AF1EE10FA3F
:1061500008D5F5EEC06AF1EE10FACCBF37EE878AAB
:1061600037EE678A83ED008A5F4B1A8893073FD02A
:10617000022D3DD05D4B9AF82E1033F9153007EE05
:10618000103A079B07EE901A2344F8EEE76AB8EE40
:10619000C77AD3ED007A4B42A6EEA77A680007EEE5
:1061A000903AF8EEE77AB4EEE77AF1EE10FA0AD414
:1061B00007EE901AF8EE677AF4EEC77AF1EE10FA6D
:1061C00088BFF0EE477A4A4B4A490344085EB3F968
:1061D0000C30C01A07EE100AB8EEC77AD007E7EE07
:1061E0004A7A41F1B582444B93ED008A27EE888AC2
:1061F000059B9BF86421234493ED01DA78EE4DCAA8
:10620000002A00F0CB803D4BDBF8682104991B6825
:106210008A1A9A4240F3C2809AF84830022B02F060
:106220008784022D05F02C80354B1B68990775D4A7
:10623000344B86ED00CA1B689342C0F2A980F7EE8A
:10624000007AF4EEE7AAF1EE10FA40F1A780059982
:106250002D4BD1ED017A93ED007AF0EEE77AF4EE72
:10626000C77AF1EE10FA40F19980D1ED027AF0EEA2
:10627000E77AB4EEE77AF1EE10FA40F38F80D1EDD1
:10628000037AF0EEE77AB4EEE77AF1EE10FA40F333
:1062900085801B4B1B689A077AD51649144B5EE024
:1062A000FC85002068550020C8490020AC8D0020E6
:1062B000005400205CA60020004D002000247449FA
:1062C000C08D002088250020CDCCCC3DAE47813F3D
:1062D000000000000000C842DC510020D051002026
:1062E00050A6002094250020FC4C0020A025002072
:1062F0000C540020AC4C002038A6002064A60020DE
:10630000A04C002060A600206CA60020D0850020B4
:10631000D08D002058240020E8510020D74BD849C8
:10632000DFF8CCE331F915C09EED008ADFF8C4E355
:1063300086ED00CA03EB450028EE0A8AB0F90C008E
:10634000A0EB0C0007EE900AF8EEE77ADEF800000A
:1063500027EE888A904278EE4DCABFF670AFB3F947
:106360000C20B1F900E0C748AEEB020E00688EEADF
:10637000EE72A2EBEE72824210DAB3F90E30B1F98E
:106380000220D21A82EAE273A3EBE273984205DD9F
:10639000002318468BF86431F8F71AF8BA4B2344F7
:1063A00093ED000A039B29EE000A022D20EE2C0A31
:1063B000A3EC010A039304F00587B44BD6ED006A01
:1063C00093ED007AB24BD3ED007AB24B93ED006AB5
:1063D000B14B67EE277A234427EEA87AD3ED007AF3
:1063E00067EE277AF0EE665AECEEA75AB1EE467ADF
:1063F000F4EEC75AF1EE10FA08D4F4EEC65AF1EEF4
:1064000010FA8CBFB0EE467AB0EE657A9BED4A6A20
:10641000F7EE007AB4EEE76AF1EE10FAACBF0123B2
:10642000002343B1F0EEE66AF0EEC77AF4EEE67AC6
:10643000F1EE10FA01D586ED007A022D04F0AE8659
:10644000964A974B52F825001B68B0EE4D0A9847C4
:10645000944A954B52F825001B6898479AF83730B4
:1064600023B1924B1B88002B01F07282B0EE4C8A54
:106470008F4B38EE400A234493ED008A83ED000AE7
:106480009AF8483030EE480A20EE298A53B3894BF7
:106490001B78DB0741F17680F7EE007AF4EEE7AA8D
:1064A000F1EE10FA9BF86431C1F2B087002B01F0D5
:1064B0000383DBF86831049AD31A7F4A12689A4240
:1064C00010DD7E4BD3ED007AF0EEECCAF4EEE7CAB5
:1064D000F1EE10FA42F13583002318468BF864314F
:1064E000F7F776FF764B9BF87421234493ED000A6F
:1064F00029EE000A20EE088A88ED008A32B9039B53
:1065000086ED00CA03ED01CA88ED00CA0135032DEE
:1065100007F1040708F1040806F1040604F1040475
:106520007FF4FFAD029B1B78072B01F08487012BC2
:1065300002F0A282002307939BF87C31002B41F0EC
:106540006084604BDFF8B0A11A68DAF8003092F886
:106550002C10D80401F128825B4B5C4803931C4645
:106560005B4B648B90ED006AD3ED005A59485A4B4F
:10657000D0ED007A93ED005AD0ED013AD0ED024A09
:106580008BED636A07EE104A544C8BED616AD4EDD3
:10659000036ACBED645AB8EEC77A35EEC64A0123DA
:1065A00036EEC77A8BED604A8BF89431C7EE055A08
:1065B000138D584206EE100A4948DFED4A6A90ED05
:1065C000005A494890ED004AB7EE007AF4EEC75AF7
:1065D00035EE045AF1EE10FA88BFF0EE475A35EE68
:1065E000275AB8EEC66AF4EEE65AF1EE10FA07EE54
:1065F000903AB4EEC65AB8BFF0EE665AF1EE10FA11
:10660000CBED675AB8EE677A01F17585B4EEC75ADB
:10661000F1EE10FA88BFB0EE475A314BDFED336A26
:10662000D3ED017A304B93ED014A77EE847A25EE73
:10663000265A77EEA37AB4EEE76AF1EE10FA08DC98
:10664000B4EEE77AF1EE10FA8CBFB0EE676AB0EE06
:10665000476A538D224A9FED257AD2ED027A5A423B
:1066600004EE102A74EEA77AB8EEC44A26EE076A42
:10667000F4EEC47AF1EE10FA4BD43FE00C54002053
:10668000AC4C002068A600200CA600209C00002036
:10669000B0A1002080A6002018A60020B8A10020EC
:1066A000B4A100200CA2002008A20020FC4C002075
:1066B000C4250020D054002064A6002070A600202D
:1066C00024A60020004D0020988400206C52002059
:1066D000E4530020DC51002018A70020C04A00200D
:1066E000D051002000000000E85100206F12833AD2
:1066F00038A6002060A60020D08D002007EE103ABA
:10670000B8EE474AB4EEE74AF1EE10FA88BFB0EEB1
:10671000674AEA4BDFEDEA7A5B7824EE274A0BB949
:10672000B1EE444A002942F0BC80B7EE003AE54E93
:106730003278002A03F03881E34BDFEDE47AD3EDC1
:10674000024AD3ED016A93ED037A66EE244AE5EE40
:10675000264AE4EE074A63EE244AF4EEE74AF1EEF5
:1067600010FAB4BFF0EE673AF0EE643A98BFF0EE7C
:10677000647A012ACDED0C4A03F0638193ED067A29
:10678000D3ED052AD3ED076A26EE077AA5EE227A25
:10679000A4EE267A23EE077AB4EEE77AF1EE10FA49
:1067A000B4EEE37A8CBFF0EE676AF0EE476AF1EE82
:1067B00010FA88BFF0EE676AB4BFF0EE637AF0EECD
:1067C000477A022A8DED0D7A00F0DE8093ED0A7A89
:1067D000D3ED092AD3ED0B3A26EE077AA5EE227AFD
:1067E000A4EE237A23EE077AB4EEE67AF1EE10FAFD
:1067F000B4EEE77A8CBFF0EE663AF0EE473AF1EE8F
:1068000010FA98BFF0EE636AA8BFF0EE477A032A49
:106810008DED0E7A00F0B88093ED0E7AD3ED0D2A4F
:10682000D3ED0F3A26EE077AA5EE227AA4EE237A6C
:1068300023EE077AB4EEE67AF1EE10FAB4EEE77AD8
:106840008CBFF0EE663AF0EE473AF1EE10FA98BFE0
:10685000F0EE636AA8BFF0EE477A042A8DED0F7A56
:1068600000F09280D3ED123AD3ED112A93ED137A12
:1068700066EE233AE5EE223AE4EE073A63EE233A77
:10688000F4EEE63AF1EE10FAF4EEE73A8CBFB0EE31
:10689000667AB0EE637AF1EE10FA98BFF0EE476ACE
:1068A000A8BFF0EE637A052ACDED103A6CD0D3ED97
:1068B000163AD3ED152A93ED177A66EE233AE5EEF4
:1068C000223AE4EE073A63EE233AF4EEE63AF1EECA
:1068D00010FAF4EEE73A8CBFB0EE667AB0EE637A67
:1068E000F1EE10FA98BFF0EE476AA8BFF0EE637AB7
:1068F000062ACDED113A47D0D3ED1A3AD3ED192A35
:1069000093ED1B7A66EE233AE5EE223AE4EE073A7F
:1069100063EE233AF4EEE63AF1EE10FAF4EEE73ADB
:106920008CBFB0EE667AB0EE637AF1EE10FA98BFE3
:10693000F0EE476AA8BFF0EE637A072ACDED123A6F
:1069400022D093ED1E7AD3ED1D2AD3ED1F3A26EE09
:10695000077AA5EE227AA3EE847A27EE037AB4EEC4
:10696000E67AF1EE10FAB4EEE77A8CBFB0EE666A22
:10697000B0EE476AF1EE10FA8DED137A98BFF0EEA3
:10698000466AA8BFF0EE477A77EEE67AF7EE006A3D
:10699000F4EEE67AF1EE10FACBED4A7A44F32C816C
:1069A00086EEA77A022ADDED0D7A67EE244A67EEBD
:1069B000877ACDED0C4ACDED0D7A2DD0DDED0E7A36
:1069C00067EE877A032ACDED0E7A25D0DDED0F7ABA
:1069D00067EE877A042ACDED0F7A1DD0DDED107AAF
:1069E00067EE877A052ACDED107A15D0DDED117AA4
:1069F00067EE877A062ACDED117A0DD0DDED127A99
:106A000067EE877A072ACDED127A05D0DDED137A8D
:106A100027EE877A8DED137A2D4B1B6813F0805883
:106A200001F0AB84F6EE005ACBED675A002A02F073
:106A3000B387284B28499BED646A0878D978089178
:106A400026490591B1F906109BF9943109910399F2
:106A5000234F9BED635A234D498B97F800C00A9151
:106A6000BDEEC66A07EE103ADAF800300899D5EDA7
:106A7000004ADBED606ADBED617A16EE107ABDEE5E
:106A8000C56A00F0010E03F4805503F0100003F412
:106A900080030B93B8EEC77A16EE103A002941F046
:106AA0000782002841F0C58507489DED0C5A90EDFE
:106AB000006A0D4925EE866A18E000BF8058002064
:106AC0006F12833AA949002088A600200000000028
:106AD000D0530020AC910020D0540020DCB900201D
:106AE000F459002084A6002030520020A5EE076A49
:106AF000B0EE675AA6EE265ABDEEC56A16EE10CA6B
:106B000016EE105ABC45A8BF3D466345C8BF1D469A
:106B100006EE105AB8EEC66A012A81ED006A00F04E
:106B2000DC8090ED046A9DED0D5A25EE866AA5EE97
:106B3000076AB0EE675AA6EE265ABDEEC56A16EE93
:106B400010CA16EE105ABC45A8BF3D466345C8BFE3
:106B50001D4606EE105AB8EEC66A022A81ED016A99
:106B600000F0BB8090ED086A9DED0E5A25EE866A16
:106B7000A5EE076AB0EE675AA6EE265ABDEEC56AC4
:106B800016EE10CA16EE105ABC45A8BF3D46634526
:106B9000C8BF1D4606EE105AB8EEC66A032A81ED3C
:106BA000026A00F09A8090ED0C6A9DED0F5A25EE76
:106BB000866AA5EE076AB0EE675AA6EE265ABDEEC3
:106BC000C56A16EE10CA16EE105ABC45A8BF3D465F
:106BD0006345C8BF1D4606EE105AB8EEC66A042AC1
:106BE00081ED036A79D090ED106A9DED105A25EE83
:106BF000866AA5EE076AB0EE675AA6EE265ABDEE83
:106C0000C56A16EE10CA16EE105ABC45A8BF3D461E
:106C10006345C8BF1D4606EE105AB8EEC66A052A7F
:106C200081ED046A59D090ED146A9DED115A25EE5C
:106C3000866AA5EE076AB0EE675AA6EE265ABDEE42
:106C4000C56A16EE10CA16EE105ABC45A8BF3D46DE
:106C50006345C8BF1D4606EE105AB8EEC66A062A3E
:106C600081ED056A39D090ED186A9DED125A25EE36
:106C7000866AA5EE076AB0EE675AA6EE265ABDEE02
:106C8000C56A16EE10CA16EE105ABC45A8BF3D469E
:106C90006345C8BF1D4606EE105AB8EEC66A072AFD
:106CA00081ED066A19D090ED1C6A9DED135A65EED0
:106CB000865AE7EE055AE6EEA57AFDEEE77A17EE7C
:106CC000900A8742A8BF07468342D8BF3B4607EEDB
:106CD000903AF8EEE77AC1ED077ABEF1000F01F0C5
:106CE000F581E44B1B68002B41F0FD81E24B1B78E2
:106CF00093B1307868B1E14FDFF8A8830025E8B29E
:106D0000D8F80030B7EC010A984730780135854251
:106D1000F5DBDB4B1B689847029B1B78072B01F0C8
:106D20007A8300230793DAF8008018F4806F41F02B
:106D30004582D44B059A1D68B2F906706A8997425C
:106D400081F211804FF07E53CBF82431DFF8589355
:106D5000059A039BB2F900001E8B99F9043099F84B
:106D6000001099F801E0002BA0EB060383EAE37C16
:106D7000ACEBE37C14BF01224FF0FF32BCF5FA7F8D
:106D8000A8BF4FF4FA7C614580F2E987ACEB0103C0
:106D900007EE903AF8EEE77A8642C4ED007A03DD1A
:106DA000F1EE677AC4ED007A059BB3F90200831B0C
:106DB00083EAE37CACEBE37CBCF5FA7FA8BF4FF43D
:106DC000FA7C614580F2C787ACEB010307EE903A8D
:106DD000F8EEE77AB042C4ED017A03DAF1EE677AB1
:106DE000C4ED017A059BB3F904108B1B83EAE370B1
:106DF000A0EBE370B0F5FA7FA8BF4FF4FA707045CE
:106E0000CCBFA0EB0E0E4FF0000E02FB0EFE07EE05
:106E100090EAF8EEE77AB142C4ED027ABCBFF1EE37
:106E2000677AC4ED027A18F4805A00F06F87B7F5DC
:106E3000FA6F3A46A8BF4FF4FA62B2F57A7F9BF830
:106E4000A431B8BF4FF47A72A2F57A72002B40F0E9
:106E500076878D49DFF854E281FB0230D317C3EB0C
:106E60006013581C6FF0630C3EF910003EF913E0FC
:106E70000CFB0323A0EB0E0003FB00F381FB0321BB
:106E8000DB17C3EB61139E440FFA8EFE07EE90EA08
:106E9000B8EEE78A84ED038ABAF1000F41F09B81D6
:106EA0007A4B1E8816F04003059300F0DD80784B86
:106EB0007849D3ED018A93ED026AD1ED020A91ED92
:106EC000043A93ED031AD3ED003A91ED030AD1EDA4
:106ED000015AD4ED011A94ED002A6F4B30EEC35ADB
:106EE00038EEC67A73EE817A25EE077A75EEC04ADF
:106EF00073EEC19A35EE80AA24EEA79AB0EE474A07
:106F0000AAEE294A16F00302B0EE495A78EE867AC4
:106F100070EE836AAAEE295AA6EEA74AA6EEE75AB1
:106F2000F0EE474AD6EEA74A34EE094AF6EE006A7A
:106F300073EEA8AA26EEC44A35EE475A35EEA07A7B
:106F4000F0EE647AEAEE694AA7EE2A4A77EEC97A49
:106F500036EE417A73EE40AA25EE265AEAEE297AF9
:106F6000AAEE875A74EE894A24EE047A73EEE83A60
:106F700033EE003A64EEA64A75EEE05A36EE016A48
:106F800067EEA66AF0EE477AE3EE234AD5EE057A7D
:106F9000A5EE057AE5EE866AF1EE648AB0EE476A00
:106FA000B0EE677AF1EE663AA8EEA47A64EE260AAD
:106FB00026EEA43AA3EEA66AB1EE450AE3EEA67A5F
:106FC000F0EE609AB0EE431A64EE243AA6EEA67A8A
:106FD000E5EE249AA0EE041AF0EE665AA8EEA46A32
:106FE000F0EE638A71EEA16AE0EE240AE5EE258AEE
:106FF00027EE217A32EE029AA5EE043A61EE211ACA
:1070000066EEA96AE4EEA47AE0EE253A0CBFD4ED70
:10701000022ADFED222A83ED005AE2EE066AA9EE8B
:10702000207AE2EE281A33EE033A67EEA27A73EE84
:10703000A33AB0EE006AA3EE227AE3EEA26AE1EE92
:10704000867A8BED6C7A84ED017ACBED6B6AC4EDB8
:10705000006ACBED6D7A83ED014AC3ED025AC3EDB0
:10706000034A0AB9C4ED027A0D4B1B6813F0140FE2
:107070001EE000BFBC5100201C5D002030520020EB
:10708000F0590020044D00201F85EB51FC4C0020DE
:10709000541C00209C0000208C1C002000000000DC
:1070A000A04C0020E85900200454002034A7002000
:1070B00003D016F4027F41F0F080DA4A12789AB1D8
:1070C000039A528BBA420FDBD74A1278012A01F099
:1070D000FA84192A01F0F7840E2A05D0082A03D071
:1070E0000022A260CBF838219BF8DA7117B1B20701
:1070F00041F0A8849BF8E071002F41F00080039AD2
:10710000927F002A00F0F985022A01F0FF83032A0A
:1071100041F0F883039A92F82020C2EB421102EB6F
:107120008101C90089B2039AD27F0232D2B2002F04
:1071300000F08486002900F08186BC4B1B68B1FBFF
:10714000F3F10FFA81F8ABF81082AAB307EE908A38
:10715000F8EEE77AF7EE006A86EEA77A012AD4ED18
:10716000007ADBED896A77EEE67A67EE877ACBED17
:10717000857A21D0D4ED017ADBED8A6A77EEE67A62
:10718000022A67EE877ACBED867A15D0D4ED027AA3
:10719000DBED8B6A77EEE67A032A67EE877ACBED32
:1071A000877A09D0D4ED037ADBED8C6A77EEE67A44
:1071B00067EE877ACBED887A029B1B78092B03F068
:1071C0009F83B8F1000F40F39E859AB39BED897AB7
:1071D000DBED857A77EE877A012ACBED897AC4EDEB
:1071E000007A21D09BED8A7ADBED867A77EE877A7A
:1071F000022ACBED8A7AC4ED017A15D09BED8B7A09
:10720000DBED877A77EE877A032ACBED8B7AC4EDB4
:10721000027A09D0DBED8C7A9BED887A77EE877A5B
:10722000CBED8C7AC4ED037A013A022AB8BF022270
:10723000D3B20693002F069818BF02202B78DFEDFB
:10724000806AAA7807EE903AF8EEE77AB0EE007A14
:1072500067EEA67A029BF4EEC77AF1EE10FA19787F
:1072600040F34587DFED736A37EEC77AB0EE676AA1
:10727000A7EE266AF0EE466A94ED007A9FED6E6AFC
:1072800027EE066AF0EEC65A8BED536ACBED565ADE
:107290009AB107EE102AB8EEC75A9FED697A66EEEA
:1072A000064A25EE075AB7EE007A37EE457A64EEC5
:1072B000A54AA5EE247A26EE076A9FED607A6B79DF
:1072C00026EE877A27EE067ACBB1DFED5D6A9FED79
:1072D0005D6A65EEA65A06EE903AF8EEE66A65EE4D
:1072E000A65AF4EEC65AF1EE10FA01F3AA82B7EEEE
:1072F000006A76EE655AC6EE256A27EE267A0C29D4
:107300009FED518ADFED516A01F04680B4EEC87AF4
:10731000F1EE10FA98BFB0EE478AB4EEE68AF1EECD
:1073200010FAB8BFB0EE668A8BED4C8A002800F0E8
:10733000F580B0EE007AF4EEC77AF1EE10FA05DDD2
:1073400037EEC77ADFED3B6AE7EE267A94ED017AF5
:10735000DFED396A27EE267AF0EEC75A8BED547AC4
:10736000CBED575A9AB106EE902A9FED356AF8EEAA
:10737000E66A27EE075A66EE866AB7EE006A36EED0
:10738000666A25EE255AA6EE856A27EE067ADFEDB7
:107390002B6AAB7967EEA67A67EE877AABB107EE18
:1073A000103AB8EEC77A9FED266ADFED266A27EE1F
:1073B000257A27EE067AB4EEE67AF1EE10FA41F37A
:1073C0005982DFED1B6A67EEA67A0C2900F0FF8771
:1073D000DFED1D6A9FED1D7AF4EEE67AF1EE10FA0C
:1073E00088BFF0EE667AF4EEC77AF1EE10FAB8BF15
:1073F000F0EE477A0128CBED4D7A40F38F806B7821
:10740000DFED0F6A07EE903AF8EEE77AB0EE007A19
:1074100067EEA67A6B7AF4EEC77AF1EE10FA1DDD0C
:1074200016E000BF2C1D0020805800207C58002052
:107430000000C842D7A368416F12033B00004843D5
:107440000AD7233CA4707D3F00C0F94400C0F9C4B2
:1074500037EEC77A5FED096AE7EE267A94ED027A95
:107460005FED0B6A27EE267AF0EEC75A8BED557A60
:10747000CBED585A9BB106EE903A1FED0F6AF8EE2D
:10748000E66A27EE075A66EE866AB7EE006A36EEBF
:10749000666A25EE255AA5EE266A27EE067A5FED86
:1074A000196AEB7967EEA67A67EE877AFBB107EE89
:1074B000103AB8EEC77A1FED1E6A5FED1E6A27EE1E
:1074C000257A27EE067AB4EEE67AF1EE10FA01F3A9
:1074D000BC81B5EEC07AF1EE10FA02F16784B7EE26
:1074E000006A36EE477AC6EE076A67EEA67A0C297E
:1074F00000F04A875FED2C6A1FED2C7AF4EEE67AF5
:10750000F1EE10FA88BFF0EE667AF4EEC77AF1EE8B
:1075100010FAB8BFF0EE477ACBED4E7A092900F0A9
:107520001E87039B93F82140002C40F0D386C04B6C
:1075300000221B688BF8E0219A0607D516F0300F61
:1075400004D0BC4B1B78DB0702F15B8127F042FCC7
:10755000002840F02F84B84B1B7823B9B74B9B7899
:10756000002B41F08482029B1C78072C7EF487ADAF
:10757000F6F726FA029AB24B1478079A801AD88046
:10758000FEF77DBD9BF86431002B3EF4ABAF0023CA
:1075900018468BF86431F6F71BFFFEF7A3BFA94B23
:1075A0001978DBF81851A84C9FEDA87AEE00A319C2
